:040000000DEF00F010
:04000800CFEF4BF0FB
:0A001800FF0011EECFF0D9EF5CF00D
:10100000000200000100E652E652E652FB0E6F00BD
:101010008FFFE6FF6F008FFFE6FFC2EC5EF0FE0E73
:101020006000BFF0E3FFFD0E6000BBF0E3FFFD0ECC
:101030006F008FFFF6FFFE0E6F008FFFF7FF000EB1
:10104000F86E0F0EF76403D00800F55007D06F005C
:10105000DBFFE9FF6F00DFFFEAFFEF50396EFF0EA5
:101060006000E7F0E3FFFB0E6F008FFFE6FF6F000D
:101070008FFFE6FF82EC5FF0FB0E6F008FFFE6FF55
:101080006F008FFFE6FF24EC5EF0F80EE126FF0E06
:10109000E22230EF0DF0FD0EE350010F386EFE0E30
:1010A0006F008CFF39F0000E39226000E3F0E6FF9C
:1010B0006000E7F0E6FF28EC50F0FB0E6F008FFFBA
:1010C000D9FFFC0E6F008FFFDAFFDF50140AD8A49F
:1010D0006CEF08F06EEF08F087EF08F0FD0E6F0080
:1010E0008FFFF6FFFE0E6F008FFFF7FF000EF86E0A
:1010F0000F0EF76404D0150EF56E0C0008D06F00CB
:10110000DBFFE9FF6F00DFFFEAFF150EEF6EFB0E5E
:101110006F008FFFD9FFFC0E6F008FFFDAFFDF50EB
:10112000150AD8A496EF08F098EF08F06FEF0DF0CD
:10113000FD0E6F008FFFF6FFFE0E6F008FFFF7FFB3
:10114000000EF86E0F0EF76404D0190EF56E0C0049
:1011500008D06F00DBFFE9FF6F00DFFFEAFF190E29
:10116000EF6E000EE66E000EE66E000EE66E000EEE
:10117000E66E000EE66E000EE66E000EE66E000EE7
:10118000E66EF50EE3501E0F386EF60E6F008CFF04
:1011900039F0000E39226000E3F0F6FF6000E7F05E
:1011A000F7FF000EF86E0F0EF76403D00800F5503D
:1011B00007D06F00DBFFE9FF6F00DFFFEAFFEF50B2
:1011C0000A0D6F00CCFF38F06F00D0FF39F06000DF
:1011D000E3F0E6FF6000E7F0E6FFF30E6F008FFF3D
:1011E000E6FF6F008FFFE6FF79EC5AF06FEF0DF02E
:1011F000FB0E6F008FFFD9FFFC0E6F008FFFDAFF31
:10120000DF50160AD8A407EF09F009EF09F06FEFD5
:101210000DF0FD0E6F008FFFF6FFFE0E6F008FFFCB
:10122000F7FF000EF86E0F0EF76404D0160EF56E81
:101230000C0008D06F00DBFFE9FF6F00DFFFEAFF63
:10124000160EEF6E6FEF0DF0FB0E6F008FFFD9FFE4
:10125000FC0E6F008FFFDAFFDF50170AD8A433EFC0
:1012600009F035EF09F06FEF0DF0FD0E6F008FFF05
:10127000F6FFFE0E6F008FFFF7FF000EF86E0F0EE9
:10128000F76404D0170EF56E0C0008D06F00DBFF7A
:10129000E9FF6F00DFFFEAFF170EEF6E000EE66E4C
:1012A000000EE66E000EE66E000EE66E000EE66EB6
:1012B000000EE66E000EE66E000EE66EF50EE350D2
:1012C0001E0F386EF60E6F008CFF39F0000E3922BB
:1012D0006000E3F0F6FF6000E7F0F7FF000EF86E45
:1012E0000F0EF76403D00800F55007D06F00DBFF46
:1012F000E9FF6F00DFFFEAFFEF50140D6F00CCFF36
:1013000038F06F00D0FF39F06000E3F0E6FF6000D6
:10131000E7F0E6FFF30E6F008FFFE6FF6F008FFF31
:10132000E6FF79EC5AF06FEF0DF0FB0E6F008FFFC8
:10133000D9FFFC0E6F008FFFDAFFDF50180AD8A428
:10134000A4EF09F0A6EF09F06FEF0DF0FD0EE350EA
:101350001E0F386EFE0E6F008CFF39F0000E392222
:101360006000E3F0F6FF6000E7F0F7FF000EF86EB4
:101370000F0EF76403D00800F55007D06F00DBFFB5
:10138000E9FF6F00DFFFEAFFEF500009D8A4CBEFC1
:1013900009F0CDEF09F00FEF0AF0FD0EE3501D0F3D
:1013A000386EFE0E6F008CFF39F0000E392260009F
:1013B000E3F0F6FF6000E7F0F7FF000EF86E0F0EA7
:1013C000F76403D00800F55007D06F00DBFFE9FF9A
:1013D0006F00DFFFEAFFEF500009D8B4F2EF09F029
:1013E000F4EF09F0AFEF0AF0FD0E6F008FFFF6FF8C
:1013F000FE0E6F008FFFF7FF000EF86E0F0EF76402
:1014000004D01A0EF56E0C0008D06F00DBFFE9FF68
:101410006F00DFFFEAFF1A0EEF6EAFEF0AF0FD0E6E
:10142000E3501A0F386EFE0E6F008CFF39F0000E7D
:1014300039226000E3F0F6FF6000E7F0F7FF000EEE
:10144000F86E0F0EF76403D00800F55007D06F0058
:10145000DBFFE9FF6F00DFFFEAFFEF500009D8B4C0
:1014600034EF0AF036EF0AF096EF0AF0FD0E6F0047
:101470008FFFF6FFFE0E6F008FFFF7FF000EF86E76
:101480000F0EF76404D0170EF56E0C0008D06F0035
:10149000DBFFE9FF6F00DFFFEAFF170EEF6E000EC4
:1014A000E66E000EE66E000EE66E000EE66E000EB4
:1014B000E66E000EE66E000EE66E000EE66EF50EAF
:1014C000E3501E0F386EF60E6F008CFF39F0000EE1
:1014D00039226000E3F0F6FF6000E7F0F7FF000E4E
:1014E000F86E0F0EF76403D00800F55007D06F00B8
:1014F000DBFFE9FF6F00DFFFEAFFEF50140D6F0025
:10150000CCFF38F06F00D0FF39F06000E3F0E6FF69
:101510006000E7F0E6FFF30E6F008FFFE6FF6F005D
:101520008FFFE6FF79EC5AF0AFEF0AF0FD0E6F0087
:101530008FFFF6FFFE0E6F008FFFF7FF000EF86EB5
:101540000F0EF76404D0180EF56E0C0008D06F0073
:10155000DBFFE9FF6F00DFFFEAFF180EEF6EFD0E05
:10156000E3501A0F386EFE0E6F008CFF39F0000E3C
:1015700039226000E3F0F6FF6000E7F0F7FF000EAD
:10158000F86E0F0EF76404D0000EF56E0C0008D054
:101590006F00DBFFE9FF6F00DFFFEAFF000EEF6E79
:1015A0006FEF0DF0FB0E6F008FFFD9FFFC0E6F0089
:1015B0008FFFDAFFDF501A0AD8A4E1EF0AF0E3EF59
:1015C0000AF06FEF0DF0FD0E6F008FFFF6FFFE0EBD
:1015D0006F008FFFF7FF000EF86E0F0EF76404D058
:1015E000150EF56E0C0008D06F00DBFFE9FF6F00F1
:1015F000DFFFEAFF150EEF6E6FEF0DF0FB0E6F00D1
:101600008FFFD9FFFC0E6F008FFFDAFFDF50180A43
:10161000D8A40DEF0BF00FEF0BF06FEF0DF0FD0EF8
:10162000E3502F0F386EFE0E6F008CFF39F0000E66
:1016300039226000E3F0F6FF6000E7F0F7FF000EEC
:10164000F86E0F0EF76409D009006F00D4FF38F070
:1016500009006F00D4FF39F00CD06F00DBFFE9FF09
:101660006F00DFFFEAFF6F00B8FF38F06F00B8FFD0
:1016700039F038503910D8B440EF0BF042EF0BF08E
:10168000A8EF0BF0FD0EE350310F386EFE0E6F0029
:101690008CFF39F0000E39226000E3F0F6FF6000A5
:1016A000E7F0F7FF000EF86E0F0EF76409D009009F
:1016B0006F00D4FF38F009006F00D4FF39F00CD070
:1016C0006F00DBFFE9FF6F00DFFFEAFF6F00B8FF8D
:1016D00038F06F00B8FF39F06000E3F0E6FF60001B
:1016E000E7F0E6FFFB0EE3502F0F386EFC0E6F00A5
:1016F0008CFF39F0000E39226000E3F0F6FF600045
:10170000E7F0F7FF000EF86E0F0EF76409D009003E
:101710006F00D4FF38F009006F00D4FF39F00CD00F
:101720006F00DBFFE9FF6F00DFFFEAFF6F00B8FF2C
:1017300038F06F00B8FF39F002D8A8EF0BF00500C1
:10174000FA6E3850FD6E3950FE6EFF6AFA50120084
:10175000FD0EE3501E0F386EFE0E6F008CFF39F049
:10176000000E39226000E3F0F6FF6000E7F0F7FFBB
:10177000000EF86E0F0EF76403D00800F55007D086
:101780006F00DBFFE9FF6F00DFFFEAFFEF500009AA
:10179000D8A4CDEF0BF0CFEF0BF011EF0CF0FD0E56
:1017A000E3501D0F386EFE0E6F008CFF39F0000EF7
:1017B00039226000E3F0F6FF6000E7F0F7FF000E6B
:1017C000F86E0F0EF76403D00800F55007D06F00D5
:1017D000DBFFE9FF6F00DFFFEAFFEF500009D8B43D
:1017E000F4EF0BF0F6EF0BF06FEF0DF0FD0E6F0066
:1017F0008FFFF6FFFE0E6F008FFFF7FF000EF86EF3
:101800000F0EF76404D01A0EF56E0C0008D06F00AE
:10181000DBFFE9FF6F00DFFFEAFF1A0EEF6E6FEFED
:101820000DF0000EE66E000EE66E000EE66E000E87
:10183000E66E000EE66E000EE66E000EE66E000E20
:10184000E66EF50EE3501E0F386EF60E6F008CFF3D
:1018500039F0000E39226000E3F0F6FF6000E7F097
:10186000F7FF000EF86E0F0EF76403D00800F55076
:1018700007D06F00DBFFE9FF6F00DFFFEAFFEF50EB
:10188000140D6F00CCFF38F06F00D0FF39F060000E
:10189000E3F0E6FF6000E7F0E6FFF30E6F008FFF76
:1018A000E6FF6F008FFFE6FF79EC5AF06FEF0DF067
:1018B000FB0E6F008FFFD9FFFC0E6F008FFFDAFF6A
:1018C000DF50190AD8A467EF0CF069EF0CF06FEF46
:1018D0000DF0000EE66E000EE66E000EE66E000ED7
:1018E000E66E000EE66E000EE66E000EE66E000E70
:1018F000E66EF50EE3501E0F386EF60E6F008CFF8D
:1019000039F0000E39226000E3F0F6FF6000E7F0E6
:10191000F7FF000EF86E0F0EF76403D00800F550C5
:1019200007D06F00DBFFE9FF6F00DFFFEAFFEF503A
:101930000A0D6F00CCFF38F06F00D0FF39F0600067
:10194000E3F0E6FF6000E7F0E6FFF30E6F008FFFC5
:10195000E6FF6F008FFFE6FF79EC5AF0FD0EE350D3
:101960001B0F386EFE0E6F008CFF39F0000E39220F
:101970006000E3F0F6FF6000E7F0F7FF000EF86E9E
:101980000F0EF76403D00800F55007D06F00DBFF9F
:10199000E9FF6F00DFFFEAFFEF500009D8B4D3EF93
:1019A0000CF0D5EF0CF0EEEF0CF0FD0E6F008FFF9A
:1019B000F6FFFE0E6F008FFFF7FF000EF86E0F0EA2
:1019C000F76404D0170EF56E0C0008D06F00DBFF33
:1019D000E9FF6F00DFFFEAFF170EEF6EFD0EE35029
:1019E0001C0F386EFE0E6F008CFF39F0000E39228E
:1019F0006000E3F0F6FF6000E7F0F7FF000EF86E1E
:101A00000F0EF76403D00800F55007D06F00DBFF1E
:101A1000E9FF6F00DFFFEAFFEF500009D8B413EFD2
:101A20000DF015EF0DF06FEF0DF0FD0E6F008FFF55
:101A3000F6FFFE0E6F008FFFF7FF000EF86E0F0E21
:101A4000F76404D0190EF56E0C0008D06F00DBFFB0
:101A5000E9FF6F00DFFFEAFF190EEF6E6FEF0DF089
:101A6000FD0E6F008FFFF6FFFE0E6F008FFFF7FF7A
:101A7000000EF86E0F0EF76403D00800F55007D083
:101A80006F00DBFFE9FF6F00DFFFEAFFEF50386E0A
:101A9000396A3950000AD8B450EF0DF06FEF0DF0ED
:101AA0003850140AD8B44BEF08F0010AD8B4F8EF54
:101AB00008F0030AD8B424EF09F0010AD8B495EF6E
:101AC00009F00F0AD8B4D2EF0AF0010AD8B4FEEF39
:101AD0000AF0030AD8B458EF0CF06FEF0DF0FF0EC8
:101AE0006F008CFF39F0FD0E6F008FFFF6FFFE0ECA
:101AF0006F008FFFF7FF000EF86E0F0EF76403D034
:101B00000800F55007D06F00DBFFE9FF6F00DFFF33
:101B1000EAFFEF503918D8B490EF0DF092EF0DF0C6
:101B2000C0EF11F0BCEF0DF0FD0EE350020F386E68
:101B3000FE0E6F008CFF39F0000E39226000E3F0DA
:101B4000E6FF6000E7F0E6FFFEEC5CF081EF11F0ED
:101B5000FD0EE350020F386EFE0E6F008CFF39F061
:101B6000000E39226000E3F0E6FF6000E7F0E6FFD8
:101B7000FEEC5CF081EF11F0FF0EE350386E396A35
:101B80003950000AD8B4C7EF0DF081EF11F038508A
:101B9000140AD8B481EF11F0010AD8B481EF11F022
:101BA000030AD8B481EF11F0010AD8B494EF0DF014
:101BB0000F0AD8B481EF11F0010AD8B4A8EF0DF0E4
:101BC000030AD8B481EF11F081EF11F0FD0EE3505C
:101BD0001B0F386EFE0E6F008CFF39F0000E39229D
:101BE0006000E3F0F6FF6000E7F0F7FF000EF86E2C
:101BF0000F0EF76404D0010EF56E0C0008D06F00D4
:101C0000DBFFE9FF6F00DFFFEAFF010EEF6EFD0E65
:101C1000E3501F0F386EFE0E6F008CFF39F0000E80
:101C200039226000E3F0F6FF6000E7F0F7FF000EF6
:101C3000F86E0F0EF76409D009006F00D4FF38F07A
:101C400009006F00D4FF39F00CD06F00DBFFE9FF13
:101C50006F00DFFFEAFF6F00B8FF38F06F00B8FFDA
:101C600039F038503910D8B438EF0EF03AEF0EF0A2
:101C7000C0EF11F0FD0EE350210F386EFE0E6F0025
:101C80008CFF39F0000E39226000E3F0F6FF6000AF
:101C9000E7F0F7FF000EF86E0F0EF76409D00900A9
:101CA0006F00D4FF38F009006F00D4FF39F00CD07A
:101CB0006F00DBFFE9FF6F00DFFFEAFF6F00B8FF97
:101CC00038F06F00B8FF39F06000E3F0E6FF600025
:101CD000E7F0E6FFFB0EE3501F0F386EFC0E6F00BF
:101CE0008CFF39F0000E39226000E3F0F6FF60004F
:101CF000E7F0F7FF000EF86E0F0EF76409D0090049
:101D00006F00D4FF38F009006F00D4FF39F00CD019
:101D10006F00DBFFE9FF6F00DFFFEAFF6F00B8FF36
:101D200038F06F00B8FF39F002D8A0EF0EF00500D0
:101D3000FA6E3850FD6E3950FE6EFF6AFA5012008E
:101D4000C0EF11F0FD0EE350230F386EFE0E6F0052
:101D50008CFF39F0000E39226000E3F0F6FF6000DE
:101D6000E7F0F7FF000EF86E0F0EF76409D00900D8
:101D70006F00D4FF38F009006F00D4FF39F00CD0A9
:101D80006F00DBFFE9FF6F00DFFFEAFF6F00B8FFC6
:101D900038F06F00B8FF39F038503910D8B4D3EFAD
:101DA0000EF0D5EF0EF0C0EF11F0FD0EE350250F51
:101DB000386EFE0E6F008CFF39F0000E3922600085
:101DC000E3F0F6FF6000E7F0F7FF000EF86E0F0E8D
:101DD000F76409D009006F00D4FF38F009006F00E4
:101DE000D4FF39F00CD06F00DBFFE9FF6F00DFFF9D
:101DF000EAFF6F00B8FF38F06F00B8FF39F06000FD
:101E0000E3F0E6FF6000E7F0E6FFFB0EE350230F90
:101E1000386EFC0E6F008CFF39F0000E3922600026
:101E2000E3F0F6FF6000E7F0F7FF000EF86E0F0E2C
:101E3000F76409D009006F00D4FF38F009006F0083
:101E4000D4FF39F00CD06F00DBFFE9FF6F00DFFF3C
:101E5000EAFF6F00B8FF38F06F00B8FF39F002D822
:101E60003BEF0FF00500FA6E3850FD6E3950FE6EF4
:101E7000FF6AFA501200C0EF11F0FD0EE350010F9F
:101E8000386EFE0E6F008CFF39F0000E39226000B4
:101E9000E3F0E6FF6000E7F0E6FF9CEC50F0000E98
:101EA000E66E000EE66EFB0EE350020F386EFC0E7F
:101EB0006F008CFF39F0000E39226000E3F0E6FF7E
:101EC0006000E7F0E6FFC2EC5BF0FD0EE350270F89
:101ED000386EFE0E6F008CFF39F0000E3922600064
:101EE000E3F0F6FF6000E7F0F7FF000EF86E0F0E6C
:101EF000F76409D009006F00D4FF38F009006F00C3
:101F0000D4FF39F00CD06F00DBFFE9FF6F00DFFF7B
:101F1000EAFF6F00B8FF38F06F00B8FF39F03850B3
:101F20003910D8B496EF0FF098EF0FF0C0EF11F022
:101F3000FD0EE350290F386EFE0E6F008CFF39F056
:101F4000000E39226000E3F0F6FF6000E7F0F7FFD3
:101F5000000EF86E0F0EF76409D009006F00D4FF71
:101F600038F009006F00D4FF39F00CD06F00DBFFB0
:101F7000E9FF6F00DFFFEAFF6F00B8FF38F06F0086
:101F8000B8FF39F06000E3F0E6FF6000E7F0E6FF3D
:101F9000FB0EE350270F386EFC0E6F008CFF39F0FC
:101FA000000E39226000E3F0F6FF6000E7F0F7FF73
:101FB000000EF86E0F0EF76409D009006F00D4FF11
:101FC00038F009006F00D4FF39F00CD06F00DBFF50
:101FD000E9FF6F00DFFFEAFF6F00B8FF38F06F0026
:101FE000B8FF39F002D8FEEF0FF00500FA6E385056
:101FF000FD6E3950FE6EFF6AFA501200C0EF11F00C
:10200000FD0EE3502B0F386EFE0E6F008CFF39F083
:10201000000E39226000E3F0F6FF6000E7F0F7FF02
:10202000000EF86E0F0EF76409D009006F00D4FFA0
:1020300038F009006F00D4FF39F00CD06F00DBFFDF
:10204000E9FF6F00DFFFEAFF6F00B8FF38F06F00B5
:10205000B8FF39F038503910D8B431EF10F033EF01
:1020600010F0C0EF11F0FD0EE3502D0F386EFE0E94
:102070006F008CFF39F0000E39226000E3F0F6FFAC
:102080006000E7F0F7FF000EF86E0F0EF76409D05E
:1020900009006F00D4FF38F009006F00D4FF39F059
:1020A0000CD06F00DBFFE9FF6F00DFFFEAFF6F007E
:1020B000B8FF38F06F00B8FF39F06000E3F0E6FFDA
:1020C0006000E7F0E6FFFB0EE3502B0F386EFC0ECE
:1020D0006F008CFF39F0000E39226000E3F0F6FF4C
:1020E0006000E7F0F7FF000EF86E0F0EF76409D0FE
:1020F00009006F00D4FF38F009006F00D4FF39F0F9
:102100000CD06F00DBFFE9FF6F00DFFFEAFF6F001D
:10211000B8FF38F06F00B8FF39F002D899EF10F02F
:102120000500FA6E3850FD6E3950FE6EFF6AFA50A7
:102130001200C0EF11F0FD0EE350010F386EFE0EDD
:102140006F008CFF39F0000E39226000E3F0E6FFEB
:102150006000E7F0E6FF9CEC50F0000EE66E000E2B
:10216000E66EFB0EE350020F386EFC0E6F008CFF24
:1021700039F0000E39226000E3F0E6FF6000E7F07E
:10218000E6FFC2EC5BF0FD0EE3501C0F386EFE0E56
:102190006F008CFF39F0000E39226000E3F0F6FF8B
:1021A0006000E7F0F7FF000EF86E0F0EF76404D042
:1021B000010EF56E0C0008D06F00DBFFE9FF6F0029
:1021C000DFFFEAFF010EEF6EC0EF11F0FD0EE350EE
:1021D000330F386EFE0E6F008CFF39F0000E39227F
:1021E0006000E3F0F6FF6000E7F0F7FF000EF86E26
:1021F0000F0EF76409D009006F00D4FF38F0090012
:102200006F00D4FF39F00CD06F00DBFFE9FF6F00E7
:10221000DFFFEAFF6F00B8FF38F06F00B8FF39F05A
:1022200038503910D8B417EF11F019EF11F0C0EF92
:1022300011F0FD0EE350350F386EFE0E6F008CFF6F
:1022400039F0000E39226000E3F0F6FF6000E7F09D
:10225000F7FF000EF86E0F0EF76409D009006F004B
:10226000D4FF38F009006F00D4FF39F00CD06F00B4
:10227000DBFFE9FF6F00DFFFEAFF6F00B8FF38F018
:102280006F00B8FF39F06000E3F0E6FF6000E7F0B0
:10229000E6FFFB0EE350330F386EFC0E6F008CFF31
:1022A00039F0000E39226000E3F0F6FF6000E7F03D
:1022B000F7FF000EF86E0F0EF76409D009006F00EB
:1022C000D4FF38F009006F00D4FF39F00CD06F0054
:1022D000DBFFE9FF6F00DFFFEAFF6F00B8FF38F0B8
:1022E0006F00B8FF39F002D87FEF11F00500FA6EE9
:1022F0003850FD6E3950FE6EFF6AFA501200C0EF82
:1023000011F0FD0E6F008FFFF6FFFE0E6F008FFFC6
:10231000F7FF000EF86E0F0EF76403D00800F550BB
:1023200007D06F00DBFFE9FF6F00DFFFEAFFEF5030
:10233000386E396A3950000AD8B4A1EF11F0C0EFF5
:1023400011F03850140AD8B4C0EF11F0010AD8B413
:10235000E6EF0DF0030AD8B4A2EF0EF0010AD8B4EC
:102360003DEF0FF00F0AD8B400EF10F0010AD8B417
:102370009BEF10F0030AD8B4E6EF10F0C0EF11F0B5
:10238000FB0EE126FF0EE2221200E652E6526F003B
:102390003CFE39F00F0E3916FE0E6000E7F0E3FF49
:1023A000FF0E6F0047FEE3FFFE0EE350100F911289
:1023B00098EF1AF080AEDFEF11F0E1EF11F0C6EF09
:1023C0001AF082A6E6EF11F0E8EF11F018EF12F024
:1023D000FC0E6F008FFFD9FFFD0E6F008FFFDAFF3D
:1023E000020EDF6E8250E66E8150E66E8450E66E1D
:1023F0008350E66EE3EC44F0FC0E6F008CFF38F087
:10240000FD0E6F008CFF39F0010E3824D96E000EDE
:102410003920DA6E6000BBF0DEFF6000BFF0DEFF47
:102420006000C3F0DEFF6000C7F0DEFF42EF12F095
:10243000FC0E6F008FFFD9FFFD0E6F008FFFDAFFDC
:10244000010EDF6E8250E66E8150E66E10EC51F0A8
:10245000FC0E6F008CFF38F0FD0E6F008CFF39F022
:10246000010E3824D96E000E3920DA6E6000BBF000
:10247000DEFF6000BFF0DEFF6000C3F0DEFF600043
:10248000C7F0DEFFFC0E6F008CFF38F0FD0E6F0012
:102490008CFF39F0050E3824D96E000E3920DA6E23
:1024A00085500F0BDF6EFC0E6F008CFF38F0FD0EB9
:1024B0006F008CFF39F00E0E3824D96E000E3920D3
:1024C000DA6E8544E846030BDF6EFC0E6F008CFF6E
:1024D00038F0FD0E6F008CFF39F0060E3824D96EEF
:1024E000000E3920DA6E6F001BFEDFFFFC0E6F005E
:1024F0008CFF38F0FD0E6F008CFF39F0070E38248A
:10250000D96E000E3920DA6E6F001FFEDFFFFC0E61
:102510006F008CFF38F0FD0E6F008CFF39F0080E55
:102520003824D96E000E3920DA6E6F0023FEDFFFEB
:10253000FC0E6F008CFF38F0FD0E6F008CFF39F041
:10254000090E3824D96E000E3920DA6E6F0027FE8E
:10255000DFFFFC0E6F008CFF38F0FD0E6F008CFF6C
:1025600039F00A0E3824D96E000E3920DA6E6F0069
:102570002BFEDFFFFC0E6F008CFF38F0FD0E6F00AE
:102580008CFF39F00B0E3824D96E000E3920DA6E2C
:102590006F002FFEDFFFFC0E6F008CFF38F0FD0E8A
:1025A0006F008CFF39F00C0E3824D96E000E3920E4
:1025B000DA6E6F0033FEDFFFFC0E6F008CFF38F029
:1025C000FD0E6F008CFF39F00D0E3824D96E000E11
:1025D0003920DA6E6F0037FEDFFF809EC6EF1AF0FB
:1025E0003701F0AFF6EF12F0F8EF12F0C6EF1AF085
:1025F00082A6FDEF12F0FFEF12F02FEF13F0FC0EAA
:102600006F008FFFD9FFFD0E6F008FFFDAFF020E04
:10261000DF6E8250E66E8150E66E8450E66E835027
:10262000E66EE3EC44F0FC0E6F008CFF38F0FD0E1C
:102630006F008CFF39F0010E3824D96E000E39205E
:10264000DA6E6000BBF0DEFF6000BFF0DEFF60000E
:10265000C3F0DEFF6000C7F0DEFF59EF13F0FC0EA1
:102660006F008FFFD9FFFD0E6F008FFFDAFF010EA5
:10267000DF6E8250E66E8150E66E10EC51F0FC0E7B
:102680006F008CFF38F0FD0E6F008CFF39F0010EEB
:102690003824D96E000E3920DA6E6000BBF0DEFF00
:1026A0006000BFF0DEFF6000C3F0DEFF6000C7F037
:1026B000DEFFFC0E6F008CFF38F0FD0E6F008CFF0C
:1026C00039F0050E3824D96E000E3920DA6E8550A7
:1026D0000F0BDF6EFC0E6F008CFF38F0FD0E6F00ED
:1026E0008CFF39F00E0E3824D96E000E3920DA6EC8
:1026F0008544E846030BDF6EFC0E6F008CFF38F05C
:10270000FD0E6F008CFF39F0060E3824D96E000ED6
:102710003920DA6E6F001BFEDFFFFC0E6F008CFFAE
:1027200038F0FD0E6F008CFF39F0070E3824D96E9B
:10273000000E3920DA6E6F001FFEDFFFFC0E6F0007
:102740008CFF38F0FD0E6F008CFF39F0080E382436
:10275000D96E000E3920DA6E6F0023FEDFFFFC0E0B
:102760006F008CFF38F0FD0E6F008CFF39F0090E02
:102770003824D96E000E3920DA6E6F0027FEDFFF95
:10278000FC0E6F008CFF38F0FD0E6F008CFF39F0EF
:102790000A0E3824D96E000E3920DA6E6F002BFE37
:1027A000DFFFFC0E6F008CFF38F0FD0E6F008CFF1A
:1027B00039F00B0E3824D96E000E3920DA6E6F0016
:1027C0002FFEDFFFFC0E6F008CFF38F0FD0E6F0058
:1027D0008CFF39F00C0E3824D96E000E3920DA6ED9
:1027E0006F0033FEDFFFFC0E6F008CFF38F0FD0E34
:1027F0006F008CFF39F00D0E3824D96E000E392091
:10280000DA6E6F0037FEDFFF3701F09FEEEF12F058
:10281000370140AF0EEF14F010EF14F0C6EF1AF0CE
:1028200082A615EF14F017EF14F047EF14F0FC0E2A
:102830006F008FFFD9FFFD0E6F008FFFDAFF020ED2
:10284000DF6E8250E66E8150E66E8450E66E8350F5
:10285000E66EE3EC44F0FC0E6F008CFF38F0FD0EEA
:102860006F008CFF39F0010E3824D96E000E39202C
:10287000DA6E6000BBF0DEFF6000BFF0DEFF6000DC
:10288000C3F0DEFF6000C7F0DEFF71EF14F0FC0E56
:102890006F008FFFD9FFFD0E6F008FFFDAFF010E73
:1028A000DF6E8250E66E8150E66E10EC51F0FC0E49
:1028B0006F008CFF38F0FD0E6F008CFF39F0010EB9
:1028C0003824D96E000E3920DA6E6000BBF0DEFFCE
:1028D0006000BFF0DEFF6000C3F0DEFF6000C7F005
:1028E000DEFFFC0E6F008CFF38F0FD0E6F008CFFDA
:1028F00039F0050E3824D96E000E3920DA6E855075
:102900000F0BDF6EFC0E6F008CFF38F0FD0E6F00BA
:102910008CFF39F00E0E3824D96E000E3920DA6E95
:102920008544E846030BDF6EFC0E6F008CFF38F029
:10293000FD0E6F008CFF39F0060E3824D96E000EA4
:102940003920DA6E6F001BFEDFFFFC0E6F008CFF7C
:1029500038F0FD0E6F008CFF39F0070E3824D96E69
:10296000000E3920DA6E6F001FFEDFFFFC0E6F00D5
:102970008CFF38F0FD0E6F008CFF39F0080E382404
:10298000D96E000E3920DA6E6F0023FEDFFFFC0ED9
:102990006F008CFF38F0FD0E6F008CFF39F0090ED0
:1029A0003824D96E000E3920DA6E6F0027FEDFFF63
:1029B000FC0E6F008CFF38F0FD0E6F008CFF39F0BD
:1029C0000A0E3824D96E000E3920DA6E6F002BFE05
:1029D000DFFFFC0E6F008CFF38F0FD0E6F008CFFE8
:1029E00039F00B0E3824D96E000E3920DA6E6F00E4
:1029F0002FFEDFFFFC0E6F008CFF38F0FD0E6F0026
:102A00008CFF39F00C0E3824D96E000E3920DA6EA6
:102A10006F0033FEDFFFFC0E6F008CFF38F0FD0E01
:102A20006F008CFF39F00D0E3824D96E000E39205E
:102A3000DA6E6F0037FEDFFF3701409FEEEF12F0D6
:102A4000370150AF26EF15F028EF15F0C6EF1AF05A
:102A500082A62DEF15F02FEF15F05FEF15F0FC0EAD
:102A60006F008FFFD9FFFD0E6F008FFFDAFF020EA0
:102A7000DF6E8250E66E8150E66E8450E66E8350C3
:102A8000E66EE3EC44F0FC0E6F008CFF38F0FD0EB8
:102A90006F008CFF39F0010E3824D96E000E3920FA
:102AA000DA6E6000BBF0DEFF6000BFF0DEFF6000AA
:102AB000C3F0DEFF6000C7F0DEFF89EF15F0FC0E0B
:102AC0006F008FFFD9FFFD0E6F008FFFDAFF010E41
:102AD000DF6E8250E66E8150E66E10EC51F0FC0E17
:102AE0006F008CFF38F0FD0E6F008CFF39F0010E87
:102AF0003824D96E000E3920DA6E6000BBF0DEFF9C
:102B00006000BFF0DEFF6000C3F0DEFF6000C7F0D2
:102B1000DEFFFC0E6F008CFF38F0FD0E6F008CFFA7
:102B200039F0050E3824D96E000E3920DA6E855042
:102B30000F0BDF6EFC0E6F008CFF38F0FD0E6F0088
:102B40008CFF39F00E0E3824D96E000E3920DA6E63
:102B50008544E846030BDF6EFC0E6F008CFF38F0F7
:102B6000FD0E6F008CFF39F0060E3824D96E000E72
:102B70003920DA6E6F001BFEDFFFFC0E6F008CFF4A
:102B800038F0FD0E6F008CFF39F0070E3824D96E37
:102B9000000E3920DA6E6F001FFEDFFFFC0E6F00A3
:102BA0008CFF38F0FD0E6F008CFF39F0080E3824D2
:102BB000D96E000E3920DA6E6F0023FEDFFFFC0EA7
:102BC0006F008CFF38F0FD0E6F008CFF39F0090E9E
:102BD0003824D96E000E3920DA6E6F0027FEDFFF31
:102BE000FC0E6F008CFF38F0FD0E6F008CFF39F08B
:102BF0000A0E3824D96E000E3920DA6E6F002BFED3
:102C0000DFFFFC0E6F008CFF38F0FD0E6F008CFFB5
:102C100039F00B0E3824D96E000E3920DA6E6F00B1
:102C20002FFEDFFFFC0E6F008CFF38F0FD0E6F00F3
:102C30008CFF39F00C0E3824D96E000E3920DA6E74
:102C40006F0033FEDFFFFC0E6F008CFF38F0FD0ECF
:102C50006F008CFF39F00D0E3824D96E000E39202C
:102C6000DA6E6F0037FEDFFF3701509FEEEF12F094
:102C7000370160AF3EEF16F040EF16F0C6EF1AF0E6
:102C800082A645EF16F047EF16F077EF16F0FC0E30
:102C90006F008FFFD9FFFD0E6F008FFFDAFF020E6E
:102CA000DF6E8250E66E8150E66E8450E66E835091
:102CB000E66EE3EC44F0FC0E6F008CFF38F0FD0E86
:102CC0006F008CFF39F0010E3824D96E000E3920C8
:102CD000DA6E6000BBF0DEFF6000BFF0DEFF600078
:102CE000C3F0DEFF6000C7F0DEFFA1EF16F0FC0EC0
:102CF0006F008FFFD9FFFD0E6F008FFFDAFF010E0F
:102D0000DF6E8250E66E8150E66E10EC51F0FC0EE4
:102D10006F008CFF38F0FD0E6F008CFF39F0010E54
:102D20003824D96E000E3920DA6E6000BBF0DEFF69
:102D30006000BFF0DEFF6000C3F0DEFF6000C7F0A0
:102D4000DEFFFC0E6F008CFF38F0FD0E6F008CFF75
:102D500039F0050E3824D96E000E3920DA6E855010
:102D60000F0BDF6EFC0E6F008CFF38F0FD0E6F0056
:102D70008CFF39F00E0E3824D96E000E3920DA6E31
:102D80008544E846030BDF6EFC0E6F008CFF38F0C5
:102D9000FD0E6F008CFF39F0060E3824D96E000E40
:102DA0003920DA6E6F001BFEDFFFFC0E6F008CFF18
:102DB00038F0FD0E6F008CFF39F0070E3824D96E05
:102DC000000E3920DA6E6F001FFEDFFFFC0E6F0071
:102DD0008CFF38F0FD0E6F008CFF39F0080E3824A0
:102DE000D96E000E3920DA6E6F0023FEDFFFFC0E75
:102DF0006F008CFF38F0FD0E6F008CFF39F0090E6C
:102E00003824D96E000E3920DA6E6F0027FEDFFFFE
:102E1000FC0E6F008CFF38F0FD0E6F008CFF39F058
:102E20000A0E3824D96E000E3920DA6E6F002BFEA0
:102E3000DFFFFC0E6F008CFF38F0FD0E6F008CFF83
:102E400039F00B0E3824D96E000E3920DA6E6F007F
:102E50002FFEDFFFFC0E6F008CFF38F0FD0E6F00C1
:102E60008CFF39F00C0E3824D96E000E3920DA6E42
:102E70006F0033FEDFFFFC0E6F008CFF38F0FD0E9D
:102E80006F008CFF39F00D0E3824D96E000E3920FA
:102E9000DA6E6F0037FEDFFF3701609FEEEF12F052
:102EA000370170AF56EF17F058EF17F0C6EF1AF072
:102EB00082A65DEF17F05FEF17F08FEF17F0FC0EB3
:102EC0006F008FFFD9FFFD0E6F008FFFDAFF020E3C
:102ED000DF6E8250E66E8150E66E8450E66E83505F
:102EE000E66EE3EC44F0FC0E6F008CFF38F0FD0E54
:102EF0006F008CFF39F0010E3824D96E000E392096
:102F0000DA6E6000BBF0DEFF6000BFF0DEFF600045
:102F1000C3F0DEFF6000C7F0DEFFB9EF17F0FC0E74
:102F20006F008FFFD9FFFD0E6F008FFFDAFF010EDC
:102F3000DF6E8250E66E8150E66E10EC51F0FC0EB2
:102F40006F008CFF38F0FD0E6F008CFF39F0010E22
:102F50003824D96E000E3920DA6E6000BBF0DEFF37
:102F60006000BFF0DEFF6000C3F0DEFF6000C7F06E
:102F7000DEFFFC0E6F008CFF38F0FD0E6F008CFF43
:102F800039F0050E3824D96E000E3920DA6E8550DE
:102F90000F0BDF6EFC0E6F008CFF38F0FD0E6F0024
:102FA0008CFF39F00E0E3824D96E000E3920DA6EFF
:102FB0008544E846030BDF6EFC0E6F008CFF38F093
:102FC000FD0E6F008CFF39F0060E3824D96E000E0E
:102FD0003920DA6E6F001BFEDFFFFC0E6F008CFFE6
:102FE00038F0FD0E6F008CFF39F0070E3824D96ED3
:102FF000000E3920DA6E6F001FFEDFFFFC0E6F003F
:103000008CFF38F0FD0E6F008CFF39F0080E38246D
:10301000D96E000E3920DA6E6F0023FEDFFFFC0E42
:103020006F008CFF38F0FD0E6F008CFF39F0090E39
:103030003824D96E000E3920DA6E6F0027FEDFFFCC
:10304000FC0E6F008CFF38F0FD0E6F008CFF39F026
:103050000A0E3824D96E000E3920DA6E6F002BFE6E
:10306000DFFFFC0E6F008CFF38F0FD0E6F008CFF51
:1030700039F00B0E3824D96E000E3920DA6E6F004D
:103080002FFEDFFFFC0E6F008CFF38F0FD0E6F008F
:103090008CFF39F00C0E3824D96E000E3920DA6E10
:1030A0006F0033FEDFFFFC0E6F008CFF38F0FD0E6B
:1030B0006F008CFF39F00D0E3824D96E000E3920C8
:1030C000DA6E6F0037FEDFFF3701709FEEEF12F010
:1030D000370180AF6EEF18F070EF18F0C6EF1AF0FE
:1030E00082A675EF18F077EF18F0A7EF18F0FC0E36
:1030F0006F008FFFD9FFFD0E6F008FFFDAFF020E0A
:10310000DF6E8250E66E8150E66E8450E66E83502C
:10311000E66EE3EC44F0FC0E6F008CFF38F0FD0E21
:103120006F008CFF39F0010E3824D96E000E392063
:10313000DA6E6000BBF0DEFF6000BFF0DEFF600013
:10314000C3F0DEFF6000C7F0DEFFD1EF18F0FC0E29
:103150006F008FFFD9FFFD0E6F008FFFDAFF010EAA
:10316000DF6E8250E66E8150E66E10EC51F0FC0E80
:103170006F008CFF38F0FD0E6F008CFF39F0010EF0
:103180003824D96E000E3920DA6E6000BBF0DEFF05
:103190006000BFF0DEFF6000C3F0DEFF6000C7F03C
:1031A000DEFFFC0E6F008CFF38F0FD0E6F008CFF11
:1031B00039F0050E3824D96E000E3920DA6E8550AC
:1031C0000F0BDF6EFC0E6F008CFF38F0FD0E6F00F2
:1031D0008CFF39F00E0E3824D96E000E3920DA6ECD
:1031E0008544E846030BDF6EFC0E6F008CFF38F061
:1031F000FD0E6F008CFF39F0060E3824D96E000EDC
:103200003920DA6E6F001BFEDFFFFC0E6F008CFFB3
:1032100038F0FD0E6F008CFF39F0070E3824D96EA0
:10322000000E3920DA6E6F001FFEDFFFFC0E6F000C
:103230008CFF38F0FD0E6F008CFF39F0080E38243B
:10324000D96E000E3920DA6E6F0023FEDFFFFC0E10
:103250006F008CFF38F0FD0E6F008CFF39F0090E07
:103260003824D96E000E3920DA6E6F0027FEDFFF9A
:10327000FC0E6F008CFF38F0FD0E6F008CFF39F0F4
:103280000A0E3824D96E000E3920DA6E6F002BFE3C
:10329000DFFFFC0E6F008CFF38F0FD0E6F008CFF1F
:1032A00039F00B0E3824D96E000E3920DA6E6F001B
:1032B0002FFEDFFFFC0E6F008CFF38F0FD0E6F005D
:1032C0008CFF39F00C0E3824D96E000E3920DA6EDE
:1032D0006F0033FEDFFFFC0E6F008CFF38F0FD0E39
:1032E0006F008CFF39F00D0E3824D96E000E392096
:1032F000DA6E6F0037FEDFFF3701809FEEEF12F0CE
:10330000370190AF86EF19F088EF19F0C6EF1AF089
:1033100082A68DEF19F08FEF19F0BFEF19F0FC0EB8
:103320006F008FFFD9FFFD0E6F008FFFDAFF020ED7
:10333000DF6E8250E66E8150E66E8450E66E8350FA
:10334000E66EE3EC44F0FC0E6F008CFF38F0FD0EEF
:103350006F008CFF39F0010E3824D96E000E392031
:10336000DA6E6000BBF0DEFF6000BFF0DEFF6000E1
:10337000C3F0DEFF6000C7F0DEFFE9EF19F0FC0EDE
:103380006F008FFFD9FFFD0E6F008FFFDAFF010E78
:10339000DF6E8250E66E8150E66E10EC51F0FC0E4E
:1033A0006F008CFF38F0FD0E6F008CFF39F0010EBE
:1033B0003824D96E000E3920DA6E6000BBF0DEFFD3
:1033C0006000BFF0DEFF6000C3F0DEFF6000C7F00A
:1033D000DEFFFC0E6F008CFF38F0FD0E6F008CFFDF
:1033E00039F0050E3824D96E000E3920DA6E85507A
:1033F0000F0BDF6EFC0E6F008CFF38F0FD0E6F00C0
:103400008CFF39F00E0E3824D96E000E3920DA6E9A
:103410008544E846030BDF6EFC0E6F008CFF38F02E
:10342000FD0E6F008CFF39F0060E3824D96E000EA9
:103430003920DA6E6F001BFEDFFFFC0E6F008CFF81
:1034400038F0FD0E6F008CFF39F0070E3824D96E6E
:10345000000E3920DA6E6F001FFEDFFFFC0E6F00DA
:103460008CFF38F0FD0E6F008CFF39F0080E382409
:10347000D96E000E3920DA6E6F0023FEDFFFFC0EDE
:103480006F008CFF38F0FD0E6F008CFF39F0090ED5
:103490003824D96E000E3920DA6E6F0027FEDFFF68
:1034A000FC0E6F008CFF38F0FD0E6F008CFF39F0C2
:1034B0000A0E3824D96E000E3920DA6E6F002BFE0A
:1034C000DFFFFC0E6F008CFF38F0FD0E6F008CFFED
:1034D00039F00B0E3824D96E000E3920DA6E6F00E9
:1034E0002FFEDFFFFC0E6F008CFF38F0FD0E6F002B
:1034F0008CFF39F00C0E3824D96E000E3920DA6EAC
:103500006F0033FEDFFFFC0E6F008CFF38F0FD0E06
:103510006F008CFF39F00D0E3824D96E000E392063
:10352000DA6E6F0037FEDFFF3701909FEEEF12F08B
:10353000FE0EE350386E396A3950000AD8B4A3EF52
:103540001AF0C6EF1AF03850000AD8B4DAEF11F0CA
:10355000010AD8B4F0EF12F0030AD8B408EF14F05F
:10356000010AD8B420EF15F0070AD8B438EF16F0E6
:10357000010AD8B450EF17F0030AD8B468EF18F076
:10358000010AD8B480EF19F0C6EF1AF0FF0E6F00F1
:103590008FFF91FFE552E552E552E5521200240EED
:1035A000E126000EE222DA0E6F008FFFE6FF6F00C9
:1035B0008FFFE6FFC2EC5EF0FC0E6000BFF0E3FFA1
:1035C000FB0E6000BBF0E3FFFB0E6F008FFFF6FF0A
:1035D000FC0E6F008FFFF7FF000EF86E0F0EF76402
:1035E00003D00800F55007D06F00DBFFE9FF6F0044
:1035F000DFFFEAFFEF50396EFF0E6000E7F0E3FFF8
:10360000DA0E6F008FFFE6FF6F008FFFE6FF82ECA0
:103610005FF0DA0E6F008FFFE6FF6F008FFFE6FFAF
:1036200024EC5EF0E5526F009CFF45F0E5526F0020
:103630009CFF44F0E5526F009CFF43F0E5526F00A1
:103640009CFF42F0E5526F009CFF41F0E5526F0095
:103650009CFF40F0E5526F009CFF3FF0E5526F0089
:103660009CFF3EF0EB0E6000FBF0E3FFEC0E600011
:10367000FFF0E3FFED0E600003F1E3FFEE0E6000EC
:1036800007F1E3FFEF0E60000BF1E3FFF00E6000C7
:103690000FF1E3FFF10E600013F1E3FFF20E6000A3
:1036A00017F1E3FFEB0E6F008CFF36F0EC0E6F00AE
:1036B0008CFF37F0ED0E6F008CFF38F0EE0E6F00D0
:1036C0008CFF39F0F70E6000DBF0E3FFF80E6000CE
:1036D000DFF0E3FFF90E6000E3F0E3FFFA0E6000B5
:1036E000E7F0E3FF85EF22F0DA0E6F008FFFD9FFDE
:1036F000DB0E6F008FFFDAFFDF500A0AD8A483EFDA
:103700001BF085EF1BF0B0EF22F0FB0E6F008FFF78
:10371000F6FFFC0E6F008FFFF7FF000EF86E0F0E26
:10372000F76404D00B0EF56E0C0008D06F00DBFFC1
:10373000E9FF6F00DFFFEAFF0B0EEF6EB0EF22F044
:10374000DA0E6F008FFFD9FFDB0E6F008FFFDAFFFD
:10375000DF500B0AD8A4AFEF1BF0B1EF1BF0BFEFA7
:103760001CF0FB0EE350020F386EFC0E6F008CFF56
:1037700039F0000E39226000E3F0F6FF6000E7F058
:10378000F7FF000EF86E0F0EF76409D009006F0006
:10379000D4FF38F009006F00D4FF39F00CD06F006F
:1037A000DBFFE9FF6F00DFFFEAFF6F00B8FF38F0D3
:1037B0006F00B8FF39F038503910D8B4E2EF1BF081
:1037C000E4EF1BF0BFEF1CF0EF0EE124D96EFF0E0B
:1037D000E220DA6E6F0078FF36F06F0078FF37F086
:1037E0006F0078FF38F06F0078FF39F036503E6E8A
:1037F00037503F6E3850406E3950416E426A436ACE
:10380000446A456AEB0E6000FBF0E3FFEC0E6000DB
:10381000FFF0E3FFED0E600003F1E3FFEE0E60004A
:1038200007F1E3FFEF0E60000BF1E3FFF00E600025
:103830000FF1E3FFF10E600013F1E3FFF20E600001
:1038400017F1E3FFEB0E6F008CFF36F0EC0E6F000C
:103850008CFF37F0ED0E6F008CFF38F0EE0E6F002E
:103860008CFF39F0F30E6000DBF0E3FFF40E600034
:10387000DFF0E3FFF50E6000E3F0E3FFF60E60001B
:10388000E7F0E3FFF30E6F008CFF2EF0FD0E6000FB
:10389000BBF0E3FFE150FD0FD96EE250DA6EFF0E90
:1038A000DA22DF3A0F0EDF16FD0E6F008CFF2EF0CE
:1038B0000F0E2E16FD0E6000BBF0E3FFF40EE124A8
:1038C000D96EFF0EE220DA6EDF50396EFE0E600018
:1038D000E7F0E3FFE150FE0FD96EE250DA6EFF0E23
:1038E000DA22DF3A0F0EDF16F70E6F008FFFE6FFCA
:1038F0006F008FFFE6FF6F008FFFE6FF6F008FFF07
:10390000E6FF000EE66EF80EE350E66EF80EE350AA
:10391000E66EF40EE350020F386EF50E6F008CFF6A
:1039200039F0000E39226000E3F0F6FF6000E7F0A6
:10393000F7FF000EF86E0F0EF76409D009006F0054
:10394000D4FF38F009006F00D4FF39F00CD06F00BD
:10395000DBFFE9FF6F00DFFFEAFF6F00B8FF38F021
:103960006F00B8FF39F002D8BFEF1CF00500FA6E07
:103970003850FD6E3950FE6EFF6AFA501200DA0EB2
:103980006F008FFFD9FFDB0E6F008FFFDAFFDF5074
:103990000C0AD8A4CEEF1CF0D0EF1CF0DEEF1DF027
:1039A000FB0EE350020F386EFC0E6F008CFF39F0F7
:1039B000000E39226000E3F0F6FF6000E7F0F7FF49
:1039C000000EF86E0F0EF76409D009006F00D4FFE7
:1039D00038F009006F00D4FF39F00CD06F00DBFF26
:1039E000E9FF6F00DFFFEAFF6F00B8FF38F06F00FC
:1039F000B8FF39F038503910D8B401EF1DF003EF9B
:103A00001DF0DEEF1DF0EF0EE124D96EFF0EE22077
:103A1000DA6E6F0078FF36F06F0078FF37F06F00D6
:103A200078FF38F06F0078FF39F036503E6E37502F
:103A30003F6E3850406E3950416E426A436A446A64
:103A4000456AEB0E6000FBF0E3FFEC0E6000FFF058
:103A5000E3FFED0E600003F1E3FFEE0E600007F1FF
:103A6000E3FFEF0E60000BF1E3FFF00E60000FF1DB
:103A7000E3FFF10E600013F1E3FFF20E600017F1B7
:103A8000E3FFEB0E6F008CFF36F0EC0E6F008CFF47
:103A900037F0ED0E6F008CFF38F0EE0E6F008CFFEC
:103AA00039F0F30E6000DBF0E3FFF40E6000DFF0AE
:103AB000E3FFF50E6000E3F0E3FFF60E6000E7F0D1
:103AC000E3FFF30E6F008CFF2EF0FD0E6000BBF0E5
:103AD000E3FFE150FD0FD96EE250DA6EFF0EDA22FD
:103AE000DF3A0F0EDF16FD0E6F008CFF2EF00F0E6B
:103AF0002E16FD0E6000BBF0E3FFF40EE124D96E3C
:103B0000FF0EE220DA6EDF50396EFE0E6000E7F045
:103B1000E3FFE150FE0FD96EE250DA6EFF0EDA22BB
:103B2000DF3A0F0EDF16F70E6F008FFFE6FF6F0014
:103B30008FFFE6FF6F008FFFE6FF6F008FFFE6FF4E
:103B4000010EE66EF80EE350E66EF80EE350E66EF8
:103B5000F40EE350020F386EF50E6F008CFF39F053
:103B6000000E39226000E3F0F6FF6000E7F0F7FF97
:103B7000000EF86E0F0EF76409D009006F00D4FF35
:103B800038F009006F00D4FF39F00CD06F00DBFF74
:103B9000E9FF6F00DFFFEAFF6F00B8FF38F06F004A
:103BA000B8FF39F002D8DEEF1DF00500FA6E38508C
:103BB000FD6E3950FE6EFF6AFA501200DA0E6F0089
:103BC0008FFFD9FFDB0E6F008FFFDAFFDF500D0A8A
:103BD000D8A4EDEF1DF0EFEF1DF0CCEF1EF0DC0EE2
:103BE000E36AE32AE10EE124D96EFF0EE220DA6EE9
:103BF000040EDF6EEA0EE124D96EFF0EE220DA6ECB
:103C0000DF6AE20EE124D96EFF0EE220DA6EEB0EDF
:103C10006F008FFFDFFF080E396EE150EB0FD96E9A
:103C2000E250DA6EFF0EDA223928DE5227EF1EF05C
:103C3000DE52DE52DE52DE52DE52DE52D890DD32ED
:103C4000DD32DD32DD32DD32DD32DD32DE32E82EF4
:103C500018EF1EF0E30EE124D96EFF0EE220DA6EBB
:103C6000EB0E6F008FFFDFFF080E396EE150EB0F98
:103C7000D96EE250DA6EFF0EDA223928DE5250EFAA
:103C80001EF0DE52DE52DE52DE52DE52DE52D8909E
:103C9000DD32DD32DD32DD32DD32DD32DD32DE32AB
:103CA000E82E41EF1EF0E40EE124D96EFF0EE22073
:103CB000DA6EEB0E6F008FFFDFFF080E396EE150FA
:103CC000EB0FD96EE250DA6EFF0EDA223928DE529F
:103CD00079EF1EF0DE52DE52DE52DE52DE52DE524E
:103CE000D890DD32DD32DD32DD32DD32DD32DD3203
:103CF000DE32E82E6AEF1EF0E50EE124D96EFF0EEB
:103D0000E220DA6EEB0E6F008FFFDFFF080E396ED8
:103D1000E150EB0FD96EE250DA6EFF0EDA2239284D
:103D2000DE52A2EF1EF0DE52DE52DE52DE52DE52D4
:103D3000DE52D890DD32DD32DD32DD32DD32DD3291
:103D4000DD32DE32E82E93EF1EF0E150EB0FD96E3C
:103D5000E250DA6EFF0EDA22DD0EE124E96EFF0E8C
:103D6000E220EA6E6F007BFFEEFF6F007BFFEEFF4D
:103D70006F007BFFEEFF6F007BFFEEFFDC0EE124A8
:103D80002E6EFF0EE2202F6E6000BBF0E6FF60009B
:103D9000BFF0E6FF38EC37F0DA0E6F008FFFD9FF87
:103DA000DB0E6F008FFFDAFFDF500E0AD8A4DBEFC7
:103DB0001EF0DDEF1EF0BAEF1FF0DC0EE36AE32A1F
:103DC000E10EE124D96EFF0EE220DA6E020EDF6E04
:103DD000EA0EE124D96EFF0EE220DA6EDF6AE20E0F
:103DE000E124D96EFF0EE220DA6EEB0E6F008FFF3A
:103DF000DFFF080E396EE150EB0FD96EE250DA6E3C
:103E0000FF0EDA223928DE5215EF1FF0DE52DE52A5
:103E1000DE52DE52DE52DE52D890DD32DD32DD324D
:103E2000DD32DD32DD32DD32DE32E82E06EF1FF02C
:103E3000E30EE124D96EFF0EE220DA6EEB0E6F0086
:103E40008FFFDFFF080E396EE150EB0FD96EE250A5
:103E5000DA6EFF0EDA223928DE523EEF1FF0DE5214
:103E6000DE52DE52DE52DE52DE52D890DD32DD32DC
:103E7000DD32DD32DD32DD32DD32DE32E82E2FEFB3
:103E80001FF0E40EE124D96EFF0EE220DA6EEB0E95
:103E90006F008FFFDFFF080E396EE150EB0FD96E18
:103EA000E250DA6EFF0EDA223928DE5267EF1FF099
:103EB000DE52DE52DE52DE52DE52DE52D890DD326B
:103EC000DD32DD32DD32DD32DD32DD32DE32E82E72
:103ED00058EF1FF0E50EE124D96EFF0EE220DA6EF6
:103EE000EB0E6F008FFFDFFF080E396EE150EB0F16
:103EF000D96EE250DA6EFF0EDA223928DE5290EFE8
:103F00001FF0DE52DE52DE52DE52DE52DE52D8901A
:103F1000DD32DD32DD32DD32DD32DD32DD32DE3228
:103F2000E82E81EF1FF0E150EB0FD96EE250DA6E10
:103F3000FF0EDA22DD0EE124E96EFF0EE220EA6ECA
:103F40006F007BFFEEFF6F007BFFEEFF6F007BFFDC
:103F5000EEFF6F007BFFEEFFDC0EE1242E6EFF0E06
:103F6000E2202F6E6000BBF0E6FF6000BFF0E6FFCE
:103F700038EC37F0DA0E6F008FFFD9FFDB0E6F00E1
:103F80008FFFDAFFDF500F0AD8A4C9EF1FF0CBEF85
:103F90001FF0A8EF20F0DC0EE36AE32AE10EE12433
:103FA000D96EFF0EE220DA6E010EDF6EEA0EE1241A
:103FB000D96EFF0EE220DA6EDF6AE20EE124D96EDE
:103FC000FF0EE220DA6EEB0E6F008FFFDFFF080EB0
:103FD000396EE150EB0FD96EE250DA6EFF0EDA2245
:103FE0003928DE5203EF20F0DE52DE52DE52DE527E
:103FF000DE52DE52D890DD32DD32DD32DD32DD32AE
:10400000DD32DD32DE32E82EF4EF1FF0E30EE12484
:10401000D96EFF0EE220DA6EEB0E6F008FFFDFFF2E
:10402000080E396EE150EB0FD96EE250DA6EFF0EDA
:10403000DA223928DE522CEF20F0DE52DE52DE5238
:10404000DE52DE52DE52D890DD32DD32DD32DD323C
:10405000DD32DD32DD32DE32E82E1DEF20F0E40EFF
:10406000E124D96EFF0EE220DA6EEB0E6F008FFFB7
:10407000DFFF080E396EE150EB0FD96EE250DA6EB9
:10408000FF0EDA223928DE5255EF20F0DE52DE52E2
:10409000DE52DE52DE52DE52D890DD32DD32DD32CB
:1040A000DD32DD32DD32DD32DE32E82E46EF20F069
:1040B000E50EE124D96EFF0EE220DA6EEB0E6F0002
:1040C0008FFFDFFF080E396EE150EB0FD96EE25023
:1040D000DA6EFF0EDA223928DE527EEF20F0DE5251
:1040E000DE52DE52DE52DE52DE52D890DD32DD325A
:1040F000DD32DD32DD32DD32DD32DE32E82E6FEFF1
:1041000020F0E150EB0FD96EE250DA6EFF0EDA22AA
:10411000DD0EE124E96EFF0EE220EA6E6F007BFF08
:10412000EEFF6F007BFFEEFF6F007BFFEEFF6F0087
:104130007BFFEEFFDC0EE1242E6EFF0EE2202F6EE1
:104140006000BBF0E6FF6000BFF0E6FF38EC37F040
:10415000DA0E6F008FFFD9FFDB0E6F008FFFDAFFE3
:10416000DF50100AD8A4B7EF20F0B9EF20F095EF98
:1041700021F0DC0EE36AE32AE10EE124D96EFF0EA2
:10418000E220DA6EDF6AEA0EE124D96EFF0EE22049
:10419000DA6EDF6AE20EE124D96EFF0EE220DA6EFB
:1041A000EB0E6F008FFFDFFF080E396EE150EB0F53
:1041B000D96EE250DA6EFF0EDA223928DE52F0EFC5
:1041C00020F0DE52DE52DE52DE52DE52DE52D89057
:1041D000DD32DD32DD32DD32DD32DD32DD32DE3266
:1041E000E82EE1EF20F0E30EE124D96EFF0EE2208D
:1041F000DA6EEB0E6F008FFFDFFF080E396EE150B5
:10420000EB0FD96EE250DA6EFF0EDA223928DE5259
:1042100019EF21F0DE52DE52DE52DE52DE52DE5265
:10422000D890DD32DD32DD32DD32DD32DD32DD32BD
:10423000DE32E82E0AEF21F0E40EE124D96EFF0E03
:10424000E220DA6EEB0E6F008FFFDFFF080E396E93
:10425000E150EB0FD96EE250DA6EFF0EDA22392808
:10426000DE5242EF21F0DE52DE52DE52DE52DE52EC
:10427000DE52D890DD32DD32DD32DD32DD32DD324C
:10428000DD32DE32E82E33EF21F0E50EE124D96E87
:10429000FF0EE220DA6EEB0E6F008FFFDFFF080EDD
:1042A000396EE150EB0FD96EE250DA6EFF0EDA2272
:1042B0003928DE526BEF21F0DE52DE52DE52DE5242
:1042C000DE52DE52D890DD32DD32DD32DD32DD32DB
:1042D000DD32DD32DE32E82E5CEF21F0E150EB0F13
:1042E000D96EE250DA6EFF0EDA22DD0EE124E96EBD
:1042F000FF0EE220EA6E6F007BFFEEFF6F007BFF98
:10430000EEFF6F007BFFEEFF6F007BFFEEFFDC0E2A
:10431000E1242E6EFF0EE2202F6E6000BBF0E6FF60
:104320006000BFF0E6FF38EC37F0DA0E6F008FFF69
:10433000D9FFDB0E6F008FFFDAFFDF50110AD8A420
:10434000A4EF21F0A6EF21F0B0EF22F0DC0EE36A3B
:10435000E32AE10EE124D96EFF0EE220DA6EDF6A75
:10436000EA0EE124D96EFF0EE220DA6E010EDF6E56
:10437000E20EE124D96EFF0EE220DA6EEB0E6F0042
:104380008FFFDFFF080E396EE150EB0FD96EE25060
:10439000DA6EFF0EDA223928DE52DEEF21F0DE522D
:1043A000DE52DE52DE52DE52DE52D890DD32DD3297
:1043B000DD32DD32DD32DD32DD32DE32E82ECFEFCE
:1043C00021F0E30EE124D96EFF0EE220DA6EEB0E4F
:1043D0006F008FFFDFFF080E396EE150EB0FD96ED3
:1043E000E250DA6EFF0EDA223928DE5207EF22F0B1
:1043F000DE52DE52DE52DE52DE52DE52D890DD3226
:10440000DD32DD32DD32DD32DD32DD32DE32E82E2C
:10441000F8EF21F0E40EE124D96EFF0EE220DA6E0F
:10442000EB0E6F008FFFDFFF080E396EE150EB0FD0
:10443000D96EE250DA6EFF0EDA223928DE5230EF02
:1044400022F0DE52DE52DE52DE52DE52DE52D890D2
:10445000DD32DD32DD32DD32DD32DD32DD32DE32E3
:10446000E82E21EF22F0E50EE124D96EFF0EE220C6
:10447000DA6EEB0E6F008FFFDFFF080E396EE15032
:10448000EB0FD96EE250DA6EFF0EDA223928DE52D7
:1044900059EF22F0DE52DE52DE52DE52DE52DE52A2
:1044A000D890DD32DD32DD32DD32DD32DD32DD323B
:1044B000DE32E82E4AEF22F0E150EB0FD96EE250E7
:1044C000DA6EFF0EDA22DD0EE124E96EFF0EE22045
:1044D000EA6E6F007BFFEEFF6F007BFFEEFF6F0069
:1044E0007BFFEEFF6F007BFFEEFFDC0EE1242E6E04
:1044F000FF0EE2202F6E6000BBF0E6FF6000BFF011
:10450000E6FF38EC37F0B0EF22F0FB0E6F008FFFC4
:10451000F6FFFC0E6F008FFFF7FF000EF86E0F0E18
:10452000F76403D00800F55007D06F00DBFFE9FF08
:104530006F00DFFFEAFFEF50386E396A3950000A2A
:10454000D8B4A5EF22F0B0EF22F038500A0AD8B460
:1045500074EF1BF0010AD8B4A0EF1BF0B0EF22F00B
:10456000FF0E6F008CFF39F0FB0E6F008FFFF6FF20
:10457000FC0E6F008FFFF7FF000EF86E0F0EF76452
:1045800003D00800F55007D06F00DBFFE9FF6F0094
:10459000DFFFEAFFEF503918D8B4D1EF22F0D3EFA4
:1045A00022F014EF23F0FF0EE350386E396A3950D1
:1045B000000AD8B4DEEF22F0E9EF22F038500A0A00
:1045C000D8B4E9EF22F0010AD8B4E9EF22F0E9EF1C
:1045D00022F0FB0E6F008FFFF6FFFC0E6F008FFFC7
:1045E000F7FF000EF86E0F0EF76403D00800F550C9
:1045F00007D06F00DBFFE9FF6F00DFFFEAFFEF503E
:10460000386E396A3950000AD8B409EF23F014EF34
:1046100023F038500A0AD8B414EF23F0010AD8B4B2
:1046200014EF23F014EF23F0DA0EE126FF0EE2225E
:104630001200E652E652E652E652FA0E6F008FFF83
:10464000E6FF6F008FFFE6FFC2EC5EF0FD0E60003C
:10465000BFF0E3FFFC0E6000BBF0E3FFFC0E6F0059
:104660008FFFF6FFFD0E6F008FFFF7FF000EF86E55
:104670000F0EF76403D00800F55007D06F00DBFF82
:10468000E9FF6F00DFFFEAFFEF50396EFF0E6000B9
:10469000E7F0E3FFFA0E6F008FFFE6FF6F008FFF7A
:1046A000E6FF82EC5FF0FE0E6000BBF0E3FFD3EFAD
:1046B00026F0FA0E6F008FFFD9FFFB0E6F008FFF01
:1046C000DAFFDF50C80AD8A468EF23F06AEF23F0BE
:1046D00006EF27F0FC0E6F008FFFF6FFFD0E6F0058
:1046E0008FFFF7FF000EF86E0F0EF76404D0010E77
:1046F000F56E0C0008D06F00DBFFE9FF6F00DFFFF5
:10470000EAFF010EEF6E06EF27F0FC0EE350050FF7
:10471000386EFD0E6F008CFF39F0000E39226000FC
:10472000E3F0F6FF6000E7F0F7FF000EF86E0F0E03
:10473000F76403D00800F55007D06F00DBFFE9FFF6
:104740006F00DFFFEAFFEF50396EFC0EE350070FFA
:10475000366EFD0E6F008CFF37F0000E37226000C2
:10476000DBF0F6FF6000DFF0F7FF000EF86E0F0ED3
:10477000F76405D06000E7F0F5FF0C0009D06F008A
:10478000DBFFE9FF6F00DFFFEAFF6000E7F0EFFF0C
:10479000FE0E6F008CFF2EF0CA0E2E18D8A4D3EF99
:1047A00023F0D5EF23F048EF24F0FC0E6F008FFFCD
:1047B000F6FFFD0E6F008FFFF7FF000EF86E0F0E75
:1047C000F76404D0020EF56E0C0008D06F00DBFF1A
:1047D000E9FF6F00DFFFEAFF020EEF6EFC0EE35011
:1047E000060F386EFD0E6F008CFF39F0000E392277
:1047F0006000E3F0F6FF6000E7F0F7FF000EF86EF0
:104800000F0EF76404D0010EF56E0C0008D06F0097
:10481000DBFFE9FF6F00DFFFEAFF010EEF6EFC0E2A
:10482000E350010F386EFD0E6F008CFF39F0000E63
:1048300039226000E3F0F6FF6000E7F0F7FF000EBA
:10484000F86E0F0EF76409D009006F00D4FF38F03E
:1048500009006F00D4FF39F00CD06F00DBFFE9FFD7
:104860006F00DFFFEAFF6F00B8FF38F06F00B8FF9E
:1048700039F06000E3F0E6FF6000E7F0E6FFFA0ED3
:104880006F008FFFE6FF6F008FFFE6FF97EC5BF096
:10489000FE0E6F008CFF2EF0C90E2E18D8A453EF19
:1048A00024F055EF24F006EF27F0FC0E6F008FFF89
:1048B000F6FFFD0E6F008FFFF7FF000EF86E0F0E74
:1048C000F76404D0020EF56E0C0008D06F00DBFF19
:1048D000E9FF6F00DFFFEAFF020EEF6EFC0EE35010
:1048E000060F386EFD0E6F008CFF39F0000E392276
:1048F0006000E3F0F6FF6000E7F0F7FF000EF86EEF
:104900000F0EF76404D0000EF56E0C0008D06F0097
:10491000DBFFE9FF6F00DFFFEAFF000EEF6EFC0E2A
:10492000E350010F386EFD0E6F008CFF39F0000E62
:1049300039226000E3F0F6FF6000E7F0F7FF000EB9
:10494000F86E0F0EF76409D009006F00D4FF38F03D
:1049500009006F00D4FF39F00CD06F00DBFFE9FFD6
:104960006F00DFFFEAFF6F00B8FF38F06F00B8FF9D
:1049700039F06000E3F0E6FF6000E7F0E6FFFA0ED2
:104980006F008FFFE6FF6F008FFFE6FF97EC5BF095
:1049900006EF27F0FC0EE350060F386EFD0E6F0099
:1049A0008CFF39F0000E39226000E3F0F6FF600062
:1049B000E7F0F7FF000EF86E0F0EF76403D0080063
:1049C000F55007D06F00DBFFE9FF6F00DFFFEAFF64
:1049D000EF500009D8B4EFEF24F0F1EF24F036EFF8
:1049E00025F0FC0EE350070F386EFD0E6F008CFFB4
:1049F00039F0000E39226000E3F0F6FF6000E7F0C6
:104A0000F7FF000EF86E0F0EF76403D00800F550A4
:104A100007D06F00DBFFE9FF6F00DFFFEAFFEF5019
:104A2000396EFF0E3926FC0EE350070F366EFD0E71
:104A30006F008CFF37F0000E37226000DBF0F6FFCE
:104A40006000DFF0F7FF000EF86E0F0EF76405D080
:104A50006000E7F0F5FF0C0009D06F00DBFFE9FF15
:104A60006F00DFFFEAFF6000E7F0EFFFFE0E6F0070
:104A70008CFF2EF0CB0E2E18D8A441EF25F043EF7B
:104A800025F006EF27F0FC0E6F008FFFF6FFFD0EFE
:104A90006F008FFFF7FF000EF86E0F0EF76404D063
:104AA000030EF56E0C0008D06F00DBFFE9FF6F000E
:104AB000DFFFEAFF030EEF6EFC0EE350030F386ECC
:104AC000FD0E6F008CFF39F0000E39226000E3F01C
:104AD000F6FF6000E7F0F7FF000EF86E0F0EF764C8
:104AE00009D009006F00D4FF38F009006F00D4FF2F
:104AF00039F00CD06F00DBFFE9FF6F00DFFFEAFF4A
:104B00006F00B8FF38F06F00B8FF39F06000E3F0D5
:104B1000E6FF6000E7F0E6FFFA0E6F008FFFE6FFAA
:104B20006F008FFFE6FF97EC5BF006EF27F0FE0EBD
:104B30006F008CFF2EF0CB0E2E18D8A4A2EF25F01C
:104B4000A4EF25F006EF27F0FC0EE350070F386EB8
:104B5000FD0E6F008CFF39F0000E39226000E3F08B
:104B6000F6FF6000E7F0F7FF000EF86E0F0EF76437
:104B700003D00800F55007D06F00DBFFE9FF6F009E
:104B8000DFFFEAFFEF500009D8A4C9EF25F0CBEF13
:104B900025F07FEF26F0FC0E6F008FFFF6FFFD0E75
:104BA0006F008FFFF7FF000EF86E0F0EF76404D052
:104BB000010EF56E0C0008D06F00DBFFE9FF6F00FF
:104BC000DFFFEAFF010EEF6EFC0EE350140F386EAC
:104BD000FD0E6F008CFF39F0000E39226000E3F00B
:104BE000F6FF6000E7F0F7FF000EF86E0F0EF764B7
:104BF00009D009006F00D4FF38F009006F00D4FF1E
:104C000039F00CD06F00DBFFE9FF6F00DFFFEAFF38
:104C10006F00B8FF38F06F00B8FF39F03850391026
:104C2000D8B415EF26F017EF26F006EF27F0FC0EAC
:104C3000E350160F386EFD0E6F008CFF39F0000E3A
:104C400039226000E3F0F6FF6000E7F0F7FF000EA6
:104C5000F86E0F0EF76409D009006F00D4FF38F02A
:104C600009006F00D4FF39F00CD06F00DBFFE9FFC3
:104C70006F00DFFFEAFF6F00B8FF38F06F00B8FF8A
:104C800039F06000E3F0E6FF6000E7F0E6FFFA0EBF
:104C9000E350140F386EFB0E6F008CFF39F0000EDE
:104CA00039226000E3F0F6FF6000E7F0F7FF000E46
:104CB000F86E0F0EF76409D009006F00D4FF38F0CA
:104CC00009006F00D4FF39F00CD06F00DBFFE9FF63
:104CD0006F00DFFFEAFF6F00B8FF38F06F00B8FF2A
:104CE00039F002D87DEF26F00500FA6E3850FD6EDF
:104CF0003950FE6EFF6AFA50120006EF27F0FC0EE4
:104D00006F008FFFF6FFFD0E6F008FFFF7FF000EA5
:104D1000F86E0F0EF76404D0020EF56E0C0008D08A
:104D20006F00DBFFE9FF6F00DFFFEAFF020EEF6EAF
:104D3000FC0EE350010F386EFD0E6F008CFF39F052
:104D4000000E39226000E3F0F6FF6000E7F0F7FFA5
:104D5000000EF86E0F0EF76409D009006F00D4FF43
:104D600038F009006F00D4FF39F00CD06F00DBFF82
:104D7000E9FF6F00DFFFEAFF6F00B8FF38F06F0058
:104D8000B8FF39F06000E3F0E6FF6000E7F0E6FF0F
:104D9000FA0E6F008FFFE6FF6F008FFFE6FF97ECC4
:104DA0005BF006EF27F0FC0E6F008FFFF6FFFD0EA5
:104DB0006F008FFFF7FF000EF86E0F0EF76403D041
:104DC0000800F55007D06F00DBFFE9FF6F00DFFF41
:104DD000EAFFEF50386E396A3950000AD8B4F3EF61
:104DE00026F006EF27F03850000AD8B459EF23F028
:104DF000010AD8B485EF23F0030AD8B4CAEF24F02F
:104E0000010AD8B497EF25F006EF27F0FF0E6F00E8
:104E10008CFF39F0FC0E6F008FFFF6FFFD0E6F0068
:104E20008FFFF7FF000EF86E0F0EF76403D0080037
:104E3000F55007D06F00DBFFE9FF6F00DFFFEAFFEF
:104E4000EF503918D8B427EF27F029EF27F04BEFB0
:104E500029F0FF0EE350386E396A3950000AD8B491
:104E600034EF27F018EF29F03850000AD8B418EFC3
:104E700029F0010AD8B418EF29F0030AD8B418EFC2
:104E800029F0010AD8B418EF29F018EF29F0FC0E28
:104E9000E350080F386EFD0E6F008CFF39F0000EE6
:104EA00039226000E3F0F6FF6000E7F0F7FF000E44
:104EB000F86E0F0EF76409D009006F00D4FF38F0C8
:104EC00009006F00D4FF39F00CD06F00DBFFE9FF61
:104ED0006F00DFFFEAFF6F00B8FF38F06F00B8FF28
:104EE00039F038503910D8B478EF27F07AEF27F03E
:104EF0004BEF29F0FC0EE3500A0F386EFD0E6F00E9
:104F00008CFF39F0000E39226000E3F0F6FF6000FC
:104F1000E7F0F7FF000EF86E0F0EF76409D00900F6
:104F20006F00D4FF38F009006F00D4FF39F00CD0C7
:104F30006F00DBFFE9FF6F00DFFFEAFF6F00B8FFE4
:104F400038F06F00B8FF39F06000E3F0E6FF600072
:104F5000E7F0E6FFFA0EE350080F386EFB0E6F0025
:104F60008CFF39F0000E39226000E3F0F6FF60009C
:104F7000E7F0F7FF000EF86E0F0EF76409D0090096
:104F80006F00D4FF38F009006F00D4FF39F00CD067
:104F90006F00DBFFE9FF6F00DFFFEAFF6F00B8FF84
:104FA00038F06F00B8FF39F002D8E0EF27F00500C5
:104FB000FA6E3850FD6E3950FE6EFF6AFA501200DC
:104FC0004BEF29F0FC0EE3500C0F386EFD0E6F0016
:104FD0008CFF39F0000E39226000E3F0F6FF60002C
:104FE000E7F0F7FF000EF86E0F0EF76409D0090026
:104FF0006F00D4FF38F009006F00D4FF39F00CD0F7
:105000006F00DBFFE9FF6F00DFFFEAFF6F00B8FF13
:1050100038F06F00B8FF39F038503910D8B413EFBA
:1050200028F015EF28F04BEF29F0FC0EE3500E0F9F
:10503000386EFD0E6F008CFF39F0000E39226000D3
:10504000E3F0F6FF6000E7F0F7FF000EF86E0F0EDA
:10505000F76409D009006F00D4FF38F009006F0031
:10506000D4FF39F00CD06F00DBFFE9FF6F00DFFFEA
:10507000EAFF6F00B8FF38F06F00B8FF39F060004A
:10508000E3F0E6FF6000E7F0E6FFFA0EE3500C0FF6
:10509000386EFB0E6F008CFF39F0000E3922600075
:1050A000E3F0F6FF6000E7F0F7FF000EF86E0F0E7A
:1050B000F76409D009006F00D4FF38F009006F00D1
:1050C000D4FF39F00CD06F00DBFFE9FF6F00DFFF8A
:1050D000EAFF6F00B8FF38F06F00B8FF39F002D870
:1050E0007BEF28F00500FA6E3850FD6E3950FE6EE9
:1050F000FF6AFA5012004BEF29F0FC0EE350100F3C
:10510000386EFD0E6F008CFF39F0000E3922600002
:10511000E3F0F6FF6000E7F0F7FF000EF86E0F0E09
:10512000F76409D009006F00D4FF38F009006F0060
:10513000D4FF39F00CD06F00DBFFE9FF6F00DFFF19
:10514000EAFF6F00B8FF38F06F00B8FF39F0385051
:105150003910D8B4AEEF28F0B0EF28F04BEF29F0BB
:10516000FC0EE350120F386EFD0E6F008CFF39F00D
:10517000000E39226000E3F0F6FF6000E7F0F7FF71
:10518000000EF86E0F0EF76409D009006F00D4FF0F
:1051900038F009006F00D4FF39F00CD06F00DBFF4E
:1051A000E9FF6F00DFFFEAFF6F00B8FF38F06F0024
:1051B000B8FF39F06000E3F0E6FF6000E7F0E6FFDB
:1051C000FA0EE350100F386EFB0E6F008CFF39F0B3
:1051D000000E39226000E3F0F6FF6000E7F0F7FF11
:1051E000000EF86E0F0EF76409D009006F00D4FFAF
:1051F00038F009006F00D4FF39F00CD06F00DBFFEE
:10520000E9FF6F00DFFFEAFF6F00B8FF38F06F00C3
:10521000B8FF39F002D816EF29F00500FA6E3850C1
:10522000FD6E3950FE6EFF6AFA5012004BEF29F006
:10523000FC0E6F008FFFF6FFFD0E6F008FFFF7FF74
:10524000000EF86E0F0EF76403D00800F55007D07B
:105250006F00DBFFE9FF6F00DFFFEAFFEF50386E02
:10526000396A3950000AD8B438EF29F04BEF29F0E9
:105270003850000AD8B44BEF29F0010AD8B447EFF0
:1052800027F0030AD8B4E2EF27F0010AD8B47DEF83
:1052900028F04BEF29F0FA0EE126FF0EE222120071
:1052A0000A0EE126000EE222EF0E6F008CFF36F0B0
:1052B000F00E6F008CFF37F0F10E6F008CFF38F0AE
:1052C000F20E6F008CFF39F0F60E6000DBF0E3FFAA
:1052D000F70E6000DFF0E3FFF80E6000E3F0E3FF9D
:1052E000F90E6000E7F0E3FFF90EE124D96EFF0E3E
:1052F000E220DA6EDF50396EFA0E6000E7F0E3FF6D
:10530000F80EE124D96EFF0EE220DA6EFB0EE124E6
:10531000E96EFF0EE220EA6E6F007FFFEFFFF70EEF
:10532000E124D96EFF0EE220DA6EFC0EE124E96E74
:10533000FF0EE220EA6E6F007FFFEFFFFD0EE1241B
:10534000D96EFF0EE220DA6EF60E6F008FFFDFFFE0
:10535000EF0E6F008CFF2EF0FE0E6000BBF0E3FF3F
:10536000F00E6F008CFF2EF0FF0E6000BBF0E3FF2D
:10537000BAEF2EF0F40EE350D8A4C1EF29F0C3EF3A
:1053800029F015EF2AF0F70EE124D96EFF0EE22086
:10539000DA6EDF50D8B4CFEF29F0D1EF29F0D3EF98
:1053A00029F06CEC60F0F60E6F008CFF01F0F90E46
:1053B000E124D96EFF0EE220DA6EDF50026E01505A
:1053C000E66E010EE66E8FEC5FF00250E66E020EA6
:1053D000E66E8FEC5FF00250E66E63EC60F060000A
:1053E000BBF0E6FF6000BFF0E6FFEDEC5BF0000E07
:1053F000E66E000EE66E000EE66E000EE66E000E25
:10540000E66E000EE66E000EE66E000EE66E000E14
:10541000E66E000EE66E63EC60F06000BBF0E6FF47
:105420006000BFF0E6FFA9EC58F0F40EE304D8A446
:105430001CEF2AF01EEF2AF041EF2AF0E150FA0F9C
:10544000D96EE250DA6EFF0EDA226F0078FF03F0B9
:105450006F0078FF04F06F0078FF05F06F0078FFB1
:1054600006F060000FF0E6FF600013F0E6FF60005A
:1054700017F0E6FF60001BF0E6FF030EE66E8DEC12
:1054800053F0F40E6F008CFF2EF0020E2E18D8A4ED
:105490004CEF2AF04EEF2AF083EF2AF0E150FA0F9A
:1054A000D96EE250DA6EFF0EDA226F0078FF07F055
:1054B0006F0078FF08F06F0078FF09F06F0078FF49
:1054C0000AF060001FF0E6FF600023F0E6FF6000D6
:1054D00027F0E6FF60002BF0E6FF070EE66E8DEC8E
:1054E00053F060001FF0E6FF600023F0E6FF60006D
:1054F00027F0E6FF60002BF0E6FF050EE66E000EDB
:10550000E66E9BEC3AF0F40E6F008CFF2EF0030E6B
:105510002E18D8A48EEF2AF090EF2AF0B3EF2AF0DD
:10552000E150FA0FD96EE250DA6EFF0EDA226F0008
:1055300078FF0BF06F0078FF0CF06F0078FF0DF034
:105540006F0078FF0EF060002FF0E6FF600033F090
:10555000E6FF600037F0E6FF60003BF0E6FF0B0E71
:10556000E66E8DEC53F0F40E6F008CFF2EF0040EFF
:105570002E18D8A4BEEF2AF0C0EF2AF0D8EF2AF0F8
:10558000F60E6F008CFF0FF0F70EE124D96EFF0EC0
:10559000E220DA6EDF50106E0F50E66E0F0EE66EF0
:1055A0008FEC5FF01050E66E100EE66E8FEC5FF041
:1055B000F40E6F008CFF2EF0050E2E18D8A4E3EF2A
:1055C0002AF0E5EF2AF009EF2BF0F60E6F008CFFC2
:1055D00015F0F70EE124D96EFF0EE220DA6EDF50EF
:1055E000196E1550E66E150EE66E8FEC5FF01950D1
:1055F000E66E190EE66E8FEC5FF0000EE66E000EA2
:10560000E66E40EC5CF0020EE66E100EE66EB0EC5C
:105610004DF0F40E6F008CFF2EF0060E2E18D8A45D
:1056200014EF2BF016EF2BF07AEF2BF0F60E6F0045
:105630008CFF11F0F70EE124D96EFF0EE220DA6E36
:10564000DF50126EF80EE124D96EFF0EE220DA6E02
:10565000DF50136EF90EE124D96EFF0EE220DA6EF0
:10566000DF50146E1150E66E110EE66E8FEC5FF097
:105670001250E66E120EE66E8FEC5FF01350E66E7F
:10568000130EE66E8FEC5FF01450E66E140EE66EAD
:105690008FEC5FF01450E66E5AEC60F06000BBF0E7
:1056A000E6FF6000BFF0E6FFEDEC5BF0000EE66E9B
:1056B000000EE66E000EE66E000EE66E000EE66E62
:1056C000000EE66E000EE66E000EE66E000EE66E52
:1056D000000EE66E5AEC60F06000BBF0E6FF600082
:1056E000BFF0E6FFA9EC58F0000EE66E000EE66E85
:1056F00023EC56F0F40E6F008CFF2EF0070E2E18E0
:10570000D8A485EF2BF087EF2BF0E5EF2BF0F60E0A
:105710006F008CFF18F0F70EE124D96EFF0EE22027
:10572000DA6EDF50166EF80EE124D96EFF0EE2201D
:10573000DA6EDF50176E1850E66E180EE66E8FECBC
:105740005FF01650E66E160EE66E8FEC5FF01750A7
:10575000E66E170EE66E8FEC5FF01850E66E48ECC2
:1057600060F0010E2E26000E2F226000BBF0E6FF37
:105770006000BFF0E6FFEDEC5BF0000EE66E000EA1
:10578000E66E000EE66E000EE66E000EE66E000E91
:10579000E66E000EE66E000EE66E000EE66E000E81
:1057A000E66E48EC60F0010E2E26000E2F226000FF
:1057B000BBF0E6FF6000BFF0E6FFA9EC58F0030E77
:1057C000E66E100EE66E2FEC55F0F40E6F008CFFB7
:1057D0002EF0080E2E18D8A4F0EF2BF0F2EF2BF0DD
:1057E0002CEF2CF0F60E6F008CFF1AF0F70EE12470
:1057F000D96EFF0EE220DA6EDF501B6EF80EE12448
:10580000D96EFF0EE220DA6EDF501C6EF90EE12435
:10581000D96EFF0EE220DA6EDF501D6E1A50E66E72
:105820001A0EE66E8FEC5FF01B50E66E1B0EE66EF6
:105830008FEC5FF01C50E66E1C0EE66E8FEC5FF096
:105840001D50E66E1D0EE66E8FEC5FF0000EE66EEC
:10585000000EE66EE8EC55F0F40E6F008CFF2EF0B3
:10586000090E2E18D8A437EF2CF039EF2CF0E4EF06
:105870002EF0F60E6F008CFF1EF0F70EE124D96EAD
:10588000FF0EE220DA6EDF501F6E1E50E66E1E0E17
:10589000E66E8FEC5FF01F50E66E1F0EE66E8FEC2B
:1058A0005FF0E4EF2EF0F40EE304D8A45AEF2CF0EE
:1058B0005CEF2CF075EF2CF0F70EE124D96EFF0EA3
:1058C000E220DA6EDF50E66EFEEC42F0F60EE350B8
:1058D000E66EEDEC41F036EC60F06000BBF0E6FF08
:1058E0006000BFF0E6FF35EC58F0F40E6F008CFF5F
:1058F0002EF00F0E2E18D8A480EF2CF082EF2CF093
:10590000E4EF2EF05AEC60F06000BBF0E6FF6000C0
:10591000BFF0E6FF66EC5FF05AEC60F06000BBF0B1
:10592000D9FF6000BFF0DAFF180EDE18D8A49BEF95
:105930002CF09DEF2CF0E4EF2EF0110EE66E51EC02
:1059400060F02E50116E120EE66E51EC60F02E508B
:10595000126E130EE66E51EC60F02E50136E140EA4
:10596000E66E51EC60F02E50146E1450E66E5AEC58
:1059700060F06000BBF0E6FF6000BFF0E6FFEDEC1A
:105980005BF0000EE66E000EE66E000EE66E000E98
:10599000E66E000EE66E000EE66E000EE66E000E7F
:1059A000E66E000EE66E000EE66E5AEC60F06000E9
:1059B000BBF0E6FF6000BFF0E6FFE3EC58F0000E3E
:1059C000E66E000EE66E000EE66E000EE66E000E4F
:1059D000E66E000EE66E000EE66E000EE66E000E3F
:1059E000E66E000EE66E5AEC60F06000BBF0E6FF7B
:1059F0006000BFF0E6FFEDEC5AF0000EE66E000E20
:105A0000E66E000EE66E000EE66E000EE66E000E0E
:105A1000E66E000EE66E000EE66E000EE66E000EFE
:105A2000E66E5AEC60F06000BBF0E6FF6000BFF08D
:105A3000E6FFB3EC5AF0E4EF2EF0F40EE350D8A4F6
:105A400024EF2DF026EF2DF03FEF2DF0FA0E6F0032
:105A50008FFFE6FF6F008FFFE6FF6F008FFFE6FF0F
:105A60006F008FFFE6FF6CEC4AF048EC60F06000DE
:105A7000BBF0E6FF6000BFF0E6FF6FEC58F0F40EFD
:105A80006F008CFF2EF00F0E2E18D8A44AEF2DF0C9
:105A90004CEF2DF0E4EF2EF048EC60F0010E2E26D6
:105AA000000E2F226000BBF0E6FF6000BFF0E6FFB3
:105AB00066EC5FF048EC60F0010E2E24D96E000E0B
:105AC0002F20DA6E180EDE18D8A469EF2DF06BEFD8
:105AD0002DF0E4EF2EF0160EE66E51EC60F02E5035
:105AE000166E170EE66E51EC60F02E50176E180E03
:105AF000E66E51EC60F02E50186E000EE66E000E51
:105B0000E66E000EE66E000EE66E000EE66E000E0D
:105B1000E66E000EE66E000EE66E000EE66E000EFD
:105B2000E66E48EC60F0010E2E26000E2F2260007B
:105B3000BBF0E6FF6000BFF0E6FFE3EC58F0000EBC
:105B4000E66E000EE66E000EE66E000EE66E000ECD
:105B5000E66E000EE66E000EE66E000EE66E000EBD
:105B6000E66E000EE66E48EC60F0010E2E26000E8A
:105B70002F226000BBF0E6FF6000BFF0E6FFEDEC17
:105B80005AF0E4EF2EF0F40EE304D8A4CAEF2DF09F
:105B9000CCEF2DF001EF2EF0E150FA0FD96EE2506C
:105BA000DA6EFF0EDA226F0078FF68F06F0078FF80
:105BB00069F06F0078FF6AF06F0078FF6BF0000EFD
:105BC000E66E000EE66E000EE66E000EE66E000E4D
:105BD000E66E000EE66E000EE66E000EE66E000E3D
:105BE000E66E000EE66E36EC60F0010E2E26000E1C
:105BF0002F226000BBF0E6FF6000BFF0E6FFB3ECD1
:105C00005AF0F40E6F008CFF2EF00F0E2E18D8A451
:105C10000CEF2EF00EEF2EF0E4EF2EF036EC60F0ED
:105C2000010E2E26000E2F226000BBF0E6FF600062
:105C3000BFF0E6FF66EC5FF036EC60F0010E2E245C
:105C4000D96E000E2F20DA6E180EDE18D8A42BEFB6
:105C50002EF02DEF2EF077EF2EF0190EE66E51ECB0
:105C600060F02E50196E000EE66E000EE66E000E0D
:105C7000E66E000EE66E000EE66E000EE66E000E9C
:105C8000E66E000EE66EF40EE66E010EE66E36EC83
:105C900060F0010E2E26000E2F226000BBF0E6FF02
:105CA0006000BFF0E6FFE3EC58F0000EE66E000E79
:105CB000E66E000EE66E000EE66E000EE66E000E5C
:105CC000E66E000EE66E000EE66EE80EE66E030E61
:105CD000E66E36EC60F0010E2E26000E2F226000DC
:105CE000BBF0E6FF6000BFF0E6FFEDEC5AF0E150DC
:105CF000FE0FD96EE250DA6EFF0EDA22DFA883EFD4
:105D00002EF085EF2EF0E4EF2EF036EC60F0010E71
:105D10002E24D96E000E2F20DA6E160EDE18D8A4AF
:105D200094EF2EF096EF2EF0E4EF2EF0000EE66EDC
:105D3000000EE66E000EE66E000EE66E000EE66EDB
:105D4000000EE66E000EE66E000EE66EE80EE66EE3
:105D5000030EE66E36EC60F0010E2E26000E2F22AA
:105D60006000BBF0E6FF6000BFF0E6FFB3EC5AF066
:105D7000E4EF2EF0F50EE350386E396A3950000A20
:105D8000D8B4C5EF2EF0E4EF2EF03850000AD8B4A6
:105D9000BAEF29F0020AD8B453EF2CF0010AD8B4B4
:105DA000E4EF2EF0070AD8B41DEF2DF0010AD8B4A5
:105DB000C3EF2DF0030AD8B4E4EF2EF0010AD8B4F3
:105DC000E4EF2EF0E4EF2EF0EF0EE126FF0EE222DC
:105DD0001200E652E652E652FB0E6F008FFFE6FF1E
:105DE0006F008FFFE6FFC2EC5EF0FE0E6000BFF0BA
:105DF000E3FFFD0E6000BBF0E3FFFD0E6F008FFFC1
:105E0000F6FFFE0E6F008FFFF7FF000EF86E0F0E0D
:105E1000F76403D00800F55007D06F00DBFFE9FFFF
:105E20006F00DFFFEAFFEF50396EFF0E6000E7F012
:105E3000E3FFFB0E6F008FFFE6FF6F008FFFE6FFB3
:105E400082EC5FF0FB0E6F008FFFE6FF6F008FFFAD
:105E5000E6FF24EC5EF0F80EE126FF0EE222B2EF40
:105E600030F0FB0E6F008FFFD9FFFC0E6F008FFF2D
:105E7000DAFFDF50640AD8A440EF2FF042EF2FF092
:105E8000E5EF30F0FD0E6F008FFFF6FFFE0E6F00A6
:105E90008FFFF7FF000EF86E0F0EF76404D0650E4B
:105EA000F56E0C0008D06F00DBFFE9FF6F00DFFF2D
:105EB000EAFF650EEF6EFD0EE350010F386EFE0E29
:105EC0006F008CFF39F0000E39226000E3F0E6FF2E
:105ED0006000E7F0E6FF5FEC5BF0E5EF30F0FB0E13
:105EE0006F008FFFD9FFFC0E6F008FFFDAFFDF50CE
:105EF000650AD8A47EEF2FF080EF2FF099EF2FF0F6
:105F0000FD0E6F008FFFF6FFFE0E6F008FFFF7FF95
:105F1000000EF86E0F0EF76404D0660EF56E0C00DE
:105F200008D06F00DBFFE9FF6F00DFFFEAFF660EBE
:105F3000EF6E1850E66EFC0EE350010F386EFD0E4A
:105F40006F008CFF39F0000E39226000E3F0E6FFAD
:105F50006000E7F0E6FFEDEC5BF0000EE66E000E91
:105F6000E66E000EE66E000EE66E000EE66E000EA9
:105F7000E66E000EE66E000EE66E640EE66E000E35
:105F8000E66EF30EE350010F386EF40E6F008CFFD7
:105F900039F0000E39226000E3F0E6FF6000E7F020
:105FA000E6FFEDEC5AF0000EE66E000EE66E000E17
:105FB000E66E000EE66E000EE66E000EE66E000E59
:105FC000E66E000EE66EC80EE66E000EE66EF30E8E
:105FD000E350010F386EF40E6F008CFF39F0000EA5
:105FE00039226000E3F0E6FF6000E7F0E6FFB3EC83
:105FF0005AF0E5EF30F0FB0E6F008FFFD9FFFC0E7B
:106000006F008FFFDAFFDF50660AD8A40AEF30F086
:106010000CEF30F025EF30F0FD0E6F008FFFF6FF34
:10602000FE0E6F008FFFF7FF000EF86E0F0EF76485
:1060300004D0670EF56E0C0008D06F00DBFFE9FF9F
:106040006F00DFFFEAFF670EEF6EFB0E6F008FFF42
:10605000D9FFFC0E6F008FFFDAFFDF50690AD8A46A
:1060600034EF30F036EF30F06DEF30F0660EE66E64
:10607000000EE66E42EC54F01750D8A442EF30F018
:1060800044EF30F046EF30F0010E176E000EE66E72
:10609000000EE66E000EE66E000EE66E000EE66E78
:1060A000000EE66E000EE66E000EE66E1750050D51
:1060B0006F00CCFF38F06F00D0FF39F06000E3F0E4
:1060C000E6FF6000E7F0E6FFF30E6F008FFFE6FFEC
:1060D0006F008FFFE6FFFBEC57F0FB0E6F008FFFAA
:1060E000D9FFFC0E6F008FFFDAFFDF50680AD8A4DB
:1060F0007CEF30F07EEF30F0E5EF30F0700EE66EC2
:10610000000EE66E6EEC55F0E5EF30F0FB0E6F0022
:106110008FFFD9FFFC0E6F008FFFDAFFDF50670A99
:10612000D8A495EF30F097EF30F0E5EF30F0FD0EAA
:106130006F008FFFF6FFFE0E6F008FFFF7FF000E60
:10614000F86E0F0EF76404D0650EF56E0C0008D0E3
:106150006F00DBFFE9FF6F00DFFFEAFF650EEF6E08
:10616000E5EF30F0FD0E6F008FFFF6FFFE0E6F00C3
:106170008FFFF7FF000EF86E0F0EF76403D00800D4
:10618000F55007D06F00DBFFE9FF6F00DFFFEAFF8C
:10619000EF50386E396A3950000AD8B4D2EF30F077
:1061A000E5EF30F03850640AD8B431EF2FF0010A2F
:1061B000D8B46FEF2FF0030AD8B4FBEF2FF0010A29
:1061C000D8B486EF30F0E5EF30F0FF0E6F008CFFB3
:1061D00039F0FD0E6F008FFFF6FFFE0E6F008FFF90
:1061E000F7FF000EF86E0F0EF76403D00800F550AD
:1061F00007D06F00DBFFE9FF6F00DFFFEAFFEF5022
:106200003918D8B406EF31F008EF31F05BEF33F016
:10621000FF0EE350386E396A3950000AD8B413EFD4
:1062200031F028EF33F03850640AD8B428EF33F057
:10623000010AD8B428EF33F0030AD8B428EF33F0BA
:10624000010AD8B428EF33F028EF33F0FD0EE35005
:10625000380F386EFE0E6F008CFF39F0000E3922B9
:106260006000E3F0F6FF6000E7F0F7FF000EF86E65
:106270000F0EF76409D009006F00D4FF38F0090051
:106280006F00D4FF39F00CD06F00DBFFE9FF6F0027
:10629000DFFFEAFF6F00B8FF38F06F00B8FF39F09A
:1062A00038503910D8B457EF31F059EF31F05BEF77
:1062B00033F0FD0EE3503A0F386EFE0E6F008CFF88
:1062C00039F0000E39226000E3F0F6FF6000E7F0DD
:1062D000F7FF000EF86E0F0EF76409D009006F008B
:1062E000D4FF38F009006F00D4FF39F00CD06F00F4
:1062F000DBFFE9FF6F00DFFFEAFF6F00B8FF38F058
:106300006F00B8FF39F06000E3F0E6FF6000E7F0EF
:10631000E6FFFB0EE350380F386EFC0E6F008CFF6B
:1063200039F0000E39226000E3F0F6FF6000E7F07C
:10633000F7FF000EF86E0F0EF76409D009006F002A
:10634000D4FF38F009006F00D4FF39F00CD06F0093
:10635000DBFFE9FF6F00DFFFEAFF6F00B8FF38F0F7
:106360006F00B8FF39F002D8BFEF31F00500FA6EC8
:106370003850FD6E3950FE6EFF6AFA5012005BEF26
:1063800033F01750D8A4C7EF31F0C9EF31F0CBEF9D
:1063900031F0010E176E000EE66E000EE66E000E76
:1063A000E66E000EE66E000EE66E000EE66E000E65
:1063B000E66E000EE66E1750050D6F00CCFF38F04C
:1063C0006F00D0FF39F06000E3F0E6FF6000E7F017
:1063D000E6FFF30E6F008FFFE6FF6F008FFFE6FF13
:1063E000FBEC57F0FD0EE3503C0F386EFE0E6F00D5
:1063F0008CFF39F0000E39226000E3F0F6FF6000F8
:10640000E7F0F7FF000EF86E0F0EF76409D00900F1
:106410006F00D4FF38F009006F00D4FF39F00CD0C2
:106420006F00DBFFE9FF6F00DFFFEAFF6F00B8FFDF
:1064300038F06F00B8FF39F038503910D8B423EF76
:1064400032F025EF32F05BEF33F0FD0EE3503E0FFC
:10645000386EFE0E6F008CFF39F0000E392260009E
:10646000E3F0F6FF6000E7F0F7FF000EF86E0F0EA6
:10647000F76409D009006F00D4FF38F009006F00FD
:10648000D4FF39F00CD06F00DBFFE9FF6F00DFFFB6
:10649000EAFF6F00B8FF38F06F00B8FF39F0600016
:1064A000E3F0E6FF6000E7F0E6FFFB0EE3503C0F91
:1064B000386EFC0E6F008CFF39F0000E3922600040
:1064C000E3F0F6FF6000E7F0F7FF000EF86E0F0E46
:1064D000F76409D009006F00D4FF38F009006F009D
:1064E000D4FF39F00CD06F00DBFFE9FF6F00DFFF56
:1064F000EAFF6F00B8FF38F06F00B8FF39F002D83C
:106500008BEF32F00500FA6E3850FD6E3950FE6E9A
:10651000FF6AFA5012005BEF33F0FD0EE350400FBC
:10652000386EFE0E6F008CFF39F0000E39226000CD
:10653000E3F0F6FF6000E7F0F7FF000EF86E0F0ED5
:10654000F76409D009006F00D4FF38F009006F002C
:10655000D4FF39F00CD06F00DBFFE9FF6F00DFFFE5
:10656000EAFF6F00B8FF38F06F00B8FF39F038501D
:106570003910D8B4BEEF32F0C0EF32F05BEF33F039
:10658000FD0EE350420F386EFE0E6F008CFF39F0A7
:10659000000E39226000E3F0F6FF6000E7F0F7FF3D
:1065A000000EF86E0F0EF76409D009006F00D4FFDB
:1065B00038F009006F00D4FF39F00CD06F00DBFF1A
:1065C000E9FF6F00DFFFEAFF6F00B8FF38F06F00F0
:1065D000B8FF39F06000E3F0E6FF6000E7F0E6FFA7
:1065E000FB0EE350400F386EFC0E6F008CFF39F04D
:1065F000000E39226000E3F0F6FF6000E7F0F7FFDD
:10660000000EF86E0F0EF76409D009006F00D4FF7A
:1066100038F009006F00D4FF39F00CD06F00DBFFB9
:10662000E9FF6F00DFFFEAFF6F00B8FF38F06F008F
:10663000B8FF39F002D826EF33F00500FA6E385073
:10664000FD6E3950FE6EFF6AFA5012005BEF33F0B8
:10665000FD0E6F008FFFF6FFFE0E6F008FFFF7FF3E
:10666000000EF86E0F0EF76403D00800F55007D047
:106670006F00DBFFE9FF6F00DFFFEAFFEF50386ECE
:10668000396A3950000AD8B448EF33F05BEF33F081
:106690003850640AD8B45BEF33F0010AD8B426EF5F
:1066A00031F0030AD8B4C1EF31F0010AD8B48DEF4C
:1066B00032F05BEF33F0FB0EE126FF0EE222120018
:1066C000E652E652E652FB0E6F008FFFE6FF6F00C8
:1066D0008FFFE6FFC2EC5EF0FE0E6000BFF0E3FF4E
:1066E000FD0E6000BBF0E3FFFD0E6F008FFFF6FFB5
:1066F000FE0E6F008FFFF7FF000EF86E0F0EF764AF
:1067000003D00800F55007D06F00DBFFE9FF6F00F2
:10671000DFFFEAFFEF50396EFF0E6000E7F0E3FFA6
:10672000FB0E6F008FFFE6FF6F008FFFE6FF82EC2E
:106730005FF0FB0E6F008FFFE6FF6F008FFFE6FF3D
:1067400024EC5EF0F80EE126FF0EE22281EF34F039
:10675000FB0E6F008FFFD9FFFC0E6F008FFFDAFF7B
:10676000DF506E0AD8A4B7EF33F0B9EF33F0B4EFCF
:1067700034F0FD0E6F008FFFF6FFFE0E6F008FFFEF
:10678000F7FF000EF86E0F0EF76404D06F0EF56E73
:106790000C0008D06F00DBFFE9FF6F00DFFFEAFFAE
:1067A0006F0EEF6EFD0EE350010F386EFE0E6F00A0
:1067B0008CFF39F0000E39226000E3F0E6FF600044
:1067C000E7F0E6FF5FEC5BF0B4EF34F0FB0E6F0038
:1067D0008FFFD9FFFC0E6F008FFFDAFFDF506F0ACB
:1067E000D8A4F5EF33F0F7EF33F0B4EF34F0FD0E4B
:1067F0006F008FFFF6FFFE0E6F008FFFF7FF000E9A
:10680000F86E0F0EF76404D0700EF56E0C0008D011
:106810006F00DBFFE9FF6F00DFFFEAFF700EEF6E36
:10682000B4EF34F0FB0E6F008FFFD9FFFC0E6F004A
:106830008FFFDAFFDF50700AD8A421EF34F023EF86
:1068400034F03CEF34F0FD0E6F008FFFF6FFFE0ECC
:106850006F008FFFF7FF000EF86E0F0EF76404D085
:10686000710EF56E0C0008D06F00DBFFE9FF6F00C2
:10687000DFFFEAFF710EEF6EFB0E6F008FFFD9FF97
:10688000FC0E6F008FFFDAFFDF50720AD8A44BEFC7
:1068900034F04DEF34F0B4EF34F06C0EE66E000ED1
:1068A000E66EB4EC4FF0B4EF34F0FB0E6F008FFFE8
:1068B000D9FFFC0E6F008FFFDAFFDF50710AD8A4FA
:1068C00064EF34F066EF34F0B4EF34F0FD0E6F0097
:1068D0008FFFF6FFFE0E6F008FFFF7FF000EF86EC2
:1068E0000F0EF76404D06F0EF56E0C0008D06F0029
:1068F000DBFFE9FF6F00DFFFEAFF6F0EEF6EB4EF23
:1069000034F0FD0E6F008FFFF6FFFE0E6F008FFF5D
:10691000F7FF000EF86E0F0EF76403D00800F55075
:1069200007D06F00DBFFE9FF6F00DFFFEAFFEF50EA
:10693000386E396A3950000AD8B4A1EF34F0B4EF98
:1069400034F038506E0AD8B4A8EF33F0010AD8B446
:10695000E6EF33F01F0AD8B412EF34F0010AD8B4CE
:1069600055EF34F0B4EF34F0FF0E6F008CFF39F0C8
:10697000FD0E6F008FFFF6FFFE0E6F008FFFF7FF1B
:10698000000EF86E0F0EF76403D00800F55007D024
:106990006F00DBFFE9FF6F00DFFFEAFFEF50391800
:1069A000D8B4D5EF34F0D7EF34F033EF37F0FF0E33
:1069B000E350386E396A3950000AD8B4E2EF34F047
:1069C00000EF37F038506E0AD8B400EF37F0010A04
:1069D000D8B400EF37F01F0AD8B400EF37F0010A3F
:1069E000D8B400EF37F000EF37F0FD0EE350380F6A
:1069F000386EFE0E6F008CFF39F0000E39226000F9
:106A0000E3F0F6FF6000E7F0F7FF000EF86E0F0E00
:106A1000F76409D009006F00D4FF38F009006F0057
:106A2000D4FF39F00CD06F00DBFFE9FF6F00DFFF10
:106A3000EAFF6F00B8FF38F06F00B8FF39F0385048
:106A40003910D8B426EF35F028EF35F08EEF35F059
:106A5000FD0EE3503A0F386EFE0E6F008CFF39F0DA
:106A6000000E39226000E3F0F6FF6000E7F0F7FF68
:106A7000000EF86E0F0EF76409D009006F00D4FF06
:106A800038F009006F00D4FF39F00CD06F00DBFF45
:106A9000E9FF6F00DFFFEAFF6F00B8FF38F06F001B
:106AA000B8FF39F06000E3F0E6FF6000E7F0E6FFD2
:106AB000FB0EE350380F386EFC0E6F008CFF39F080
:106AC000000E39226000E3F0F6FF6000E7F0F7FF08
:106AD000000EF86E0F0EF76409D009006F00D4FFA6
:106AE00038F009006F00D4FF39F00CD06F00DBFFE5
:106AF000E9FF6F00DFFFEAFF6F00B8FF38F06F00BB
:106B0000B8FF39F002D88EEF35F00500FA6E385034
:106B1000FD6E3950FE6EFF6AFA5012001950E66E93
:106B2000FC0EE350010F386EFD0E6F008CFF39F044
:106B3000000E39226000E3F0E6FF6000E7F0E6FFB8
:106B4000EDEC5BF0000EE66E000EE66E000EE66EFB
:106B5000000EE66E000EE66E000EE66E000EE66EAD
:106B6000000EE66EF40EE66E010EE66EF30EE350D6
:106B7000010F386EF40E6F008CFF39F0000E3922D1
:106B80006000E3F0E6FF6000E7F0E6FFEDEC5AF0AE
:106B900033EF37F0FD0EE3503C0F386EFE0E6F0002
:106BA0008CFF39F0000E39226000E3F0F6FF600040
:106BB000E7F0F7FF000EF86E0F0EF76409D009003A
:106BC0006F00D4FF38F009006F00D4FF39F00CD00B
:106BD0006F00DBFFE9FF6F00DFFFEAFF6F00B8FF28
:106BE00038F06F00B8FF39F038503910D8B4FBEFE7
:106BF00035F0FDEF35F033EF37F0FD0EE3503E0F8B
:106C0000386EFE0E6F008CFF39F0000E39226000E6
:106C1000E3F0F6FF6000E7F0F7FF000EF86E0F0EEE
:106C2000F76409D009006F00D4FF38F009006F0045
:106C3000D4FF39F00CD06F00DBFFE9FF6F00DFFFFE
:106C4000EAFF6F00B8FF38F06F00B8FF39F060005E
:106C5000E3F0E6FF6000E7F0E6FFFB0EE3503C0FD9
:106C6000386EFC0E6F008CFF39F0000E3922600088
:106C7000E3F0F6FF6000E7F0F7FF000EF86E0F0E8E
:106C8000F76409D009006F00D4FF38F009006F00E5
:106C9000D4FF39F00CD06F00DBFFE9FF6F00DFFF9E
:106CA000EAFF6F00B8FF38F06F00B8FF39F002D884
:106CB00063EF36F00500FA6E3850FD6E3950FE6E07
:106CC000FF6AFA50120033EF37F0FD0EE350400F29
:106CD000386EFE0E6F008CFF39F0000E3922600016
:106CE000E3F0F6FF6000E7F0F7FF000EF86E0F0E1E
:106CF000F76409D009006F00D4FF38F009006F0075
:106D0000D4FF39F00CD06F00DBFFE9FF6F00DFFF2D
:106D1000EAFF6F00B8FF38F06F00B8FF39F0385065
:106D20003910D8B496EF36F098EF36F033EF37F0ED
:106D3000FD0EE350420F386EFE0E6F008CFF39F0EF
:106D4000000E39226000E3F0F6FF6000E7F0F7FF85
:106D5000000EF86E0F0EF76409D009006F00D4FF23
:106D600038F009006F00D4FF39F00CD06F00DBFF62
:106D7000E9FF6F00DFFFEAFF6F00B8FF38F06F0038
:106D8000B8FF39F06000E3F0E6FF6000E7F0E6FFEF
:106D9000FB0EE350400F386EFC0E6F008CFF39F095
:106DA000000E39226000E3F0F6FF6000E7F0F7FF25
:106DB000000EF86E0F0EF76409D009006F00D4FFC3
:106DC00038F009006F00D4FF39F00CD06F00DBFF02
:106DD000E9FF6F00DFFFEAFF6F00B8FF38F06F00D8
:106DE000B8FF39F002D8FEEF36F00500FA6E3850E1
:106DF000FD6E3950FE6EFF6AFA50120033EF37F025
:106E0000FD0E6F008FFFF6FFFE0E6F008FFFF7FF86
:106E1000000EF86E0F0EF76403D00800F55007D08F
:106E20006F00DBFFE9FF6F00DFFFEAFFEF50386E16
:106E3000396A3950000AD8B420EF37F033EF37F011
:106E400038506E0AD8B433EF37F0010AD8B4F5EFF2
:106E500034F01F0AD8B4CAEF35F0010AD8B465EF90
:106E600036F033EF37F0FB0EE126FF0EE222120080
:106E7000E652E652E652E652FF0EE36AFE0EE36A7F
:106E8000FD0EE36AFC0EE36A3701E0B74AEF37F024
:106E90004CEF37F060EF38F0FC0EE1242E6EFF0E61
:106EA000E2202F6E6000BBF0E6FF6000BFF0E6FF5F
:106EB000FB0EE1242E6EFF0EE2202F6E6000BBF071
:106EC000E6FF6000BFF0E6FFFA0EE1242E6EFF0E33
:106ED000E2202F6E6000BBF0E6FF6000BFF0E6FF2F
:106EE000F90EE1242E6EFF0EE2202F6E6000BBF043
:106EF000E6FF6000BFF0E6FFF20E6F008FFFD9FFE4
:106F0000F30E6F008FFFDAFFDF50E66EF10E6F00B9
:106F10008CFF38F0F20E6F008CFF39F0010E382430
:106F2000D96E000E3920DA6E6F007BFFE6FF6F002E
:106F30007BFFE6FF6F007BFFE6FF6F007BFFE6FF56
:106F4000CFEC40F0FF0E6F008FFFE3F7FE0E6F00F7
:106F50008FFFE4F7FD0E6F008FFFE1F7FC0E6F006F
:106F60008FFFE2F7FA0E6F008CFF38F0FB0E6F0018
:106F70008CFF39F0050E3824D96E000E3920DA6EF8
:106F8000DF50396EFA0E6F008CFF36F0FB0E6F008B
:106F90008CFF37F00E0E3624D96E000E3720DA6ED5
:106FA000DF50386E060E2E6ED89038362E2ED4EF67
:106FB00037F0385039103701E56FFA0E6F008CFF4B
:106FC00038F0FB0E6F008CFF39F0060E3824D96EB6
:106FD000000E3920DA6EDF50E66FFA0E6F008CFF7C
:106FE00038F0FB0E6F008CFF39F0070E3824D96E95
:106FF000000E3920DA6EDF50E76FFA0E6F008CFF5B
:1070000038F0FB0E6F008CFF39F0080E3824D96E73
:10701000000E3920DA6EDF50E86FFA0E6F008CFF39
:1070200038F0FB0E6F008CFF39F0090E3824D96E52
:10703000000E3920DA6EDF50E96FFA0E6F008CFF18
:1070400038F0FB0E6F008CFF39F00A0E3824D96E31
:10705000000E3920DA6EDF50EA6FFA0E6F008CFFF7
:1070600038F0FB0E6F008CFF39F00B0E3824D96E10
:10707000000E3920DA6EDF50EB6FFA0E6F008CFFD6
:1070800038F0FB0E6F008CFF39F00C0E3824D96EEF
:10709000000E3920DA6EDF50EC6FFA0E6F008CFFB5
:1070A00038F0FB0E6F008CFF39F00D0E3824D96ECE
:1070B000000E3920DA6EDF50ED6FE08796EF3AF080
:1070C000D0B765EF38F067EF38F07BEF39F0FC0EA2
:1070D000E1242E6EFF0EE2202F6E6000BBF0E6FF73
:1070E0006000BFF0E6FFFB0EE1242E6EFF0EE220F3
:1070F0002F6E6000BBF0E6FF6000BFF0E6FFFA0E07
:10710000E1242E6EFF0EE2202F6E6000BBF0E6FF42
:107110006000BFF0E6FFF90EE1242E6EFF0EE220C4
:107120002F6E6000BBF0E6FF6000BFF0E6FFF20EDE
:107130006F008FFFD9FFF30E6F008FFFDAFFDF5074
:10714000E66EF10E6F008CFF38F0F20E6F008CFFD0
:1071500039F0010E3824D96E000E3920DA6E6F0036
:107160007BFFE6FF6F007BFFE6FF6F007BFFE6FF24
:107170006F007BFFE6FFCFEC40F0FF0E6F008FFF4C
:10718000D3F7FE0E6F008FFFD4F7FD0E6F008FFF59
:10719000D1F7FC0E6F008FFFD2F7FA0E6F008CFF55
:1071A00038F0FB0E6F008CFF39F0050E3824D96ED5
:1071B000000E3920DA6EDF50396EFA0E6F008CFF48
:1071C00036F0FB0E6F008CFF37F00E0E3624D96EB2
:1071D000000E3720DA6EDF50386E060E2E6ED89015
:1071E00038362E2EEFEF38F0385039103701D56F82
:1071F000FA0E6F008CFF38F0FB0E6F008CFF39F039
:10720000060E3824D96E000E3920DA6EDF50D66FA4
:10721000FA0E6F008CFF38F0FB0E6F008CFF39F018
:10722000070E3824D96E000E3920DA6EDF50D76F82
:10723000FA0E6F008CFF38F0FB0E6F008CFF39F0F8
:10724000080E3824D96E000E3920DA6EDF50D86F60
:10725000FA0E6F008CFF38F0FB0E6F008CFF39F0D8
:10726000090E3824D96E000E3920DA6EDF50D96F3E
:10727000FA0E6F008CFF38F0FB0E6F008CFF39F0B8
:107280000A0E3824D96E000E3920DA6EDF50DA6F1C
:10729000FA0E6F008CFF38F0FB0E6F008CFF39F098
:1072A0000B0E3824D96E000E3920DA6EDF50DB6FFA
:1072B000FA0E6F008CFF38F0FB0E6F008CFF39F078
:1072C0000C0E3824D96E000E3920DA6EDF50DC6FD8
:1072D000FA0E6F008CFF38F0FB0E6F008CFF39F058
:1072E0000D0E3824D96E000E3920DA6EDF50DD6FB6
:1072F000D0875EEF38F0C0B780EF39F082EF39F019
:1073000096EF3AF0FC0EE1242E6EFF0EE2202F6E77
:107310006000BBF0E6FF6000BFF0E6FFFB0EE1247B
:107320002E6EFF0EE2202F6E6000BBF0E6FF6000C5
:10733000BFF0E6FFFA0EE1242E6EFF0EE2202F6E64
:107340006000BBF0E6FF6000BFF0E6FFF90EE1244D
:107350002E6EFF0EE2202F6E6000BBF0E6FF600095
:10736000BFF0E6FFF20E6F008FFFD9FFF30E6F0044
:107370008FFFDAFFDF50E66EF10E6F008CFF38F002
:10738000F20E6F008CFF39F0010E3824D96E000E1A
:107390003920DA6E6F007BFFE6FF6F007BFFE6FFB0
:1073A0006F007BFFE6FF6F007BFFE6FFCFEC40F056
:1073B000FF0E6F008FFFC3F7FE0E6F008FFFC4F745
:1073C000FD0E6F008FFFC1F7FC0E6F008FFFC2F73D
:1073D000FA0E6F008CFF38F0FB0E6F008CFF39F057
:1073E000050E3824D96E000E3920DA6EDF50396E62
:1073F000FA0E6F008CFF36F0FB0E6F008CFF37F03B
:107400000E0E3624D96E000E3720DA6EDF50386E3D
:10741000060E2E6ED89038362E2E0AEF3AF03850DF
:1074200039103701C56FFA0E6F008CFF38F0FB0E74
:107430006F008CFF39F0060E3824D96E000E39200B
:10744000DA6EDF50C66FFA0E6F008CFF38F0FB0E5D
:107450006F008CFF39F0070E3824D96E000E3920EA
:10746000DA6EDF50C76FFA0E6F008CFF38F0FB0E3C
:107470006F008CFF39F0080E3824D96E000E3920C9
:10748000DA6EDF50C86FFA0E6F008CFF38F0FB0E1B
:107490006F008CFF39F0090E3824D96E000E3920A8
:1074A000DA6EDF50C96FFA0E6F008CFF38F0FB0EFA
:1074B0006F008CFF39F00A0E3824D96E000E392087
:1074C000DA6EDF50CA6FFA0E6F008CFF38F0FB0ED9
:1074D0006F008CFF39F00B0E3824D96E000E392066
:1074E000DA6EDF50CB6FFA0E6F008CFF38F0FB0EB8
:1074F0006F008CFF39F00C0E3824D96E000E392045
:10750000DA6EDF50CC6FFA0E6F008CFF38F0FB0E96
:107510006F008CFF39F00D0E3824D96E000E392023
:10752000DA6EDF50CD6FC0875EEF38F0FA0EE126DD
:10753000FF0EE2221200080EE126000EE222600099
:10754000ACF03EF03F6A406A416A426A436A446A6C
:10755000456AF80E6000FBF0E3FFF90E6000FFF0F3
:10756000E3FFFA0E600003F1E3FFFB0E600007F19A
:10757000E3FFFC0E60000BF1E3FFFD0E60000FF176
:10758000E3FFFE0E600013F1E3FFFF0E600017F152
:10759000E3FFF80E6F008CFF3EF0F90E6F008CFFDA
:1075A0003FF0FA0E6F008CFF40F0FB0E6F008CFF77
:1075B00041F0FC0E6F008CFF42F0FD0E6F008CFF5F
:1075C00043F0FE0E6F008CFF44F0FF0E6F008CFF47
:1075D00045F0040ED8903E363F36403641364236AE
:1075E000433644364536E82EEAEF3AF0F70EE350DC
:1075F0003E10466E3F50476E4050486E4150496EB7
:1076000042504A6E43504B6E44504C6E45504D6E46
:10761000F80E60001BF1E3FFF90E60001FF1E3FFBD
:10762000FA0E600023F1E3FFFB0E600027F1E3FF99
:10763000FC0E60002BF1E3FFFD0E60002FF1E3FF75
:10764000FE0E600033F1E3FFFF0E600037F1E3FF51
:10765000F80E6F008CFF3EF0F90E6F008CFF3FF0CC
:10766000FA0E6F008CFF40F0FB0E6F008CFF41F0B4
:10767000FC0E6F008CFF42F0FD0E6F008CFF43F09C
:10768000FE0E6F008CFF44F0FF0E6F008CFF45F084
:10769000040ED8903E363F364036413642364336A9
:1076A00044364536E82E49EF3BF0F60EE3503E10E7
:1076B000466E3F50476E4050486E4150496E4250B2
:1076C0004A6E43504B6E44504C6E45504D6EF80E12
:1076D00060001BF1E3FFF90E60001FF1E3FFFA0EFB
:1076E000600023F1E3FFFB0E600027F1E3FFFC0ED7
:1076F00060002BF1E3FFFD0E60002FF1E3FFFE0EB3
:10770000600033F1E3FFFF0E600037F1E3FFF20E9C
:107710006F008CFF36F0F30E6F008CFF37F0F40E25
:107720006F008CFF38F0F50E6F008CFF39F036508B
:107730003E6E37503F6E3850406E3950416E426A4F
:10774000436A446A456AF80E6F008CFF46F0F90EF2
:107750006F008CFF47F0FA0E6F008CFF48F0FB0EB5
:107760006F008CFF49F0FC0E6F008CFF4AF0FD0E9D
:107770006F008CFF4BF0FE0E6F008CFF4CF0FF0E85
:107780006F008CFF4DF0200ED890463647364836B5
:1077900049364A364B364C364D36E82EC4EF3BF070
:1077A0003E504610366E3F504710376E40504810DE
:1077B000386E41504910396E42504A103A6E43506B
:1077C0004B103B6E44504C103C6E45504D103D6E7E
:1077D000F80E6000DBF0E3FFF90E6000DFF0E3FF7E
:1077E000FA0E6000E3F0E3FFFB0E6000E7F0E3FF5A
:1077F000FC0E6000EBF0E3FFFD0E6000EFF0E3FF36
:10780000FE0E6000F3F0E3FFFF0E6000F7F0E3FF11
:10781000E150F80FD96EE250DA6EFF0EDA226F00F7
:107820007BFFE6FF6F007BFFE6FF6F007BFFE6FF5D
:107830006F007BFFE6FF6F007BFFE6FF6F007BFFC3
:10784000E6FF6F007BFFE6FF6F007BFFE6FF000EA9
:10785000E66E000EE66E0D0EE66E9E0EE66E350EC0
:10786000E66E2A0EE66E000EE66EB5EC49F0F20EFC
:10787000E126FF0EE2221200E652000EE66E51EC07
:1078800060F0FF0E6000BBF0E3FFFF0E6F008CFFA7
:107890002EF0420E2E18D8B450EF3CF052EF3CF0D0
:1078A00038EF3DF0016AFA0E026E070E036EB20E5B
:1078B000046E010E056E000E066E100E076E270E8A
:1078C000086E000E096E000E0A6EF00E0B6E730E3F
:1078D0000C6E550E0D6E000E0E6E320E0F6E190EE2
:1078E000106E116A050E126E010E136E190E146ED3
:1078F000640E156E140E166E0A0E176EFA0E186EC2
:10790000640E196E320E1A6E320E1B6E320E1C6E23
:10791000320E1D6E0A0E1E6E0A0E1F6E0150E66EAE
:10792000010EE66E8FEC5FF00250E66E020EE66E20
:107930008FEC5FF060000FF0E6FF600013F0E6FFF1
:10794000600017F0E6FF60001BF0E6FF030EE66E36
:107950008DEC53F060001FF0E6FF600023F0E6FFBF
:10796000600027F0E6FF60002BF0E6FF070EE66EF2
:107970008DEC53F060002FF0E6FF600033F0E6FF7F
:10798000600037F0E6FF60003BF0E6FF0B0EE66EAE
:107990008DEC53F00F50E66E0F0EE66E8FEC5FF03D
:1079A0001050E66E100EE66E8FEC5FF01150E66E32
:1079B000110EE66E8FEC5FF01250E66E120EE66E60
:1079C0008FEC5FF01350E66E130EE66E8FEC5FF0F7
:1079D0001450E66E140EE66E8FEC5FF01550E66EF6
:1079E000150EE66E8FEC5FF01650E66E160EE66E24
:1079F0008FEC5FF01750E66E170EE66E8FEC5FF0BF
:107A00001850E66E180EE66E8FEC5FF01950E66EB9
:107A1000190EE66E8FEC5FF01A50E66E1A0EE66EE7
:107A20008FEC5FF01B50E66E1B0EE66E8FEC5FF086
:107A30001C50E66E1C0EE66E8FEC5FF01D50E66E7D
:107A40001D0EE66E8FEC5FF01F50E66E1F0EE66EA9
:107A50008FEC5FF01E50E66E1E0EE66E8FEC5FF050
:107A6000420EE66E000EE66E8FEC5FF0DAEF3DF050
:107A7000010EE66E51EC60F02E50016E020EE66EC5
:107A800051EC60F02E50026E030EE66EEFEC53F0F8
:107A90006000B8F003F06000BCF004F06000C0F0DB
:107AA00005F06000C4F006F0070EE66EEFEC53F050
:107AB0006000B8F007F06000BCF008F06000C0F0B3
:107AC00009F06000C4F00AF00B0EE66EEFEC53F024
:107AD0006000B8F00BF06000BCF00CF06000C0F08B
:107AE0000DF06000C4F00EF00F0EE66E51EC60F089
:107AF0002E500F6E100EE66E51EC60F02E50106E90
:107B0000110EE66E51EC60F02E50116E120EE66E04
:107B100051EC60F02E50126E130EE66E51EC60F0D8
:107B20002E50136E140EE66E51EC60F02E50146E53
:107B3000150EE66E51EC60F02E50156E160EE66EC8
:107B400051EC60F02E50166E170EE66E51EC60F0A0
:107B50002E50176E180EE66E51EC60F02E50186E17
:107B6000190EE66E51EC60F02E50196E1A0EE66E8C
:107B700051EC60F02E501A6E1B0EE66E51EC60F068
:107B80002E501B6E1C0EE66E51EC60F02E501C6EDB
:107B90001D0EE66E51EC60F02E501D6E1F0EE66E4F
:107BA00051EC60F02E501F6E1E0EE66E51EC60F030
:107BB0002E501E6EE5521200170EE126000EE22234
:107BC000E90EE1242E6EFF0EE2202F6E6000BBF066
:107BD000E6FF6000BFF0E6FFC5EC11F0EA0EE1241D
:107BE000D96EFF0EE220DA6E6F0078FF36F06F007C
:107BF00078FF37F06F0078FF38F06F0078FF39F0CA
:107C000036503E6E37503F6E3850406E3950416EA0
:107C1000426A436A446A456AF80E6000FBF0E3FF7B
:107C2000F90E6000FFF0E3FFFA0E600003F1E3FFDE
:107C3000FB0E600007F1E3FFFC0E60000BF1E3FFB9
:107C4000FD0E60000FF1E3FFFE0E600013F1E3FF95
:107C5000FF0E600017F1E3FFE150F80FD96EE2501C
:107C6000DA6EFF0EDA220C0ED890DE36DE36DE3605
:107C7000DE36DE36DE36DE36DD36DD52DD52DD5214
:107C8000DD52DD52DD52E82E34EF3EF0E150F80FC8
:107C9000D96EE250DA6EFF0EDA22F20EE124E96EBE
:107CA000FF0EE220EA6EEF50DE12000EDE12DE1250
:107CB000DE12DE12DE12DE12DE12E150F80FD96E95
:107CC000E250DA6EFF0EDA22080ED890DE36DE368B
:107CD000DE36DE36DE36DE36DE36DD36DD52DD52CF
:107CE000DD52DD52DD52DD52E82E65EF3EF0E1500F
:107CF000F80FD96EE250DA6EFF0EDA22F10EE124AF
:107D0000E96EFF0EE220EA6EEF50DE12000EDE1288
:107D1000DE12DE12DE12DE12DE12DE12E150F80F8B
:107D2000D96EE250DA6EFF0EDA22080ED890DE36F7
:107D3000DE36DE36DE36DE36DE36DE36DD36DD5289
:107D4000DD52DD52DD52DD52DD52E82E96EF3EF07F
:107D5000E150F80FD96EE250DA6EFF0EDA22F00E23
:107D6000E124E96EFF0EE220EA6EEF50DE12000E13
:107D7000DE12DE12DE12DE12DE12DE12DE12E15042
:107D8000F80FD96EE250DA6EFF0EDA22080ED890A4
:107D9000DE36DE36DE36DE36DE36DE36DE36DD3644
:107DA000DD52DD52DD52DD52DD52DD52E82EC7EFED
:107DB0003EF0E150F80FD96EE250DA6EFF0EDA2293
:107DC000EF0EE124E96EFF0EE220EA6EEF50DE12C4
:107DD000000EDE12DE12DE12DE12DE12DE12DE1205
:107DE000F70EE124D96EFF0EE220DA6EDF50D8B430
:107DF000FCEF3EF0FEEF3EF02FEF3FF0E150F80FCA
:107E0000D96EE250DA6EFF0EDA226F007BFFE6FFDA
:107E10006F007BFFE6FF6F007BFFE6FF6F007BFFDD
:107E2000E6FF6F007BFFE6FF6F007BFFE6FF6F0062
:107E30007BFFE6FF6F007BFFE6FF000EE66E000EA5
:107E4000E66E0C0EE66E9E0EE66E350EE66E2A0EA1
:107E5000E66E000EE66EB5EC49F05EEF3FF0E150E5
:107E6000F80FD96EE250DA6EFF0EDA226F007BFF58
:107E7000E6FF6F007BFFE6FF6F007BFFE6FF6F0012
:107E80007BFFE6FF6F007BFFE6FF6F007BFFE6FFF7
:107E90006F007BFFE6FF6F007BFFE6FF000EE66EE4
:107EA000000EE66E0B0EE66E9E0EE66E350EE66E6C
:107EB0002A0EE66E000EE66EB5EC49F0E90EE126FC
:107EC000FF0EE2221200FE0E6F008FFFD9FFFF0EA1
:107ED0006F008FFFDAFF140EDF6EFE0E6F008CFF57
:107EE00038F0FF0E6F008CFF39F01A0E3824D96E6F
:107EF000000E3920DA6EDF6AFE0E6F008CFF38F05C
:107F0000FF0E6F008CFF39F01B0E3824D96E000E67
:107F10003920DA6EDF6AFE0E6F008CFF38F0FF0E3C
:107F20006F008CFF39F01C0E3824D96E000E3920FA
:107F3000DA6EDF6AFE0E6F008CFF38F0FF0E6F0006
:107F40008CFF39F01D0E3824D96E000E3920DA6E00
:107F5000010EDF6EFE0E6F008CFF38F0FF0E6F001B
:107F60008CFF39F01E0E3824D96E000E3920DA6EDF
:107F70000A0EDF6EFE0E6F008CFF38F0FF0E6F00F2
:107F80008CFF39F01F0E3824D96E000E3920DA6EBE
:107F9000DE6ADD6AFE0E6F008CFF38F0FF0E6F00A8
:107FA0008CFF39F0230E3824D96E000E3920DA6E9A
:107FB000DE6ADD6AFE0E6F008CFF38F0FF0E6F0088
:107FC0008CFF39F0270E3824D96E000E3920DA6E76
:107FD000DE6ADD6AFE0E6F008CFF38F0FF0E6F0068
:107FE0008CFF39F02B0E3824D96E000E3920DA6E52
:107FF000DE6ADD6AFE0E6F008CFF38F0FF0E6F0048
:108000008CFF39F02F0E3824D96E000E3920DA6E2D
:10801000DE6ADD6AFE0E6F008CFF38F0FF0E6F0027
:108020008CFF39F0330E3824D96E000E3920DA6E09
:10803000DE6ADD6AFD0EE350E66EFD0EE350010FD1
:10804000386EFE0E6F008CFF39F0000E3922600092
:10805000E3F0E6FF6000E7F0E6FF38EC5FF0FE0ECD
:10806000E350010F386EFF0E6F008CFF39F0000EE9
:1080700039226000E3F0E6FF6000E7F0E6FFB4ECD1
:108080005FF0FE0EE350020F386EFF0E6F008CFFA4
:1080900039F0000E39226000E3F0E6FF6000E7F0FF
:1080A000E6FF75EC4CF0320EE66E000EE66EFC0E4E
:1080B000E350020F386EFD0E6F008CFF39F0000E9A
:1080C00039226000E3F0E6FF6000E7F0E6FFE4EC51
:1080D0005DF0320EE66E000EE66EFC0EE350020F0F
:1080E000386EFD0E6F008CFF39F0000E39226000F3
:1080F000E3F0E6FF6000E7F0E6FF04EC5EF0FE0E62
:10810000E350010F386EFF0E6F008CFF39F0000E48
:1081100039226000E3F0E6FF6000E7F0E6FF500E72
:10812000E66EA00EE66EFA0EE350020F386EFB0EFE
:108130006F008CFF39F0000E39226000E3F0E6FF9B
:108140006000E7F0E6FFD4EC56F0FE0EE350010FBE
:10815000386EFF0E6F008CFF39F0000E3922600080
:10816000E3F0E6FF6000E7F0E6FF380EE66EA10EF2
:10817000E66EFA0EE350020F386EFB0E6F008CFFB6
:1081800039F0000E39226000E3F0E6FF6000E7F00E
:10819000E6FF0FEC57F0E552E552E5521200E652C9
:1081A000FA0E6F008CFF2EF0020E2E18D8A4DBEF13
:1081B00040F0DDEF40F0B6EF41F0F60E6F008FFFBC
:1081C000D9FFF70E6F008FFFDAFFFB0E6F008FFFF6
:1081D000DFFFFC0EE124D96EFF0EE220DA6E6F00A5
:1081E00078FF37F06F0078FF38F06F0078FF39F0D4
:1081F0003750326E3850336E3950346E356AFB0E5C
:108200006000CBF0E3FFFC0E6000CFF0E3FFFD0E5B
:108210006000D3F0E3FFFE0E6000D7F0E3FFF80E3E
:108220006F008FFFD9FFF90E6F008FFFDAFFFB0E93
:108230006F008FFFDFFFFC0EE124D96EFF0EE220FE
:10824000DA6E6F0078FF37F06F0078FF38F06F005C
:1082500078FF39F03750326E3850336E3950346E03
:10826000356AFB0E6000CBF0E3FFFC0E6000CFF040
:10827000E3FFFD0E6000D3F0E3FFFE0E6000D7F0D9
:10828000E3FFFB0E6F008CFF39F0030E3916FF0E73
:108290006000E7F0E3FFE150FB0FD96EE250DA6EC9
:1082A000FF0EDA22030ED890DE36DE36DE36DD36FD
:1082B000DD52DD52E82E53EF41F0FB0E6F008CFFD4
:1082C00039F0E00E3916E150FF0FD96EE250DA6E48
:1082D000FF0EDA223950DF26FF0E6F008CFF2EF0E2
:1082E000080E2E26FF0E6000BBF0E3FFF20E6F00BB
:1082F0008FFFD9FFF30E6F008FFFDAFFFF0EE35001
:10830000EB0BDF6EFC0EE124D96EFF0EE220DA6E7D
:108310006F0078FF37F06F0078FF38F06F0078FF5C
:1083200039F03750326E3850336E3950346E356A0A
:10833000FB0E6000CBF0E3FFFC0E6000CFF0E3FF2C
:10834000FD0E6000D3F0E3FFFE0E6000D7F0E3FF08
:10835000F40E6F008FFFD9FFF50E6F008FFFDAFF6D
:10836000FB0E6F008FFFDFFFE8EF41F0F80E6F00AC
:108370008FFFD9FFF90E6F008FFFDAFFDF6AF60E6D
:108380006F008FFFD9FFF70E6F008FFFDAFFDF6AF4
:10839000E150FB0FD96EE250DA6EFF0EDA22050EC5
:1083A000D890DE36DE36DE36DD36DD52DD52E82EA2
:1083B000D0EF41F0F20E6F008FFFD9FFF30E6F0088
:1083C0008FFFDAFFFB0E6F008FFFDFFF82EF41F0C0
:1083D000F20EE126FF0EE2221200050EE126000E4B
:1083E000E222FA0E6F008CFF39F02850395C396EAA
:1083F000FF0E6000E7F0E3FFFF0E6F008CFF39F027
:108400001E50D880D88439AE395CD8A0D884D8B46E
:108410000CEF42F00EEF42F02DEF42F01E506000E4
:10842000A0F038F0396A38BE39063826000E3922F5
:10843000FB0E6000E3F0E3FFFC0E6000E7F0E3FFFB
:108440002E6AE3BE2E68FD0E6000BBF0E3FFFE0E59
:108450006000BBF0E3FF80EF42F01E50386E396AD7
:10846000381E391E384A392AFF0E6F008CFF37F04C
:10847000800E37BE7F0E2E6E3850375C3950800A22
:108480002E58D8B046EF42F048EF42F067EF42F086
:108490001E506000A0F038F0396A38BE3906385EE8
:1084A000000E395AFB0E6000E3F0E3FFFC0E6000A3
:1084B000E7F0E3FF2E6AE3BE2E68FD0E6000BBF01E
:1084C000E3FFFE0E6000BBF0E3FF80EF42F0FA0E28
:1084D000E350366E000E36BEFF0E376E386E396EC4
:1084E000FB0E6000DBF0E3FFFC0E6000DFF0E3FF5B
:1084F000FD0E6000E3F0E3FFFE0E6000E7F0E3FF37
:10850000FB0E6F008CFF28F060002FF0E6FF60008C
:1085100033F0E6FF600037F0E6FF60003BF0E6FF77
:10852000F70E6F008FFFE6FF6F008FFFE6FF6F0013
:108530008FFFE6FF6F008FFFE6FF3FEC4FF0FB0E73
:108540006000BBF0E3FFFC0E6000BFF0E3FFFD0E38
:108550006000C3F0E3FFFE0E6000C7F0E3FFE80E2B
:10856000E66E030EE66E000EE66E000EE66EF70E89
:108570006F008FFFE6FF6F008FFFE6FF6F008FFF3A
:10858000E6FF6F008FFFE6FFF4EC43F0FB0E6000A8
:10859000BBF0E3FFFC0E6000BFF0E3FFFD0E6000E8
:1085A000C3F0E3FFFE0E6000C7F0E3FFE150FB0FF6
:1085B000D96EE250DA6EFF0EDA2200016851DE2633
:1085C0006951DE226A51DE226B51DE22E150FB0F3F
:1085D000D96EE250DA6EFF0EDA226F0078FF6CF08F
:1085E0006F0078FF6DF06F0078FF6EF06F0078FF1E
:1085F0006FF0FA0EE126FF0EE2221200050EE126D0
:10860000000EE222FA0E6F008CFF39F02950395C1F
:10861000396EFF0E6000E7F0E3FFFF0E6F008CFF86
:1086200039F01F50D880D88439AE395CD8A0D884AE
:10863000D8B41DEF43F01FEF43F03EEF43F01F505F
:108640006000A4F038F0396A38BE39063826000ECA
:108650003922FB0E6000E3F0E3FFFC0E6000E7F060
:10866000E3FF2E6AE3BE2E68FD0E6000BBF0E3FF61
:10867000FE0E6000BBF0E3FF91EF43F01F50386E39
:10868000396A381E391E384A392AFF0E6F008CFFAE
:1086900037F0800E37BE7F0E2E6E3850375C395063
:1086A000800A2E58D8B057EF43F059EF43F078EFD7
:1086B00043F01F506000A4F038F0396A38BE390624
:1086C000385E000E395AFB0E6000E3F0E3FFFC0E4B
:1086D0006000E7F0E3FF2E6AE3BE2E68FD0E600047
:1086E000BBF0E3FFFE0E6000BBF0E3FF91EF43F051
:1086F000FA0EE350366E000E36BEFF0E376E386E41
:10870000396EFB0E6000DBF0E3FFFC0E6000DFF073
:10871000E3FFFD0E6000E3F0E3FFFE0E6000E7F014
:10872000E3FFFB0E6F008CFF29F060001FF0E6FFF7
:10873000600023F0E6FF600027F0E6FF60002BF00A
:10874000E6FFF70E6F008FFFE6FF6F008FFFE6FF7B
:108750006F008FFFE6FF6F008FFFE6FF3FEC4FF0EB
:10876000FB0E6000BBF0E3FFFC0E6000BFF0E3FF18
:10877000FD0E6000C3F0E3FFFE0E6000C7F0E3FFF4
:10878000E80EE66E030EE66E000EE66E000EE66E76
:10879000F70E6F008FFFE6FF6F008FFFE6FF6F00A1
:1087A0008FFFE6FF6F008FFFE6FFF4EC43F0FB0E58
:1087B0006000BBF0E3FFFC0E6000BFF0E3FFFD0EC6
:1087C0006000C3F0E3FFFE0E6000C7F0E3FFFB0EA6
:1087D0006F008CFF66F0FC0E6F008CFF67F0FA0EE6
:1087E000E126FF0EE2221200060EE126000EE22232
:1087F000FE0EE36AF50EE3BE02EF44F000EF44F034
:1088000016EF44F0F20EE36CF30EE31EF40EE31EDB
:10881000F50EE31E08E3F30EE32A05E3F40EE32A64
:1088200002E3F50EE32AFE0EE36AE32AF90EE3BE45
:108830001EEF44F01CEF44F031EF44F0F60EE36C11
:10884000F70EE31EF80EE31EF90EE31E08E3F70E23
:10885000E32A05E3F80EE32A02E3F90EE32AFE0E0B
:10886000E370FA0EE36AFB0EE36AFC0EE36AFD0EA8
:10887000E36AF20EE3500FE1F30EE3500CE1F40E65
:10888000E35009E1F50EE350D8B449EF44F04BEF63
:1088900044F0B4EF44F0FF0EE36AE32A5BEF44F0E8
:1088A000D890F20EE336F30EE336F40EE336F50E0F
:1088B000E336FF0EE32AF50EE3AE61EF44F063EF1B
:1088C00044F050EF44F0D890FA0EE336FB0EE33656
:1088D000FC0EE336FD0EE336E150F60FD96EE250A2
:1088E000DA6EFF0EDA22F20EE350DE5CF30EE35096
:1088F000DE58F40EE350DE58F50EE350DE58D8A0F3
:1089000084EF44F086EF44F09BEF44F0E150F60F23
:10891000D96EE250DA6EFF0EDA22F20EE350DE5E1E
:10892000F30EE350DE5AF40EE350DE5AF50EE35038
:10893000DE5AFA0EE380D890F50EE332F40EE332FD
:10894000F30EE332F20EE332FF0EE3502E6E010E11
:108950002E5EFF0E6000BBF0E3FFD8A4B2EF44F040
:10896000B4EF44F063EF44F0FE0EE350D8B4BBEF35
:1089700044F0BDEF44F0CEEF44F0FA0EE36CFB0E92
:10898000E31EFC0EE31EFD0EE31E08E3FB0EE32ACE
:1089900005E3FC0EE32A02E3FD0EE32AFA0E6F0064
:1089A0008CFF2EF0FB0E6F008CFF2FF0FC0E6F0083
:1089B0008CFF30F0FD0E6F008CFF31F0F20EE126DF
:1089C000FF0EE22212000A0EE126000EE222F60E4F
:1089D000E36AF70EE36AF80EE36AF90EE36AF20E51
:1089E0006F008CFF39F0030E3916FF0E6000E7F0C0
:1089F000E3FFF20E6F008CFF39F0050E2E6ED8905B
:108A000039322E2EFFEF44F0FE0E6000E7F0E3FF58
:108A1000F30EE350386E396AD89038363936D8902C
:108A200038363936D89038363936F60E6000E3F0ED
:108A3000E3FFF70E6000E7F0E3FF2E6AE3BE2E6867
:108A4000F80E6000BBF0E3FFF90E6000BBF0E3FF3F
:108A5000E150F60FD96EE250DA6EFF0EDA22FE0E0A
:108A6000E350DE26000EDE22DE22DE22E150F60F8B
:108A7000D96EE250DA6EFF0EDA22020ED890DE36A0
:108A8000DE36DE36DD36DD52DD52E82E3EEF45F0D5
:108A9000E150F60FD96EE250DA6EFF0EDA22FF0EC9
:108AA000E350DE26000EDE22DE22DE22E150F60F4B
:108AB000D96EE250DA6EFF0EDA22080ED890DE365A
:108AC000DE36DE36DD36DD52DD52E82E5EEF45F075
:108AD000E150F60FD96EE250DA6EFF0EDA22F50E93
:108AE000E350DE26000EDE22DE22DE22E150F60F0B
:108AF000D96EE250DA6EFF0EDA22080ED890DE361A
:108B0000DE36DE36DD36DD52DD52E82E7EEF45F014
:108B1000E150F60FD96EE250DA6EFF0EDA22F40E53
:108B2000E350DE26000EDE22DE22DE22F60E6F008D
:108B30008CFF36F0F70E6F008CFF37F0F80E6F00E9
:108B40008CFF38F0F90E6F008CFF39F0FA0E6000E0
:108B5000DBF0E3FFFB0E6000DFF0E3FFFC0E6000E4
:108B6000E3F0E3FFFD0E6000E7F0E3FFFA0E6F00B5
:108B70008CFF2EF0FB0E6F008CFF2FF0FC0E6F00B1
:108B80008CFF30F0FD0E6F008CFF31F0F20EE1260D
:108B9000FF0EE2221200800E8F6E8E50E00B800AD4
:108BA000D8A4D5EF45F0D7EF45F0CDEF45F0900EC6
:108BB000916E3701006B3D6BB90EE66E370EE66EB7
:108BC000B80EE66E370EE66EBB0EE66E370EE66E3C
:108BD000BA0EE66E370EE66E010EE66E700EE66EAB
:108BE000000EE66E000EE66E000EE66ECFEC40F074
:108BF000BD0EE66E370EE66EBC0EE66E370EE66E06
:108C0000BF0EE66E370EE66EBE0EE66E370EE66EF1
:108C1000010EE66E700EE66E000EE66E000EE66E5B
:108C2000000EE66ECFEC40F0A10EE66E370EE66E5B
:108C3000A00EE66E370EE66EA30EE66E370EE66EFB
:108C4000A20EE66E370EE66E010EE66E000EE66EC2
:108C5000000EE66E000EE66E000EE66ECFEC40F003
:108C6000A50EE66E370EE66EA40EE66E370EE66EC5
:108C7000A70EE66E370EE66EA60EE66E370EE66EB1
:108C8000010EE66E100EE66E000EE66E000EE66E4B
:108C9000000EE66ECFEC40F0A90EE66E370EE66EE3
:108CA000A80EE66E370EE66EAB0EE66E370EE66E7B
:108CB000AA0EE66E370EE66E010EE66E700EE66EDA
:108CC000000EE66E000EE66E000EE66ECFEC40F093
:108CD000070E3701066F100E396F0F0E036F980ED7
:108CE000046F810E056F1A0EE66EC10EE66E0DEC76
:108CF00060F03901A5939583240EE66EC10EE66EF1
:108D0000F7EC5FF0260EE66EC10EE66E02EC60F048
:108D10001E0EE66EC10EE66ED6EC5FF0220EE66E1B
:108D2000C10EE66EECEC5FF01C0EE66EC10EE66E58
:108D3000CBEC5FF0200EE66EC10EE66EE1EC5FF06C
:108D40003901A59B958B8F6A6F0038FE39F0E00ED4
:108D50003916D8A4AEEF46F0B0EF46F0A4EF46F0D7
:108D60001200FE0E6F008FFFD9FFFF0E6F008FFF06
:108D7000DAFF6E0EDF6E030EE66EFD0EE350010F9E
:108D8000386EFE0E6F008CFF39F0000E3922600045
:108D9000E3F0E6FF6000E7F0E6FF63EC3FF0010E72
:108DA000E66E100EE66E600EE66E9B0EE66EFA0E36
:108DB000E350010F386EFB0E6F008CFF39F0000E90
:108DC00039226000E3F0E6FF6000E7F0E6FF4AECDE
:108DD00057F0FE0E6F008FFFE6FF6F008FFFE6FF7C
:108DE000AE0EE66EB20EE66EFA0EE350010F386E6E
:108DF000FB0E6F008CFF39F0000E39226000E3F0AB
:108E0000E6FF6000E7F0E6FF5EEC56F0FE0E6F0056
:108E10008FFFE6FF6F008FFFE6FF3A0EE66EB20EA1
:108E2000E66EFA0EE350010F386EFB0E6F008CFFFA
:108E300039F0000E39226000E3F0E6FF6000E7F051
:108E4000E6FF85EC57F0FE0E6F008FFFE6FF6F0028
:108E50008FFFE6FFC80EE66EBA0EE66EFA0EE3501E
:108E6000010F386EFB0E6F008CFF39F0000E3922B7
:108E70006000E3F0E6FF6000E7F0E6FF99EC56F0F3
:108E8000FE0E6F008CFF38F0FF0E6F008CFF39F084
:108E9000380E3824D96E000E3920DA6EDE6ADD6AAB
:108EA000FE0E6F008CFF38F0FF0E6F008CFF39F064
:108EB0003C0E3824D96E000E3920DA6EDE6ADD6A87
:108EC000FE0E6F008CFF38F0FF0E6F008CFF39F044
:108ED000400E3824D96E000E3920DA6EDE6ADD6A63
:108EE000980E0001686F8B0E696F080E6A6F000E96
:108EF0006B6FE552E5521200FE0E6F008FFFD9FF37
:108F0000FF0E6F008FFFDAFF640EDF6E020EE66E5B
:108F1000FD0EE350010F386EFE0E6F008CFF39F02E
:108F2000000E39226000E3F0E6FF6000E7F0E6FFA4
:108F300063EC3FF0040EE66E100EE66E5E0EE66E1B
:108F4000AA0EE66EFA0EE350010F386EFB0E6F00AC
:108F50008CFF39F0000E39226000E3F0E6FF60007C
:108F6000E7F0E6FF4AEC57F0FE0E6F008FFFE6FFDA
:108F70006F008FFFE6FF0A0EE66EB40EE66EFA0E85
:108F8000E350010F386EFB0E6F008CFF39F0000EBE
:108F900039226000E3F0E6FF6000E7F0E6FF5EECF8
:108FA00056F0FE0E6F008FFFE6FF6F008FFFE6FFAB
:108FB000960EE66EB30EE66EFA0EE350010F386EB3
:108FC000FB0E6F008CFF39F0000E39226000E3F0D9
:108FD000E6FF6000E7F0E6FF85EC57F0FE0E6F005D
:108FE0008FFFE6FF6F008FFFE6FF220EE66EB30EE7
:108FF000E66EFA0EE350010F386EFB0E6F008CFF29
:1090000039F0000E39226000E3F0E6FF6000E7F07F
:10901000E6FF99EC56F0FE0E6F008CFF38F0FF0E65
:109020006F008CFF39F0380E3824D96E000E3920CD
:10903000DA6EDE6ADD6AFE0E6F008CFF38F0FF0E1E
:109040006F008CFF39F03C0E3824D96E000E3920A9
:10905000DA6EDE6ADD6AFE0E6F008CFF38F0FF0EFE
:109060006F008CFF39F0400E3824D96E000E392085
:10907000DA6EDE6ADD6AE552E5521200E652E65229
:10908000FE0EE36AFF0EE36AFE0E6F008CFF38F0FF
:10909000FF0E6F008CFF39F00F0E38026F00CCFF0F
:1090A00036F06F00D0FF37F03902F3503726A10EAB
:1090B0003624386E030E3720396E6000E3F0E6FF89
:1090C0006000E7F0E6FFE1EC54F0FE0EE350010F24
:1090D0002E6EFE0E6000BBF0E3FF2E6AFF0EE35023
:1090E0002E202E6EFF0E6000BBF0E3FFFF0EE3BEEE
:1090F00088EF48F0FF0EE3500DE1FE0E6F008CFF8D
:109100002EF0140E2E5ED8A088EF48F08AEF48F0BB
:1091100044EF48F0FE0EE36AFF0EE36AFE0E6F00B6
:109120008CFF38F0FF0E6F008CFF39F0110E380203
:109130006F00CCFF36F06F00D0FF37F03902F350EC
:109140003726F80E3624D96E010E3720DA6EDE6A25
:10915000DD6AFE0E6F008CFF38F0FF0E6F008CFF93
:1091600039F0110E38026F00CCFF36F06F00D0FFDF
:1091700037F03902F3503726FA0E3624386E010ED6
:109180003720396E6000E3F0E6FF6000E7F0E6FFAD
:10919000E1EC54F0FE0EE350010F2E6EFE0E600067
:1091A000BBF0E3FF2E6AFF0EE3502E202E6EFF0E63
:1091B0006000BBF0E3FFFF0EE3BEEDEF48F0FF0EF3
:1091C000E3500DE1FE0E6F008CFF2EF0190E2E5EA7
:1091D000D8A0EDEF48F0EFEF48F08EEF48F0000E2A
:1091E0006F00A0FFCDF4000E6F00A0FFCEF4E5529B
:1091F000E5521200E652E652E652EE0EE1242E6EE1
:10920000FF0EE2202F6E6000BBF0E6FF6000BFF0B3
:10921000E6FFD9EC5EF0FD0E6000BBF0E3FFFE0E52
:109220006000BFF0E3FFFD0E6F008CFF2EF0FE0E1E
:10923000E3502E10D8B41FEF49F021EF49F059EF59
:1092400049F0000EE66E000EE66EEC0EE1242E6E86
:10925000FF0EE2202F6E6000BBF0E6FF6000BFF063
:10926000E6FF84EC5DF0ED0EE350E66EED0EE124DA
:10927000D96EFF0EE220DA6E0F0E6F007BFFE6FF65
:10928000E82C3DEF49F0ED0E6F008FFFE6FF6F0019
:109290008FFFE6FF2BEC53F0EB0E6F008FFFD9FF33
:1092A000EC0E6F008FFFDAFF6000BBF0DFFFAEEF68
:1092B00049F0ED0EE350E66EA8EC5FF0140EE66E9A
:1092C000000EE66E21EECDF0DF50386E396A010EE9
:1092D0003826000E39226000E3F0E6FF6000E7F078
:1092E000E6FF1EEC4BF0FF0E6000BBF0E3FF21EE4B
:1092F000CEF0FF0EE350DE18D8A481EF49F083EFE3
:1093000049F08CEF49F0ED0EE350E66E9CEC5FF017
:10931000000E2E6EB0EF49F0EE0EE124D96EFF0E76
:10932000E220DA6E01EECDF0EF500F0DA10EF32426
:10933000E96E030EF420EA6E0E0E6F006FFFEBFF76
:10934000E806FBE2FF0E6F008CFF39F06000E4F0EE
:10935000CDF4ED0EE350E66E9CEC5FF0010E2E6E48
:10936000EB0EE126FF0EE2221200100EE126000EA7
:10937000E222190E396EFF0E6000E7F0E3FFF00EF7
:10938000E1242E6EFF0EE2202F6E6000BBF0E6FFA0
:109390006000BFF0E6FFE1EC54F0EE0E6F008FFFCF
:1093A000E6FF6F008FFFE6FFEE0EE1242E6EFF0E4C
:1093B000E2202F6E6000BBF0E6FF6000BFF0E6FF2A
:1093C000A4EC5DF0EC0E6F008FFFE6FF6F008FFFE7
:1093D000E6FFEE0EE1242E6EFF0EE2202F6E6000FF
:1093E000BBF0E6FF6000BFF0E6FFC4EC5DF0EB0E03
:1093F000E350E66EEF0EE1242E6EFF0EE2202F6E9C
:109400006000BBF0E6FF6000BFF0E6FF28EC5FF015
:10941000E90E6F008FFFE6FF6F008FFFE6FFEE0E95
:10942000E1242E6EFF0EE2202F6E6000BBF0E6FFFF
:109430006000BFF0E6FF84EC5DF0E150E10FD96E13
:10944000E250DA6EFF0EDA226F007BFFE6FF6F005C
:109450007BFFE6FF6F007BFFE6FF6F007BFFE6FF11
:109460006F007BFFE6FF6F007BFFE6FF6F007BFF77
:10947000E6FF6F007BFFE6FFE80EE1242E6EFF0E95
:10948000E2202F6E6000BBF0E6FF6000BFF0E6FF59
:1094900040EC5EF0FF0EE1242E6EFF0EE2202F6EF8
:1094A0006000BBF0E6FF6000BFF0E6FF000EE66E76
:1094B000ED0EE124D96EFF0EE220DA6E0F0E6F0082
:1094C0007BFFE6FFE82C5FEF4AF0FAEC48F0E10E94
:1094D000E126FF0EE2221200E652E652E652E65282
:1094E000FB0EE3BE76EF4AF078EF4AF09AEF4AF0CF
:1094F000F80E6F008CFF36F0F90E6F008CFF37F01E
:10950000FA0E6F008CFF38F0FB0E6F008CFF39F005
:10951000FC0E6000DBF0E3FFFD0E6000DFF0E3FF18
:10952000FE0E6000E3F0E3FFFF0E6000E7F0E3FFF4
:10953000C3EF4AF0F80E6F008CFF36F0F90E6F00A3
:109540008CFF37F0FA0E6F008CFF38F0FB0E6F00C7
:109550008CFF39F0361E371E381E391E362A000E93
:10956000372238223922FC0E6000DBF0E3FFFD0ECB
:109570006000DFF0E3FFFE0E6000E3F0E3FFFF0EAC
:109580006000E7F0E3FFE80EE66E030EE66E000E05
:10959000E66E000EE66EF80E6F008FFFE6FF6F00BE
:1095A0008FFFE6FF6F008FFFE6FF6F008FFFE6FF84
:1095B0003FEC4FF0FC0E6000BBF0E3FFFD0E6000DF
:1095C000BFF0E3FFFE0E6000C3F0E3FFFF0E60009C
:1095D000C7F0E3FF60000FF0E6FF600013F0E6FF66
:1095E000600017F0E6FF60001BF0E6FFF80E6F006A
:1095F0008FFFE6FF6F008FFFE6FF6F008FFFE6FF34
:109600006F008FFFE6FF14EC4DF0FC0E6000BBF026
:10961000E3FFFD0E6000BFF0E3FFFE0E6000C3F04D
:10962000E3FFFF0E6000C7F0E3FFFC0E6F008CFF4E
:1096300070F0F80EE126FF0EE2221200E652E6522A
:10964000FE0EE36AFD0EE3BE2AEF4BF028EF4BF06F
:1096500033EF4BF0FC0EE36CFD0EE31ED8B0E32AB3
:10966000FE0EE36AE32AFB0EE3BE3BEF4BF039EF5D
:109670004BF041EF4BF0FA0EE36CFB0EE31ED8B05B
:10968000E32AFA0E6F008CFF2EF0FB0EE3502E1033
:10969000D8B44DEF4BF04FEF4BF0B3EF4BF0FF0E64
:1096A000E36AE32A67EF4BF0FA0EE350D890E83410
:1096B0002E6EFA0E6000BBF0E3FFFB0EE350E834C1
:1096C0002E6EFB0E6000BBF0E3FFFF0EE32AFB0EE5
:1096D000E3AE6DEF4BF06FEF4BF054EF4BF0FA0E43
:1096E0006F008CFF38F0FB0E6F008CFF39F0FC0E22
:1096F0006F008CFF36F0FD0E6F008CFF37F0385096
:10970000365C39503758D8A088EF4BF08AEF4BF0D1
:109710009EEF4BF0FC0EE3502E6EFA0EE3502E5EE1
:10972000FC0E6000BBF0E3FFFD0EE3502E6EFB0E5F
:10973000E3502E5AFD0E6000BBF0E3FFD890FB0E05
:10974000E332FA0EE332FF0EE3502E6E010E2E5E70
:10975000FF0E6000BBF0E3FFD8A4B1EF4BF0B3EF16
:109760004BF06FEF4BF0FE0EE350D8B4BAEF4BF076
:10977000BCEF4BF0C2EF4BF0FC0EE36CFD0EE31EB2
:10978000D8B0E32AFC0E6F008CFF2EF0FD0E6F00A8
:109790008CFF2FF0FA0EE126FF0EE22212006F007E
:1097A000E8FF4EF06F00ECFF4FF06000B8F050F0B3
:1097B0006000BCF051F06000C0F052F06000C4F0F6
:1097C00053F06000D8F054F06000DCF055F0600019
:1097D000E0F056F06000E4F057F06000F8F058F068
:1097E0006000FCF059F0600000F15AF0600004F1F4
:1097F0005BF0600008F15CF060000CF15DF060006F
:1098000010F15EF0600014F15FF012EE68F23901C1
:1098100093AF0DEF4CF00FEF4CF01AEF4CF0A3AFFD
:1098200014EF4CF016EF4CF01AEF4CF0A9EC5EF090
:109830003EEF4CF095AB1FEF4CF021EF4CF02CEFCE
:109840004CF0A5AB26EF4CF028EF4CF02CEF4CF091
:10985000C6EC4EF03EEF4CF095A331EF4CF033EFF9
:109860004CF03EEF4CF0A5A338EF4CF03AEF4CF043
:109870003EEF4CF057EC5FF03EEF4CF060007CF1B7
:1098800045F0600078F144F0600074F143F060004E
:1098900070F142F060006CF141F0600068F140F05E
:1098A000600064F13FF0600060F13EF060005CF148
:1098B00039F0600058F138F0600054F137F0600082
:1098C00050F136F060004CF131F0600048F130F0BA
:1098D000600044F12FF0600040F12EF060003FF195
:1098E000FBFF60003BF1FAFF1100FE0E6F008FFFDF
:1098F000D9FFFF0E6F008FFFDAFFDF6AFE0E6F00E9
:109900008CFF38F0FF0E6F008CFF39F0010E382409
:10991000D96E000E3920DA6EF40EDE6E010EDD6EA9
:10992000FE0E6F008CFF38F0FF0E6F008CFF39F0D9
:10993000030E3824D96E000E3920DA6EF40EDE6E76
:10994000010EDD6EFE0E6F008CFF38F0FF0E6F0013
:109950008CFF39F0050E3824D96E000E3920DA6EEE
:10996000030EDF6EFE0E6F008CFF38F0FF0E6F00EF
:109970008CFF39F0060E3824D96E000E3920DA6ECD
:10998000DF6AFE0E6F008CFF38F0FF0E6F008CFF59
:1099900039F0070E3824D96E000E3920DA6E030E26
:1099A000DF6EFE0E6F008CFF38F0FF0E6F008CFF35
:1099B00039F0080E3824D96E000E3920DA6EDE6ACE
:1099C000DD6AFE0E6F008CFF38F0FF0E6F008CFF1B
:1099D00039F00C0E3824D96E000E3920DA6EDE6AAA
:1099E000DD6AFE0E6F008CFF38F0FF0E6F008CFFFB
:1099F00039F0100E3824D96E000E3920DA6EDE6A86
:109A0000DD6AFE0E6F008CFF38F0FF0E6F008CFFDA
:109A100039F0140E3824D96E000E3920DA6EDE6A61
:109A2000DD6AE552E5521200050EE126000EE22243
:109A3000FB0EE36AFC0EE36AFD0EE36AFE0EE36AC8
:109A4000F30EE3500FE1F40EE3500CE1F50EE3509A
:109A500009E1F60EE350D8B430EF4DF032EF4DF09F
:109A60009BEF4DF0FF0EE36AE32A42EF4DF0D890F2
:109A7000F30EE336F40EE336F50EE336F60EE33678
:109A8000FF0EE32AF60EE3AE48EF4DF04AEF4DF03D
:109A900037EF4DF0D890FB0EE336FC0EE336FD0EAB
:109AA000E336FE0EE336E150F70FD96EE250DA6E80
:109AB000FF0EDA22F30EE350DE5CF40EE350DE58C4
:109AC000F50EE350DE58F60EE350DE58D8A06BEFEB
:109AD0004DF06DEF4DF082EF4DF0E150F70FD96E84
:109AE000E250DA6EFF0EDA22F30EE350DE5EF40E81
:109AF000E350DE5AF50EE350DE5AF60EE350DE5A1E
:109B0000FB0EE380D890F60EE332F50EE332F40E4E
:109B1000E332F30EE332FF0EE3502E6E010E2E5EA3
:109B2000FF0E6000BBF0E3FFD8A499EF4DF09BEF70
:109B30004DF04AEF4DF0FB0E6F008CFF2EF0FC0E47
:109B40006F008CFF2FF0FD0E6F008CFF30F0FE0ECB
:109B50006F008CFF31F0F30EE126FF0EE2221200BF
:109B6000050EE126000EE222F90E6F008FFFF6FFD0
:109B7000FA0E6F008FFFF7FF000EF86E0F0EF764FE
:109B800003D00800F55007D06F00DBFFE9FF6F003E
:109B9000DFFFEAFFEF50396EFF0E6000E7F0E3FFF2
:109BA00008EF4EF0FB0EE36AE32AFC0EE124D96EC7
:109BB000FF0EE220DA6EDF6AFD0EE124D96EFF0EA1
:109BC000E220DA6EDF6A22EF4EF0FB0EE36AFC0E53
:109BD000E124D96EFF0EE220DA6E010EDF6EDCEFBB
:109BE0004DF0FB0EE36AFC0EE124D96EFF0EE2207D
:109BF000DA6EDF6AFD0EE124D96EFF0EE220DA6E26
:109C0000010EDF6E22EF4EF0FB0EE36AD5EF4DF052
:109C1000FF0EE350386E396A3950000AD8B413EF9A
:109C20004EF004EF4EF03850010AD8B4D2EF4DF0A8
:109C3000030AD8B4E5EF4DF0010AD8B4F1EF4DF0C6
:109C400004EF4EF0FE0EE124D96EFF0EE220DA6E34
:109C5000600067F0DFFFFB0E6F008FFFE6FF6F0015
:109C60008FFFE6FF6F008FFFE6FF6F008FFFE6FFBD
:109C7000000EE66E050EE66E9BEC3AF0F90EE1265C
:109C8000FF0EE2221200E652E652FF0EE36AFF0EDA
:109C9000E350110DFA0EF324D96E010EF420DA6EA2
:109CA000DF50D8B456EF4EF058EF4EF0B5EF4EF00F
:109CB000FF0EE350110DF80EF324D96E010EF420BF
:109CC000DA6E0A0EDE5E000EDD5AFF0EE350110D55
:109CD000F80EF324D96E010EF420DA6EDE50DE1099
:109CE000D8A475EF4EF077EF4EF0B5EF4EF0FE0EC4
:109CF000E1242E6EFF0EE2202F6E6000BBF0E6FF27
:109D00006000BFF0E6FF010EE66EFC0EE350110DA1
:109D1000FA0EF324D96E010EF420DA6E0F0E6F00E6
:109D20007BFFE6FFE82C8FEF4EF0FAEC48F02E04B4
:109D3000D8A49DEF4EF09FEF4EF0A8EF4EF0010E2D
:109D4000E66EFE0EE350E66E17EC5CF0B5EF4EF0FB
:109D5000FF0EE350110DF80EF324D96E010EF4201E
:109D6000DA6E010EDE6E000EDD6EFF0EE32AFF0ED0
:109D70006F008CFF2EF0180E2E64C1EF4EF0C3EF73
:109D80004EF047EF4EF0E552E552120090ACCBEFAB
:109D90004EF0CDEF4EF0DAEF4EF002D8D9EF4EF0A4
:109DA0000500FA6E2450FD6E2550FE6EFF6AFA50D3
:109DB0001200909C90AADFEF4EF0E1EF4EF0EDEF35
:109DC0004EF002D8EDEF4EF00500FA6E2250FD6E17
:109DD0002350FE6EFF6AFA50120090A8F2EF4EF088
:109DE000F4EF4EF000EF4FF002D800EF4FF0050017
:109DF000FA6E2050FD6E2150FE6EFF6AFA5012007E
:109E000090A605EF4FF007EF4FF014EF4FF002D898
:109E100014EF4FF00500FA6E00016451FD6E6551BC
:109E2000FE6EFF6AFA50120090A419EF4FF01BEF7C
:109E30004FF028EF4FF002D828EF4FF00500FA6EF0
:109E400000016251FD6E6351FE6EFF6AFA5012000E
:109E500090A22DEF4FF02FEF4FF03CEF4FF002D8D4
:109E60003CEF4FF00500FA6E00016051FD6E61514C
:109E7000FE6EFF6AFA5012003901A59B1200E652ED
:109E8000E652E652E652FC0EE36AFD0EE36AFE0E6F
:109E9000E36AFF0EE36AF80EE3A051EF4FF053EFD1
:109EA0004FF07BEF4FF0FC0EE3502E6EF40EE350BC
:109EB0002E26FC0E6000BBF0E3FFFD0EE3502E6E7D
:109EC000F50EE3502E22FD0E6000BBF0E3FFFE0E08
:109ED000E3502E6EF60EE3502E22FE0E6000BBF015
:109EE000E3FFFF0EE3502E6EF70EE3502E22FF0E1F
:109EF0006000BBF0E3FFD890F40EE336F50EE336D6
:109F0000F60EE336F70EE336D890FB0EE332FA0E88
:109F1000E332F90EE332F80EE332F80EE3500DE1CE
:109F2000F90EE3500AE1FA0EE35007E1FB0EE350AD
:109F3000D8A49DEF4FF09FEF4FF04BEF4FF0FC0E8A
:109F40006F008CFF2EF0FD0E6F008CFF2FF0FE0EC9
:109F50006F008CFF30F0FF0E6F008CFF31F0F40EBD
:109F6000E126FF0EE2221200080EE126000EE22298
:109F7000F60E6F008FFFD9FFF70E6F008FFFDAFF2D
:109F80006F0078FF36F06F0078FF37F06F0078FFD2
:109F900038F06F0078FF39F0FC0E6000DBF0E3FF73
:109FA000FD0E6000DFF0E3FFFE0E6000E3F0E3FF74
:109FB000FF0E6000E7F0E3FFFF0EE124D96EFF0E15
:109FC000E220DA6EDF50396EF80E6000E7F0E3FF52
:109FD000FE0EE124D96EFF0EE220DA6EF90EE124C6
:109FE000E96EFF0EE220EA6E6F007FFFEFFFFD0ECD
:109FF000E124D96EFF0EE220DA6EFA0EE124E96E5A
:10A00000FF0EE220EA6E6F007FFFEFFFFB0EE12400
:10A01000D96EFF0EE220DA6EFC0E6F008FFFDFFFBD
:10A02000F80E6F008FFFE6FF6F008FFFE6FF6F00F7
:10A030008FFFE6FF6F008FFFE6FF010EE66E050E55
:10A04000E66E9BEC3AF0F60EE126FF0EE2221200DD
:10A05000E652E652FC0E6F008CFF38F0FD0E6F00EA
:10A060008CFF39F0FF0E6000E7F0E3FFFE0E6000AA
:10A07000E3F0E3FF54EF50F0BA8097EF50F0BA826C
:10A0800097EF50F0BA8497EF50F0BA8697EF50F000
:10A09000BA8897EF50F0BA8A97EF50F0BA8C97EFE2
:10A0A00050F0BA8E97EF50F0FE0E6F008FFFF6FF64
:10A0B000FF0E6F008FFFF7FF000EF86E0F0EF764B4
:10A0C00003D00800F55007D06F00DBFFE9FF6F00F9
:10A0D000DFFFEAFFEF50386E396A3950000AD8B412
:10A0E00074EF50F097EF50F03850010AD8B43CEFBD
:10A0F00050F0030AD8B43FEF50F0010AD8B442EF51
:10A1000050F0070AD8B445EF50F0010AD8B448EF30
:10A1100050F0030AD8B44BEF50F0010AD8B44EEF18
:10A1200050F00F0AD8B451EF50F097EF50F0E552CD
:10A13000E552E552E5521200E652E652FC0E6F007F
:10A140008CFF38F0FD0E6F008CFF39F0FF0E6000C1
:10A15000E7F0E3FFFE0E6000E3F0E3FFC8EF50F02E
:10A16000BA900BEF51F0BA920BEF51F0BA940BEF9B
:10A1700051F0BA960BEF51F0BA980BEF51F0BA9A32
:10A180000BEF51F0BA9C0BEF51F0BA9E0BEF51F070
:10A19000FE0E6F008FFFF6FFFF0E6F008FFFF7FFC1
:10A1A000000EF86E0F0EF76403D00800F55007D0CC
:10A1B0006F00DBFFE9FF6F00DFFFEAFFEF50386E53
:10A1C000396A3950000AD8B4E8EF50F00BEF51F07B
:10A1D0003850010AD8B4B0EF50F0030AD8B4B3EF46
:10A1E00050F0010AD8B4B6EF50F0070AD8B4B9EF6E
:10A1F00050F0010AD8B4BCEF50F0030AD8B4BFEF56
:10A2000050F0010AD8B4C2EF50F00F0AD8B4C5EF2D
:10A2100050F00BEF51F0E552E552E552E5521200D5
:10A22000080EE126000EE222F70EE350386E396A7E
:10A23000D89038363936D89038363936D8903836BE
:10A240003936F80E6000E3F0E3FFF90E6000E7F046
:10A25000E3FF2E6AE3BE2E68FA0E6000BBF0E3FF58
:10A26000FB0E6000BBF0E3FFE150F80FD96EE25047
:10A27000DA6EFF0EDA22F60E6F008CFF39F0050E53
:10A280002E6ED89039322E2E41EF51F03950DE2605
:10A29000000EDE22DE22DE22F80E6F008CFF36F08A
:10A2A000F90E6F008CFF37F0FA0E6F008CFF38F05C
:10A2B000FB0E6F008CFF39F0FC0E6000DBF0E3FF5B
:10A2C000FD0E6000DFF0E3FFFE0E6000E3F0E3FF51
:10A2D000FF0E6000E7F0E3FFFC0E6F008CFF2EF036
:10A2E000FD0E6F008CFF2FF0FE0E6F008CFF30F024
:10A2F000FF0E6F008CFF31F0F60EE126FF0EE2221A
:10A3000012001D0EE126000EE222F10EE36AF40EA9
:10A31000E124D96EFF0EE220DA6EDE6ADD6AF20E0B
:10A32000E124D96EFF0EE220DA6EDE6ADD6AE20E0B
:10A33000E350E66EA8EC5FF021EECEF001EECDF03A
:10A34000DE50EE18D8A4A7EF51F0A9EF51F0BFEFFF
:10A3500051F0E20EE350E66E9CEC5FF0F10EE1246A
:10A36000D96EFF0EE220DA6E0F0E2E6EE20E6F0037
:10A370007BFFE3FFE8282E2EFAD7ECEF51F021EE19
:10A38000CEF0DF500F0DA10EF324D96E030EF42092
:10A39000DA6E0F0E2E6EF10E6F007BFFE3FFE828E2
:10A3A0002E2EFAD7140EE66E000EE66E21EECEF0DB
:10A3B000DF50386E396A010E3826000E39226000EF
:10A3C000E3F0E6FF6000E7F0E6FF1EEC4BF0600014
:10A3D000B8F0CEF4A9EF51F0F10EE126FF0EE22223
:10A3E0001200070EE66E85EC60F06000BBF0E6FF41
:10A3F0006000BFF0E6FF38EC5FF0080EE66E3FEC61
:10A4000060F06000BBF0E6FF6000BFF0E6FF38ECF4
:10A410005FF085EC60F06000BBF0E6FF6000BFF02D
:10A42000E6FFB4EC5FF03FEC60F06000BBF0E6FFED
:10A430006000BFF0E6FFB4EC5FF07FEC60F0010E6F
:10A44000E66E79EC60F03CEC3CF0060EE66E63ECF8
:10A4500060F06000BBF0E6FF6000BFF0E6FF63EC79
:10A460003FF00250E66E63EC60F06000BBF0E6FF88
:10A470006000BFF0E6FFEDEC5BF0010EE66E5AEC1B
:10A4800060F06000BBF0E6FF6000BFF0E6FF63EC49
:10A490003FF048EC60F06000BBF0E6FF6000BFF00A
:10A4A000E6FF7CEC47F036EC60F06000BBF0E6FFC6
:10A4B0006000BFF0E6FFB1EC46F0120043EC5DF047
:10A4C00048EC60F06000BBF0E6FF6000BFF0E6FF24
:10A4D0008DEC5CF036EC60F06000BBF0E6FF6000F5
:10A4E000BFF0E6FF67EC5CF063EC60F06000BBF08F
:10A4F000E6FF6000BFF0E6FF27EC5BF05AEC60F08F
:10A500006000BBF0E6FF6000BFF0E6FF5FEC5BF0D1
:10A51000000EE66E000EE66E000EE66E000EE66EB3
:10A52000000EE66E000EE66E000EE66E000EE66EA3
:10A53000640EE66E000EE66E5AEC60F06000BBF052
:10A54000E6FF6000BFF0E6FFEDEC5AF0000EE66EAD
:10A55000000EE66E000EE66E000EE66E000EE66E73
:10A56000000EE66E000EE66E000EE66EC80EE66E9B
:10A57000000EE66E5AEC60F06000BBF0E6FF600093
:10A58000BFF0E6FFB3EC5AF012000F0EE126000E0A
:10A59000E222000EE66E81EC51F0F10EE124D96E5C
:10A5A000FF0EE220DA6E0F0E2E6EDD50E552E75000
:10A5B000DF6E2E2EFAD7F10EE350D8B4E2EF52F050
:10A5C000E4EF52F026EF53F0F40EE124D96EFF0EC3
:10A5D000E220DA6EDE50DE10D8B4F1EF52F0F3EF85
:10A5E00052F026EF53F0F20EE124D96EFF0EE22076
:10A5F000DA6EDE50DE10D8B400EF53F002EF53F005
:10A6000026EF53F0F10EE1242E6EFF0EE2202F6EA6
:10A610006000BBF0E6FF6000BFF0E6FFF00EE12453
:10A62000D96EFF0EE220DA6E6F0078FF38F06F000F
:10A6300074FF39F002D826EF53F00500FA6E385057
:10A64000FD6E3950FE6EFF6AFA501200F10EE126DF
:10A65000FF0EE2221200E652ED0EE350E66EA8EC89
:10A660005FF0FF0EE36AFF0EE350110DFA0EF324C4
:10A67000D96E010EF420DA6EDF50D8A442EF53F009
:10A6800044EF53F071EF53F0E150FD0FD96EE250FB
:10A69000DA6EFF0EDA22FF0EE350110DF80EF324EE
:10A6A000E96E010EF420EA6E6F007BFFEEFF6F0093
:10A6B00077FFEDFFEE0EE124D96EFF0EE220DA6E99
:10A6C000FF0EE350110DFA0EF324E96E010EF42093
:10A6D000EA6E0E0E6F006FFFEBFFE806FBE27FEF06
:10A6E00053F0FF0EE32AFF0E6F008CFF2EF0180EC2
:10A6F0002E647DEF53F07FEF53F033EF53F0ED0E08
:10A70000E350E66E9CEC5FF0FF0E6F008CFF2EF0C6
:10A71000ED0EE126FF0EE2221200060EE126000EEB
:10A72000E222F50E6F008CFF36F0F60E6F008CFF04
:10A7300037F0F70E6F008CFF38F0F80E6F008CFFCB
:10A7400039F0FC0E6000DBF0E3FFFD0E6000DFF08F
:10A75000E3FFFE0E6000E3F0E3FFFF0E6000E7F0B2
:10A76000E3FFFB0EE36AF90E6F008CFF2EF0FA0E8A
:10A770006000BBF0E3FFFA0EE3502E6EFB0EE350D9
:10A780002E26FA0E6000BBF0E3FFFB0E6F008CFF7D
:10A7900039F0FC0EE124366EFF0EE220376E3950A0
:10A7A0003624D96E000E3720DA6EDF50E66EF90ED1
:10A7B000E350E66E8FEC5FF0FB0EE32AFB0E6F00BA
:10A7C0008CFF2EF0030E2E64E8EF53F0EAEF53F007
:10A7D000B3EF53F0F50EE126FF0EE2221200060E53
:10A7E000E126000EE222FB0EE36AF90E6F008CFFF9
:10A7F0002EF0FA0E6000BBF0E3FFFA0EE3502E6E6F
:10A80000FB0EE3502E26FA0E6000BBF0E3FFFA0EBB
:10A81000E350E66E51EC60F0FB0E6F008CFF39F0F8
:10A82000FC0EE124366EFF0EE220376E39503624DE
:10A83000D96E000E3720DA6E6000BBF0DFFFFB0E32
:10A84000E32AFB0E6F008CFF2EF0030E2E642BEF1D
:10A8500054F02DEF54F0F5EF53F0FC0E6F008CFF29
:10A860002EF0FD0E6F008CFF2FF0FE0E6F008CFFA0
:10A8700030F0FF0E6F008CFF31F0F90EE126FF0E75
:10A88000E2221200060EE126000EE222F80E6F0010
:10A890008FFFE9FFF90E6F008FFFEAFFFE0E6F00DA
:10A8A000BBFFE3FFFF0E6F00B7FFE3FFFF0EE124E6
:10A8B000D96EFF0EE220DA6EDF50396EFA0E6000BC
:10A8C000E7F0E3FFFB0EE124D96EFF0EE220DA6E23
:10A8D000FE0E6F008FFFDFFFFC0EE124D96EFF0E2E
:10A8E000E220DA6EDF6AFD0EE124D96EFF0EE2206F
:10A8F000DA6EDF6AFA0E6F008FFFE6FF6F008FFFE0
:10A90000E6FF6F008FFFE6FF6F008FFFE6FF010E8F
:10A91000E66E040EE66E9BEC3AF0F80EE126FF0EB2
:10A92000E2221200B80EE66E7B0EE66E0DEC60F0D1
:10A93000A00EE66E520EE66E18EC60F0000EE66EAB
:10A94000000EE66E0C0EE66EBE0EE66E63EC60F078
:10A950006000BBF0E6FF6000BFF0E6FFC0EC57F020
:10A96000000EE66E000EE66E460EE66EAC0EE66E6D
:10A970005AEC60F06000BBF0E6FF6000BFF0E6FF5D
:10A980004AEC57F01450E66E5AEC60F06000BBF0F1
:10A99000E6FF6000BFF0E6FFEDEC5BF0000EE66E58
:10A9A000000EE66EE80EE66EBE0EE66E5AEC60F045
:10A9B0006000BBF0E6FF6000BFF0E6FF85EC57F0FB
:10A9C0001200FE0E6F008FFFD9FFFF0E6F008FFF8A
:10A9D000DAFFDF6AFE0E6F008CFF38F0FF0E6F00AB
:10A9E0008CFF39F0050E3824D96E000E3920DA6E4E
:10A9F000DE6ADD6AFE0E6F008CFF38F0FF0E6F001E
:10AA00008CFF39F0030E3824D96E000E3920DA6E2F
:10AA1000DE6ADD6AFE0E6F008CFF38F0FF0E6F00FD
:10AA20008CFF39F0070E3824D96E000E3920DA6E0B
:10AA3000070EDE6AE806FDE2FE0E6F008CFF38F0BE
:10AA4000FF0E6F008CFF39F0010E3824D96E000E16
:10AA50003920DA6EDE6ADD6AE552E5521200E6520E
:10AA6000E652E652E652FA0E6F008CFF2EF0FC0E14
:10AA70006000BBF0E3FFFD0EE124D96EFF0EE22083
:10AA8000DA6E60005BF0DFFFFE0EE124D96EFF0E90
:10AA9000E220DA6E60005FF0DFFFFF0EE124D96E86
:10AAA000FF0EE220DA6E600063F0DFFFFC0E6F0045
:10AAB0008FFFE6FF6F008FFFE6FF6F008FFFE6FF5F
:10AAC0006F008FFFE6FF000EE66E040EE66E9BEC55
:10AAD0003AF0FA0EE126FF0EE2221200E652E652AA
:10AAE000E652E652FC0EE36AFA0E6F008FFFD9FFC2
:10AAF000FB0E6F008FFFDAFFFD0EE124E96EFF0E03
:10AB0000E220EA6E6F007FFFEFFFFE0EE124D96EB8
:10AB1000FF0EE220DA6EDF6AFF0EE124D96EFF0E2F
:10AB2000E220DA6EDF6AFC0E6F008FFFE6FF6F0037
:10AB30008FFFE6FF6F008FFFE6FF6F008FFFE6FFDE
:10AB4000020EE66E030EE66E9BEC3AF0FA0EE1267C
:10AB5000FF0EE2221200E652D2BEB1EF55F0B5EF81
:10AB600055F0396A392AB6EF55F0396AFF0E6000A0
:10AB7000E7F0E3FFFE0EE124D96EFF0EE220DA6E6D
:10AB8000DF50030B3901E16FFD0E6F008FFFE0F91D
:10AB9000FC0E6F008FFFE3F93F0EE517E585D29EAF
:10ABA000550EE66FAA0EE66FE583E5B3DAEF55F0D2
:10ABB000DCEF55F0D5EF55F0E595FF0EE3B002D090
:10ABC000D29E01D0D28EE552E552E552E5521200F6
:10ABD000E652E652E652E652FC0E60006BF0E3FFEE
:10ABE000FD0EE124D96EFF0EE220DA6E60006FF0F8
:10ABF000DFFFFE0EE124D96EFF0EE220DA6E600068
:10AC000073F0DFFFFF0EE124D96EFF0EE220DA6E53
:10AC1000600077F0DFFFFC0E6F008FFFE6FF6F0034
:10AC20008FFFE6FF6F008FFFE6FF6F008FFFE6FFED
:10AC3000000EE66E060EE66E9BEC3AF0FA0EE1268A
:10AC4000FF0EE2221200E652E652E652E652FC0EF7
:10AC5000600047F0E3FFFD0EE124D96EFF0EE22015
:10AC6000DA6E60004BF0DFFFFE0EE124D96EFF0EBE
:10AC7000E220DA6E60004FF0DFFFFF0EE124D96EB4
:10AC8000FF0EE220DA6E600053F0DFFFFC0E6F0073
:10AC90008FFFE6FF6F008FFFE6FF6F008FFFE6FF7D
:10ACA0006F008FFFE6FF000EE66E020EE66E9BEC75
:10ACB0003AF0FA0EE126FF0EE2221200E150FC0FFC
:10ACC000D96EE250DA6EFF0EDA22FE0E6F008CFFB4
:10ACD00038F0FF0E6F008CFF39F0270E3824E96E34
:10ACE000000E3920EA6E6F007BFFEEFF6F0077FFEA
:10ACF000EDFFE150FA0FD96EE250DA6EFF0EDA2264
:10AD0000FE0E6F008CFF38F0FF0E6F008CFF39F0E5
:10AD1000290E3824E96E000E3920EA6E6F007BFFA1
:10AD2000EEFF6F0077FFEDFFFA0EE126FF0EE22245
:10AD30001200E150FC0FD96EE250DA6EFF0EDA22FB
:10AD4000FE0E6F008CFF38F0FF0E6F008CFF39F0A5
:10AD5000230E3824E96E000E3920EA6E6F007BFF67
:10AD6000EEFF6F0077FFEDFFE150FA0FD96EE25072
:10AD7000DA6EFF0EDA22FE0E6F008CFF38F0FF0E47
:10AD80006F008CFF39F0250E3824E96E000E392053
:10AD9000EA6E6F007BFFEEFF6F0077FFEDFFFA0EAC
:10ADA000E126FF0EE2221200E150FC0FD96EE250C4
:10ADB000DA6EFF0EDA22FE0E6F008CFF38F0FF0E07
:10ADC0006F008CFF39F00C0E3824E96E000E39202C
:10ADD000EA6E6F007BFFEEFF6F0077FFEDFFE15043
:10ADE000FA0FD96EE250DA6EFF0EDA22FE0E6F0015
:10ADF0008CFF38F0FF0E6F008CFF39F00E0E3824F8
:10AE0000E96E000E3920EA6E6F007BFFEEFF6F00E7
:10AE100077FFEDFFFA0EE126FF0EE2221200E1506D
:10AE2000FC0FD96EE250DA6EFF0EDA22FE0E6F00D2
:10AE30008CFF38F0FF0E6F008CFF39F0100E3824B5
:10AE4000E96E000E3920EA6E6F007BFFEEFF6F00A7
:10AE500077FFEDFFE150FA0FD96EE250DA6EFF0E88
:10AE6000DA22FE0E6F008CFF38F0FF0E6F008CFFB1
:10AE700039F0120E3824E96E000E3920EA6E6F00A8
:10AE80007BFFEEFF6F0077FFEDFFFA0EE126FF0E6E
:10AE9000E2221200E150FC0FD96EE250DA6EFF0E92
:10AEA000DA22FE0E6F008CFF38F0FF0E6F008CFF71
:10AEB00039F01F0E3824E96E000E3920EA6E6F005B
:10AEC0007BFFEEFF6F0077FFEDFFE150FA0FD96EC9
:10AED000E250DA6EFF0EDA22FE0E6F008CFF38F0C1
:10AEE000FF0E6F008CFF39F0210E3824E96E000E42
:10AEF0003920EA6E6F007BFFEEFF6F0077FFEDFFFA
:10AF0000FA0EE126FF0EE2221200E150FC0FD96E8C
:10AF1000E250DA6EFF0EDA22FE0E6F008CFF38F080
:10AF2000FF0E6F008CFF39F02B0E3824E96E000EF7
:10AF30003920EA6E6F007BFFEEFF6F0077FFEDFFB9
:10AF4000E150FA0FD96EE250DA6EFF0EDA22FE0EF1
:10AF50006F008CFF38F0FF0E6F008CFF39F02D0E64
:10AF60003824E96E000E3920EA6E6F007BFFEEFF99
:10AF70006F0077FFEDFFFA0EE126FF0EE2221200CE
:10AF8000E150FC0FD96EE250DA6EFF0EDA22FE0EAF
:10AF90006F008CFF38F0FF0E6F008CFF39F02F0E22
:10AFA0003824E96E000E3920EA6E6F007BFFEEFF59
:10AFB0006F0077FFEDFFE150FA0FD96EE250DA6EC5
:10AFC000FF0EDA22FE0E6F008CFF38F0FF0E6F00CE
:10AFD0008CFF39F0310E3824E96E000E3920EA6E0C
:10AFE0006F007BFFEEFF6F0077FFEDFFFA0EE126AB
:10AFF000FF0EE2221200E150F40FD96EE250DA6E39
:10B00000FF0EDA226F007BFFE6FF6F007BFFE6FF9B
:10B010006F007BFFE6FF6F007BFFE6FF6F007BFFAB
:10B02000E6FF6F007BFFE6FF6F007BFFE6FF6F0030
:10B030007BFFE6FFF40E6F008FFFE6FF6F008FFFD0
:10B04000E6FF690EE66ED20EE66E5D0EE66EF10E5E
:10B050006F008FFFE6FF6F008FFFE6FFB5EC49F052
:10B06000F40EE126FF0EE2221200E652E652FC0E3A
:10B070006F008CFF38F0FD0E6F008CFF39F0FF0E73
:10B080006000E7F0E3FFFE0E6000E3F0E3FF000E78
:10B09000E66E000EE66E000EE66E000EE66E000E28
:10B0A000E66E000EE66E000EE66E000EE66E000E18
:10B0B000E66E000EE66E720EE66EC00EE66E660E70
:10B0C000E66EF10E6F008FFFE6FF6F008FFFE6FF69
:10B0D000B5EC49F0E552E552E552E5521200E65270
:10B0E000E652FC0E6F008CFF38F0FD0E6F008CFFF7
:10B0F00039F0FF0E6000E7F0E3FFFE0E6000E3F0C2
:10B10000E3FF000EE66E000EE66E000EE66E000E29
:10B11000E66E000EE66E000EE66E000EE66E000EA7
:10B12000E66E000EE66E000EE66E680EE66ED20E5D
:10B13000E66E5D0EE66EF10E6F008FFFE6FF6F00AC
:10B140008FFFE6FFB5EC49F0E552E552E552E552D6
:10B150001200E150F40FD96EE250DA6EFF0EDA22DF
:10B160006F007BFFE6FF6F007BFFE6FF6F007BFF5A
:10B17000E6FF6F007BFFE6FF6F007BFFE6FF6F00DF
:10B180007BFFE6FF6F007BFFE6FF6F007BFFE6FFC4
:10B19000F40E6F008FFFE6FF6F008FFFE6FF190EC2
:10B1A000E66E060EE66E100EE66EF10E6F008FFF75
:10B1B000E6FF6F008FFFE6FFB5EC49F0F40EE126E5
:10B1C000FF0EE2221200E150F40FD96EE250DA6E67
:10B1D000FF0EDA226F007BFFE6FF6F007BFFE6FFCA
:10B1E0006F007BFFE6FF6F007BFFE6FF6F007BFFDA
:10B1F000E6FF6F007BFFE6FF6F007BFFE6FF6F005F
:10B200007BFFE6FFF40E6F008FFFE6FF6F008FFFFE
:10B21000E6FF1A0EE66E060EE66E100EE66EF10EF4
:10B220006F008FFFE6FF6F008FFFE6FFB5EC49F080
:10B23000F40EE126FF0EE2221200E652E652FC0E68
:10B240006F008CFF38F0FD0E6F008CFF39F0FF0EA1
:10B250006000E7F0E3FFFE0E6000E3F0E3FF000EA6
:10B26000E66E000EE66E000EE66E000EE66E000E56
:10B27000E66E000EE66E000EE66E000EE66E000E46
:10B28000E66E000EE66E700EE66EC00EE66E660EA0
:10B29000E66EF10E6F008FFFE6FF6F008FFFE6FF97
:10B2A000B5EC49F0E552E552E552E5521200E6529E
:10B2B000E652FC0E6F008CFF38F0FD0E6F008CFF25
:10B2C00039F0FF0E6000E7F0E3FFFE0E6000E3F0F0
:10B2D000E3FF000EE66E000EE66E000EE66E000E58
:10B2E000E66E000EE66E000EE66E000EE66E000ED6
:10B2F000E66E000EE66E000EE66E6F0EE66EC00E97
:10B30000E66E660EE66EF10E6F008FFFE6FF6F00D1
:10B310008FFFE6FFB5EC49F0E552E552E552E55204
:10B320001200E652E652FC0E6F008CFF38F0FD0E64
:10B330006F008CFF39F0FF0E6000E7F0E3FFFE0EB8
:10B340006000E3F0E3FF000EE66E000EE66E000E16
:10B35000E66E000EE66E000EE66E000EE66E000E65
:10B36000E66E000EE66E000EE66E000EE66E670EEE
:10B37000E66ED20EE66E5D0EE66EF10E6F008FFF8A
:10B38000E6FF6F008FFFE6FFB5EC49F0E552E552AE
:10B39000E552E5521200E652E652FC0E6F008CFFB9
:10B3A00038F0FD0E6F008CFF39F0FF0E6000E7F003
:10B3B000E3FFFE0E6000E3F0E3FF000EE66E000E1A
:10B3C000E66E000EE66E000EE66E000EE66E000EF5
:10B3D000E66E000EE66E000EE66E000EE66E000EE5
:10B3E000E66E660EE66ED20EE66E5D0EE66EF10E4F
:10B3F0006F008FFFE6FF6F008FFFE6FFB5EC49F0AF
:10B40000E552E552E552E5521200E652E652FC0ED4
:10B410006F008CFF38F0FD0E6F008CFF39F0FF0ECF
:10B420006000E7F0E3FFFE0E6000E3F0E3FF000ED4
:10B43000E66E000EE66E000EE66E000EE66E000E84
:10B44000E66E000EE66E000EE66E000EE66E000E74
:10B45000E66E000EE66E650EE66ED20EE66E5D0ED0
:10B46000E66EF10E6F008FFFE6FF6F008FFFE6FFC5
:10B47000B5EC49F0E552E552E552E5521200E652CC
:10B48000E652FC0E6F008CFF38F0FD0E6F008CFF53
:10B4900039F0FF0E6000E7F0E3FFFE0E6000E3F01E
:10B4A000E3FF000EE66E000EE66E000EE66E000E86
:10B4B000E66E000EE66E000EE66E000EE66E000E04
:10B4C000E66E000EE66E000EE66E710EE66EC00EC3
:10B4D000E66E660EE66EF10E6F008FFFE6FF6F0000
:10B4E0008FFFE6FFB5EC49F0E552E552E552E55233
:10B4F0001200E150F40FD96EE250DA6EFF0EDA223C
:10B500006F007BFFE6FF6F007BFFE6FF6F007BFFB6
:10B51000E6FF6F007BFFE6FF6F007BFFE6FF6F003B
:10B520007BFFE6FF6F007BFFE6FF6F007BFFE6FF20
:10B53000F40E6F008FFFE6FF6F008FFFE6FF180E1F
:10B54000E66E060EE66E100EE66EF10E6F008FFFD1
:10B55000E6FF6F008FFFE6FFB5EC49F0F40EE12641
:10B56000FF0EE2221200E150F40FD96EE250DA6EC3
:10B57000FF0EDA226F007BFFE6FF6F007BFFE6FF26
:10B580006F007BFFE6FF6F007BFFE6FF6F007BFF36
:10B59000E6FF6F007BFFE6FF6F007BFFE6FF6F00BB
:10B5A0007BFFE6FFF40E6F008FFFE6FF6F008FFF5B
:10B5B000E6FF170EE66E060EE66E100EE66EF10E54
:10B5C0006F008FFFE6FF6F008FFFE6FFB5EC49F0DD
:10B5D000F40EE126FF0EE2221200E150F40FD96EC4
:10B5E000E250DA6EFF0EDA226F007BFFE6FF6F009B
:10B5F0007BFFE6FF6F007BFFE6FF6F007BFFE6FF50
:10B600006F007BFFE6FF6F007BFFE6FF6F007BFFB5
:10B61000E6FF6F007BFFE6FFF40E6F008FFFE6FF93
:10B620006F008FFFE6FF160EE66E060EE66E100E3A
:10B63000E66EF10E6F008FFFE6FF6F008FFFE6FFF3
:10B64000B5EC49F0F40EE126FF0EE2221200FE0EE8
:10B65000E350020F386EFF0E6F008CFF39F0000EC2
:10B6600039226000E3F0E6FF6000E7F0E6FFB3ECAC
:10B670005CF0000EE66E000EE66E000EE66E000E4A
:10B68000E66E000EE66E000EE66E000EE66E000E32
:10B69000E66E0A0EE66E000EE66E150EE66E060EFD
:10B6A000E66E100EE66EF10E6F008FFFE6FF6F0084
:10B6B0008FFFE6FFB5EC49F0E552E5521200FE0EB1
:10B6C000E350020F386EFF0E6F008CFF39F0000E52
:10B6D00039226000E3F0E6FF6000E7F0E6FFB3EC3C
:10B6E0005CF0000EE66E000EE66E000EE66E000EDA
:10B6F000E66E000EE66E000EE66E000EE66E000EC2
:10B70000E66E0A0EE66E000EE66E140EE66E060E8D
:10B71000E66E100EE66EF10E6F008FFFE6FF6F0013
:10B720008FFFE6FFB5EC49F0E552E5521200000E3E
:10B73000E66E000EE66E000EE66E000EE66E000E81
:10B74000E66E000EE66E000EE66E000EE66EF40E7D
:10B750006F008FFFE6FF6F008FFFE6FFCB0EE66EF8
:10B76000320EE66E460EE66EF10E6F008FFFE6FFBC
:10B770006F008FFFE6FFB5EC49F0E552E552E55268
:10B78000E5521200000EE66E000EE66E000EE66E4A
:10B79000000EE66E000EE66E000EE66E000EE66E21
:10B7A000000EE66EF40E6F008FFFE6FF6F008FFF56
:10B7B000E6FFC90EE66E320EE66E460EE66EF10E3E
:10B7C0006F008FFFE6FF6F008FFFE6FFB5EC49F0DB
:10B7D000E552E552E552E5521200FE0EE3501E0F0F
:10B7E000386EFF0E6F008CFF39F0000E39226000BA
:10B7F000E3F0F6FF6000E7F0F7FF000EF86EFD0ED5
:10B80000E350396E0F0EF76405D06000E7F0F5FFE6
:10B810000C0009D06F00DBFFE9FF6F00DFFFEAFFDC
:10B820006000E7F0EFFFE552E552E5521200FE0E30
:10B83000E350E66EA8EC5FF0FF0EE350110DF80E3A
:10B84000F324D96E010EF420DA6EDE6ADD6AFF0E93
:10B85000E350110DFA0EF324386E010EF420396E08
:10B860006000E3F0E6FF6000E7F0E6FFE1EC54F093
:10B87000FE0EE350E66E9CEC5FF0E552E5521200DE
:10B88000E652E652E652E652FC0EE36AFF0EE1246F
:10B89000D96EFF0EE220DA6E600057F0DFFFFC0E7B
:10B8A0006F008FFFE6FF6F008FFFE6FF6F008FFFD7
:10B8B000E6FF6F008FFFE6FF000EE66E030EE66EFA
:10B8C0009BEC3AF0FA0EE126FF0EE2221200000E87
:10B8D000E66E000EE66E000EE66E000EE66E000EE0
:10B8E000E66E000EE66E000EE66E000EE66EB80E18
:10B8F000E66E0B0EE66E6E0EE66EC00EE66E660E21
:10B90000E66EF10E6F008FFFE6FF6F008FFFE6FF20
:10B91000B5EC49F0E552E5521200000EE66E000E5D
:10B92000E66E000EE66E000EE66E000EE66E000E8F
:10B93000E66E000EE66E000EE66EB80EE66E0B0EBC
:10B94000E66E640EE66ED20EE66E5D0EE66EF10EEB
:10B950006F008FFFE6FF6F008FFFE6FFB5EC49F049
:10B96000E552E5521200000EE66E000EE66E000E85
:10B97000E66E000EE66E000EE66E000EE66E000E3F
:10B98000E66E000EE66E000EE66E000EE66EC80E67
:10B99000E66E320EE66E460EE66EF10E6F008FFF1B
:10B9A000E6FF6F008FFFE6FFB5EC49F0E552E55288
:10B9B000120000EEF8F120EED7F2EE6ADD50D95019
:10B9C000FCE1DA50FAE100EE00F1F80EEE6AE8066A
:10B9D000FDE100EE60F0110EEE6AE806FDE100EE1A
:10B9E00001F02D0EEE6AE806FDE1080ED56E000EA0
:10B9F000D66E000ED76E000177EF5EF0FE0EE350BC
:10BA0000070F386EFF0E6F008CFF39F0000E3922E1
:10BA10006000E3F0F6FF6000E7F0F7FF000EF86E5D
:10BA20000F0EF76404D0000EF56E0C0008D06F0006
:10BA3000DBFFE9FF6F00DFFFEAFF000EEF6EE5526C
:10BA4000E5521200BA6ABB6ABC6AC26AF60EC36EDD
:10BA5000C4683A016069EE0E506F406B816B516BA8
:10BA6000800E416F616B426B526B626B436953692D
:10BA70006369446954696469080E846F0C0EED6F44
:10BA8000330E0B6F1200000EE66E000EE66E000E17
:10BA9000E66E000EE66E000EE66E000EE66E000E1E
:10BAA000E66E000EE66E000EE66E000EE66E0A0E04
:10BAB000E66E9E0EE66E350EE66E2A0EE66E000E01
:10BAC000E66EB5EC49F01200E652E652FC0E6F004D
:10BAD0008CFF38F0FD0E6F008CFF39F0FF0E600018
:10BAE000E7F0E3FFFE0E6000E3F0E3FFFE0E6F0001
:10BAF0008FFFE6FF6F008FFFE6FF3FEC5AF0E55245
:10BB0000E552E552E5521200E150FC0FD96EE250C9
:10BB1000DA6EFF0EDA22FE0E6F008CFF38F0FF0E99
:10BB20006F008CFF39F0050E3824E96E000E3920C5
:10BB3000EA6E6F007BFFEEFF6F0077FFEDFFE552CF
:10BB4000E552E552E5521200E150FC0FD96EE25089
:10BB5000DA6EFF0EDA22FE0E6F008CFF38F0FF0E59
:10BB60006F008CFF39F0030E3824E96E000E392087
:10BB7000EA6E6F007BFFEEFF6F0077FFEDFFE5528F
:10BB8000E552E552E5521200E150FC0FD96EE25049
:10BB9000DA6EFF0EDA22FE0E6F008CFF38F0FF0E19
:10BBA0006F008CFF39F0010E3824E96E000E392049
:10BBB000EA6E6F007BFFEEFF6F0077FFEDFFE5524F
:10BBC000E552E552E5521200E150FC0FD96EE25009
:10BBD000DA6EFF0EDA22FE0E6F008CFF38F0FF0ED9
:10BBE0006F008CFF39F0010E3824E96E000E392009
:10BBF000EA6E6F007BFFEEFF6F0077FFEDFFE5520F
:10BC0000E552E552E5521200E150FC0FD96EE250C8
:10BC1000DA6EFF0EDA22FE0E6F008CFF38F0FF0E98
:10BC20006F008CFF39F0030E3824E96E000E3920C6
:10BC3000EA6E6F007BFFEEFF6F0077FFEDFFE552CE
:10BC4000E552E552E5521200060EE126000EE22210
:10BC5000F80E6F008CFF38F0F90E6F008CFF39F092
:10BC6000070E3824D96E000E3920DA6E080E2E6EBB
:10BC7000F80E6F007BFFE3FFE8282E2EFAD71200A4
:10BC8000FE0E6F008CFF38F0FF0E6F008CFF39F056
:10BC9000070E3824D96E000E3920DA6E070E2E6E8C
:10BCA000F60E6F008FFFDEFFE82A2E06FAE2F60E90
:10BCB000E126FF0EE2221200E652D2BE62EF5EF0F3
:10BCC00066EF5EF0396A392A67EF5EF0396AFF0E77
:10BCD0006000E7F0E3FFD29E39015B510400FF0EE4
:10BCE000E3B002D0D29E01D0D28EE552120048ECD1
:10BCF0005FF03EEC48F0F1EC51F092EC54F05EEC69
:10BD000052F0860EE66E9C0EE66EC0EC5FF0D28EB0
:10BD10005CEC5EF0C5EC52F088EF5EF00DEF00F0E9
:10BD2000FF0EE124D96EFF0EE220DA6EDF50030B26
:10BD30003901E16FFE0E6F008FFFE0F93F0EE5174E
:10BD4000E58100F000F06E008CF72EF0E552E55230
:10BD500012003901A39F000171517211D8B4B3EFE1
:10BD60005EF0B5EF5EF0C1EF5EF002D8C1EF5EF0BD
:10BD70000500FA6E7151FD6E7251FE6EFF6AFA5047
:10BD800012001200FE0E6F008CFF38F0FF0E6F00E5
:10BD90008CFF39F0030E3824D96E000E3920DA6E8C
:10BDA0006F0078FF2EF06F0074FF2FF0E552E55220
:10BDB0001200FE0E6F008CFF38F0FF0E6F008CFF3C
:10BDC00039F0050E3824D96E000E3920DA6E6F0076
:10BDD00078FF2EF06F0074FF2FF0E552E55212004D
:10BDE000FE0E6F008CFF38F0FF0E6F008CFF39F0F5
:10BDF0001A0E3824D96E000E3920DA6EFD0E6F004F
:10BE00008FFFDFFFE552E552E5521200000EE66EAD
:10BE1000000EE66E000EE66E000EE66E0F0EE66E8B
:10BE2000000EE66E9BEC3AF0E552E5521200460E2B
:10BE3000B96EF90EB76EB66A3901A39F938F180ECB
:10BE4000E66EC10EE66EC0EC5FF0890EB86E1200B1
:10BE5000FE0E6F008FFFD9FFFF0E6F008FFFDAFF1E
:10BE6000FD0E6F008FFFDFFFE552E552E552120035
:10BE7000FE0E6F008FFFD9FFFF0E6F008FFFDAFFFE
:10BE8000FD0E6F008FFFDFFFE552E552E552120015
:10BE90008AEC60F023EC60F022EC5DF02DEC60F0B9
:10BEA00073EC60F017EC5FF0CBEC45F0120002D8B9
:10BEB00063EF5FF00500FA6E2650FD6E2750FE6EB0
:10BEC000FF6AFA5012003901A5931200010EE66EC6
:10BED000FD0E6F008FFFE6FF6F008FFFE6FFF0ECB7
:10BEE0005EF0E552E55212000001666B676B68C0B8
:10BEF0006CF069C06DF06AC06EF06BC06FF0E55217
:10BF0000E5521200FE0E6F008FFFD9FFFF0E6F008B
:10BF10008FFFDAFFDF502E6EE552E5521200FE0E63
:10BF2000E350E66EFE0EE350E66E000EE66EABECFE
:10BF300055F0E552E5521200FF0EE350D8A4A3EFEE
:10BF40005FF0A5EF5FF0A6EF5FF0D28EE552120032
:10BF5000FF0EE350D8A4AFEF5FF0B1EF5FF0B2EFA8
:10BF60005FF0D29EE5521200FE0E6F008FFFE6FFDB
:10BF70006F008FFFE6FF9CEC50F0E552E552120097
:10BF8000FE0E6F008CFF71F0FF0E6F008CFF72F0E1
:10BF9000E552E5521200FE0E6F008CFF62F0FF0EBC
:10BFA0006F008CFF63F0E552E5521200FE0E6F0049
:10BFB0008CFF20F0FF0E6F008CFF21F0E552E55260
:10BFC0001200FE0E6F008CFF60F0FF0E6F008CFF02
:10BFD00061F0E552E5521200FE0E6F008CFF64F036
:10BFE000FF0E6F008CFF65F0E552E5521200FE0E69
:10BFF0006F008CFF24F0FF0E6F008CFF25F0E552E0
:10C00000E5521200FE0E6F008CFF22F0FF0E6F0053
:10C010008CFF23F0E552E5521200FE0E6F008CFFFC
:10C0200026F0FF0E6F008CFF27F0E552E55212005C
:10C03000FE0E6F008CFF2CF0FF0E6F008CFF2DF0BA
:10C04000E552E55212003901C06BC16BC26BC36B84
:10C05000C46BC56BC66BC76B1200600E3901D96F1C
:10C06000DB6BDD6B080EDF6FDE6B1200000E2E6ED9
:10C07000010E2F6EB40E2E26000E2F221200000E7F
:10C080002E6E010E2F6E010E2E26000E2F22120094
:10C09000000E2E6E010E2F6E700E2E26000E2F2219
:10C0A0001200FF0EE350E66E000EE66E90EC5EF0BE
:10C0B000E5521200000E2E6E010E2F6E390E2E2646
:10C0C000000E2F221200000E2E6E010E2F6E020E99
:10C0D0002E26000E2F221200000EE66E000EE66ED7
:10C0E0008FEC5FF012000C0E39015B6F370E5C6F46
:10C0F0001200FF0E6F008CFF2BF0E55212000A0EAB
:10C100002A6E2C6A2D6A2B6A1200000E2E6E010E0A
:10C110002F6E1200D29A12001200120012001200AA
:08C120001200120012001200CF
:020000040020DA
:10000000FFFFFFFFFFFFFFFFFFFFFFFFFFFFFFFF00
:020000040030CA
:0A0000008CFFF7FFA6FFFFFFFFFFD4
:00000001FF
